:020000040800F2
:1000000000500020FD7A0108000000000000000000
:10001000317B0108317B0108317B010800000000C1
:10002000000000000000000000000000317B01081B
:10003000317B010800000000317B0108716D01086F
:10004000317B0108317B0108317B0108317B0108DC
:10005000317B0108317B0108317B0108317B0108CC
:10006000317B0108317B0108317B0108317B0108BC
:10007000317B0108317B0108317B0108317B0108AC
:10008000317B0108317B0108317B0108317B01089C
:10009000317B0108317B0108317B0108317B01088C
:1000A000317B0108317B0108317B0108317B01087C
:1000B000D9710108317B0108317B0108317B0108CE
:1000C000317B0108317B0108317B0108317B01085C
:1000D000317B010855710108317B0108317B010832
:1000E000317B0108317B0108317B010800000000F1
:1000F0000000000000000000000000000000000000
:1001000000000000000000005FF808F100210A2252
:1001100000F070BD00220A2300F0BABC032AC9B265
:1001200070B408D82AB10346121803F8011B934291
:10013000FBD170BC70478218044601E004F8011B33
:1001400014F0030FFAD14FF0013303FB01F31FE06A
:1001500044F8403C44F83C3C44F8383C44F8343CD7
:1001600044F8303C44F82C3C44F8283C44F8243C07
:1001700044F8203C44F81C3C44F8183C44F8143C37
:1001800044F8103C44F80C3C44F8083C44F8043C67
:10019000161B254640343F2EDADC2C4607E044F897
:1001A000103C44F80C3C44F8083C44F8043C161B52
:1001B000254610340F2EF2DC01E045F8043B541BB9
:1001C000032CFADC01E005F8011B9542FBD3B0E7F4
:1001D00010F0030F38B5044612D10368A3F10132C1
:1001E00022EA030313F0803F0AD1031D184653F897
:1001F000042BA2F1013525EA020212F0803FF5D06E
:1002000003782BB1431C184613F8012B002AFAD1AE
:1002100000F0F0F8204638BD80EA010212F0030F2A
:100220003AD110F0030220F0030021F0030150F84E
:1002300004CB08BF51F8043B0DD082F003024FEA13
:10024000C2026FF07F4323FA02F251F8043B4CEAFA
:10025000020C43EA020300BFACF101329C4501BF2E
:1002600022EA0C0212F0803F50F804CB51F8043B14
:10027000F2D04FEA0C604FEA1C2C012828BFB0EBEB
:10028000036F08BF1B0AF4D003F0FF034FEA1060AE
:10029000A0EB0300704700BF10F0030F0AD010F866
:1002A000012B11F8013B012A28BF9A42F4D0A2EB9E
:1002B000030070474DF8045D4DF8044D4FF0010206
:1002C00042EA022242EA024201F0030C21F0030159
:1002D00050F8044B51F8045BBCF1020F26D04BD808
:1002E00024F07F4CBCEB152FA4EB020323EA04039C
:1002F0000DD113EAC21308BF51F8045B0AD18CEA8E
:10030000040CBCEB056F0CD150F8044BE8E74FEA46
:1003100015255CE033F07F4352D10D784FEA146C21
:1003200055E04FEA146C05F0FF0550E04FEA044C2D
:10033000A4EB02034FEA1C4C23EA0403BCEB154F69
:1003400017D113EAC21308BF51F8045B07D18CEA36
:10035000040CBCEB054F08D150F8044BE6E71B0436
:100360002ED10D884FEA144C31E04FEA05454FEA93
:10037000144C4FEA15452AE004F0FF0CBCEB156F56
:10038000A4EB020323EA04030DD113EAC21308BF4E
:1003900051F8045B0AD18CEA040CBCEB052F0AD19E
:1003A00050F8044BE8E74FEA156510E014F0FF0F32
:1003B00006D051F8045B4FEA142C25F07F4506E087
:1003C0004FF000005DF8044B5DF8045B70470CF0E3
:1003D000FF0205F0FF00012828BF904204BF4FEA4A
:1003E0001C2C2D0AF3D0A2EB00005DF8044B5DF845
:1003F000045B704780EA0102844612F0030F4FD17C
:1004000011F0030F32D14DF8044D11F0040F51F8E3
:10041000043B0BD0A3F101329A4312F0803F04BF9A
:100420004CF8043B51F8043B16D100BF51F8044B83
:10043000A3F101329A4312F0803FA4F101320BD1B3
:100440004CF8043BA24312F0803F04BF51F8043B38
:100450004CF8044BEAD023460CF8013B13F0FF0F95
:100460004FEA3323F8D15DF8044B704711F0010FC8
:1004700006D011F8012B0CF8012B002A08BF704799
:1004800011F0020FBFD031F8022B12F0FF0F16BF90
:100490002CF8022B8CF8002012F47F4FB3D1704758
:1004A00011F8012B0CF8012B002AF9D1704700BF7D
:1004B00020F0030110F00300C0F1000051F8043BEC
:1004C00000F1040C4FEACC0C6FF000021CBF22FAC2
:1004D0000CF213434FF0010C4CEA0C2C4CEA0C4C80
:1004E000A3EB0C0222EA030212EACC1204BF51F879
:1004F000043B0430F4D013F0FF0F1FBF013013F49E
:100500007F4F013013F47F0F18BF0130704700BFD9
:1005100041EA000313F0030F0B4670B414BF00242C
:100520000124032A94BF002404F001040546D4B931
:10053000BAB10E782B46013A03F8016B56B1AC1CE8
:100540007AB111F8015F2346013A04F8015C0134E5
:10055000002DF5D12AB19A18002103F8011B93420E
:10056000FBD170BC7047194653F8044BA4F1013617
:1005700026EA040616F0803FDAD1043A45F8044B27
:10058000032A1946EFD8D3E701232DE9F0071D46CA
:1005900000264FF0FF37AC1900EB070C8C420DD250
:1005A0001CF805C010F80480E0452ED2012526462F
:1005B000E31BAC198C4200EB070CF1D34FF001099F
:1005C00000264D464FF0FF3C1360AC1900EB0C08C1
:1005D000A1420ED918F8058010F804A0C2451AD916
:1005E00001252646CCEB0409AC19A14200EB0C080E
:1005F000F0D80CF101000137B8423CBF99463846AB
:10060000C2F80090BDE8F00770470BD001233746D1
:100610001D46F618BFE709D04FF00109B4464D4614
:100620004E44D2E79D4205D00135B4E74D4505D093
:100630000135CAE72B4626460125ACE7A9462646E2
:100640000125C2E72DE9F04FADF5826D81B014466A
:10065000074610460DF580628B460C3219461D4642
:10066000FFF792FF03AE04A901F57E72331F0090DD
:1006700043F8045F9342FBD14DB1681E0023E25C56
:10068000C11A013303AEAB4246F82210F7D1DDF8B0
:100690000C142046009A611800F0FEFA002877D169
:1006A0000099814605F1FF380646C1F10102019229
:1006B0005A46AB4609EB0B0501F1FF3AB818002189
:1006C000AA1A00F0A3FA00284FD1002D00F0C08034
:1006D0007B1903A913F8013C51F82330002B4CD1AE
:1006E000009B9E4228BF334698450FD903EB090172
:1006F000E05C7A18795C884205D038E012F8011F76
:10070000E05C884233D101339845F7D8009A96428D
:1007100080F0A48007EB090214F80A10534612F87F
:100720000A20914204BF0AEB0901791807D095E02D
:1007300014F802C011F8010D844503D113465A1E66
:10074000B342F5D101369E4200F28D80DDF80C6493
:100750002A46B144C6EB0B0609EB0B05B81800217D
:10076000AA1A00F053FA0028AFD0002071E0019AD5
:100770000026914499442A46EEE7002EFAD0DDF88F
:100780000C2493423CBFC2EB0B0306469944F2E7AC
:10079000009E4FF000080099AB1BB34238BF3346B0
:1007A000C1F101026E1E019201F1FF3A5A468946DB
:1007B000AB460133CDF80C3408EB0B05B81800211B
:1007C000AA1A00F023FA0028CFD1002D40D07B19BF
:1007D00003A913F8013C51F82330002B30D1B14567
:1007E00013D208EB090314F80910FA18FB5C9942BC
:1007F00018BF4B4627D14B4604E012F8011FE05CBE
:10080000884220D10133B342F7D3BAF1FF3F5346B8
:100810002CD007EB080C14F80A101CF80A2091429F
:100820000CD10AEB0802BA1804E0E05C12F8011DD2
:10083000884203D1013BF8D260460AE0DDF80C346F
:1008400098442A46B8E701992A4688449844B3E771
:10085000284605B00DF5806DBDE8F08F009B013690
:100860009E427FF673AF07EB0900F2E707EB080C37
:100870006046EEE72DE9F04F8346037885B00C46DD
:10088000002B00F0F9800A78A2B106460131012060
:1008900002E011F8012B8AB1934214BF002000F04E
:1008A000010016F8013F0D46002BF2D12B782BB139
:1008B0004FF0000B584605B0BDE8F08F0028F9D185
:1008C0000BF10100217800F019FA2D1BA5F10102AE
:1008D000534243EB0203002808BF43F001030746DD
:1008E00083B90BEB0508404594BFC0EB08084FF0F7
:1008F00001081F2D08D9414622462B46FFF7A2FECC
:100900008346D7E78346D5E7294603AA2046FFF763
:100910003BFE03996118814620464A4600F0BCF927
:1009200000284FD109F1FF33C9F1010206460192B7
:1009300082464246C84699460AEB050BB818002184
:10094000C2EB0B0200F062F90028B1D1BBF1000F3D
:10095000B0D046452CBF334643469D420FD903EBEA
:100960000A01E05C7A18795C884205D075E012F8DB
:10097000011FE05C884270D101339D42F7D1B04540
:100980007DD907EB0A0214F809104B4612F809202A
:10099000914202BF09EB0A01AC46791806D06EE01D
:1009A000A55C11F8010D854203D113465A1EB342CE
:1009B000F6D1654601369E4267D8039E5A46B24438
:1009C000AE1BB9E7C9F10101C9EB05034246002698
:1009D00009F1FF3A88464B4538BF4B460133039334
:1009E00006EB050BB8180021C2EB0B0200F00EF964
:1009F00000287FF45DAFBBF1000F3FF45BAF4D45C6
:100A000012D906EB090314F80910FA18FB5C994295
:100A100008BF4B4605D026E012F8011FE05C884273
:100A200022D101339D42F7D1BAF1FF3F534628D07E
:100A300007EB060C14F80A101CF80A20914217D193
:100A40000AEB0602BA1804E0E05C12F8011D8842C5
:100A50000ED1013BF8D2E3462CE7019A00269244DE
:100A60005A469A4468E74B4646445A46F618B7E752
:100A7000039B5A46F618B3E70D46012016E7434696
:100A800098E707EB060CE34614E707EB0A0B11E7C0
:100A90002DE9F04F40F23424C2F2000485B01F4625
:100AA0008C4626680B460390029213F8014B3219CC
:100AB0001D4692F801B01BF0080BF6D12D2C73D017
:100AC0002B2C08BF15F8014BD7F1010338BF0023C9
:100AD000102F14BF1A4643F0010232B1302C73D0EC
:100AE0001BB1302C00F083800A27B946BBF1000F00
:100AF00049460CBF6FF0004A4FF0004ACDF804C0E1
:100B0000504600F0AFFA50468846494600F07CF95E
:100B100033190022DDF804C05B78114613F0040F8E
:100B20001ED0303CA74225DD814294BF0023012323
:100B300053EAD2722ED10A1A534243EB02034445C0
:100B4000D4BF002303F00103002B23D109FB014193
:100B500015F8014B012233195B7813F0040FE0D133
:100B600013F0030306D0012B14BF57233723E41AD5
:100B7000A742D9DCB2F1FF3F1BD00846BBF1000F02
:100B800010D1029B1BB152B90299C1F800C005B047
:100B9000BDE8F08F4FF0FF3215F8014BDBE705F1B0
:100BA000FF3CF1E74842ECE715F8014B4FF0010B31
:100BB0008AE70399BBF1000F0CBF6FF000404FF0C4
:100BC000004022230B60DCE72A78A2F17800414242
:100BD00041EB0001582A14BF0A4641F00102002AE5
:100BE0003FF47EAF10276C78B94602357EE70827C0
:100BF000B9467BE730B440F23824C2F200040D4617
:100C0000134601462A46206830BC41E710F0030F26
:100C1000034670B4C9B211D0002A22D003788B42A7
:100C20001DD0013A013005E0DAB110F8014B013A6C
:100C30008C4218D010F0030F0346F5D1032A14D8C4
:100C40007AB1187888420ED0541E5D1C03E015F866
:100C5000016B8E4203D0013C2846F8D2002070BCC4
:100C600070471046FBE71846F9E741EA012646EAD5
:100C70000646184653F8044B86EA0404A4F10135ED
:100C800025EA040414F0803F03D1043A1846032AED
:100C9000EFD80346D4E700BF032A70B404460D46DC
:100CA00026D941EA000313F0030F13D020782B78E4
:100CB000984208BF294606D01EE014F8010F11F82B
:100CC000013F984218D1012A02F1FF32F5D10020EC
:100CD00070BC70470B46044651F8045B50F8046B37
:100CE000AE4204D1043A0446032A0B46F2D81D460C
:100CF0001046002ADAD1EBE7C01AE9E7C9B2F0B42E
:100D0000002950D010F0030F10D00378002B79D0B9
:100D1000994246D0431C05E013F8012B002A3FD02E
:100D200091423ED013F0030F1846F5D1036841EA13
:100D300001270646A3F1013247EA074722EA0302E8
:100D400012F0803F1DD187EA0303A3F1013222EAAA
:100D5000030313F0803F14D1043002E012F0803F0F
:100D60000FD1064650F8043BA3F1013587EA030290
:100D700025EA0303A2F1013413F0803F24EA0202C2
:100D8000ECD033783046002B3CD0994209D0731C0C
:100D900001E0914205D0184613F8012B002AF8D142
:100DA0001046F0BC704710F0030F0CD00378002BF6
:100DB000F7D0431C03E013F8012B002AF1D013F005
:100DC000030F1846F7D102680346A2F1013121EA68
:100DD000020212F0803F0AD10430034650F8042B7F
:100DE000A2F1013121EA020212F0803FF5D01A7817
:100DF0001846002AD5D00133184613F8012B002AD3
:100E0000FAD1CEE71846CCE74A1E08BF7047C0F0BB
:100E10002481884240F21681114200F01781B0FA15
:100E200080F3B1FA81F2A2EB0303C3F11F0304A222
:100E300002EB03134FF000029F4600BFAFF30080A8
:100E4000B0EBC17F00BF42EB020228BFA0EBC17034
:100E5000B0EB817F00BF42EB020228BFA0EB8170A4
:100E6000B0EB417F00BF42EB020228BFA0EB417014
:100E7000B0EB017F00BF42EB020228BFA0EB017084
:100E8000B0EBC16F00BF42EB020228BFA0EBC16014
:100E9000B0EB816F00BF42EB020228BFA0EB816084
:100EA000B0EB416F00BF42EB020228BFA0EB4160F4
:100EB000B0EB016F00BF42EB020228BFA0EB016064
:100EC000B0EBC15F00BF42EB020228BFA0EBC150F4
:100ED000B0EB815F00BF42EB020228BFA0EB815064
:100EE000B0EB415F00BF42EB020228BFA0EB4150D4
:100EF000B0EB015F00BF42EB020228BFA0EB015044
:100F0000B0EBC14F00BF42EB020228BFA0EBC140D3
:100F1000B0EB814F00BF42EB020228BFA0EB814043
:100F2000B0EB414F00BF42EB020228BFA0EB4140B3
:100F3000B0EB014F00BF42EB020228BFA0EB014023
:100F4000B0EBC13F00BF42EB020228BFA0EBC130B3
:100F5000B0EB813F00BF42EB020228BFA0EB813023
:100F6000B0EB413F00BF42EB020228BFA0EB413093
:100F7000B0EB013F00BF42EB020228BFA0EB013003
:100F8000B0EBC12F00BF42EB020228BFA0EBC12093
:100F9000B0EB812F00BF42EB020228BFA0EB812003
:100FA000B0EB412F00BF42EB020228BFA0EB412073
:100FB000B0EB012F00BF42EB020228BFA0EB0120E3
:100FC000B0EBC11F00BF42EB020228BFA0EBC11073
:100FD000B0EB811F00BF42EB020228BFA0EB8110E3
:100FE000B0EB411F00BF42EB020228BFA0EB411053
:100FF000B0EB011F00BF42EB020228BFA0EB0110C3
:10100000B0EBC10F00BF42EB020228BFA0EBC10052
:10101000B0EB810F00BF42EB020228BFA0EB8100C2
:10102000B0EB410F00BF42EB020228BFA0EB410032
:10103000B0EB010F00BF42EB020228BFA0EB0100A2
:10104000104670470CBF012000207047B1FA81F2B2
:10105000C2F11F0220FA02F0704708B14FF0FF30D2
:1010600000F00EB80029F8D02DE90340FFF7CCFEC0
:10107000BDE8064002FB00F3A1EB0301704700BF8F
:10108000704700BF81F0004102E000BF83F00043E1
:1010900030B54FEA41044FEA430594EA050F08BF13
:1010A00090EA020F1FBF54EA000C55EA020C7FEAD7
:1010B000645C7FEA655C00F0E2804FEA5454D4EB54
:1010C0005555B8BF6D420CDD2C4480EA020281EA1E
:1010D000030382EA000083EA010180EA020281EA56
:1010E0000303362D88BF30BD11F0004F4FEA0131A8
:1010F0004FF4801C4CEA113102D0404261EB4101B7
:1011000013F0004F4FEA03334CEA133302D052423C
:1011100063EB430394EA050F00F0A780A4F10104F8
:10112000D5F1200E0DDB02FA0EFC22FA05F2801832
:1011300041F1000103FA0EF2801843FA05F3594118
:101140000EE0A5F120050EF1200E012A03FA0EFC97
:1011500028BF4CF0020C43FA05F3C01851EBE371C1
:1011600001F0004507D54FF0000EDCF1000C7EEBDE
:1011700000006EEB0101B1F5801F1BD3B1F5001F1C
:101180000CD349085FEA30004FEA3C0C04F101043B
:101190004FEA445212F5800F80F09A80BCF1004F64
:1011A00008BF5FEA500C50F1000041EB045141EAE6
:1011B000050130BD5FEA4C0C404141EB010111F4E7
:1011C000801FA4F10104E9D191F0000F04BF014692
:1011D0000020B1FA81F308BF2033A3F10B03B3F170
:1011E00020020CDA0C3208DD02F1140CC2F10C0200
:1011F00001FA0CF021FA02F10CE002F11402D8BF5E
:10120000C2F1200C01FA02F120FA0CFCDCBF41EA29
:101210000C019040E41AA2BF01EB0451294330BDF8
:101220006FEA04041F3C1CDA0C340EDC04F11404D5
:10123000C4F1200220FA04F001FA02F340EA0300AC
:1012400021FA04F345EA030130BDC4F10C04C4F1F2
:10125000200220FA02F001FA04F340EA03002946D2
:1012600030BD21FA04F0294630BD94F0000F83F41C
:10127000801306BF81F480110134013D4EE77FEAFF
:10128000645C18BF7FEA655C29D094EA050F08BF4B
:1012900090EA020F05D054EA000C04BF194610462C
:1012A00030BD91EA030F1EBF0021002030BD5FEA70
:1012B000545C05D14000494128BF41F0004130BD98
:1012C00014F580043CBF01F5801130BD01F00045EC
:1012D00045F0FE4141F470014FF0000030BD7FEA5F
:1012E000645C1ABF194610467FEA655C1CBF0B465A
:1012F000024650EA013406BF52EA033591EA030F71
:1013000041F4002130BD00BF90F0000F04BF002168
:10131000704730B54FF4806404F132044FF000059B
:101320004FF0000150E700BF90F0000F04BF002114
:10133000704730B54FF4806404F1320410F000457A
:1013400048BF40424FF000013EE700BF42004FEA75
:10135000E2014FEA31014FEA02701FBF12F07F43F2
:1013600093F07F4F81F06051704792F0000F14BFEF
:1013700093F07F4F704730B54FF4607401F0004533
:1013800021F0004120E700BF50EA010208BF70478A
:1013900030B54FF000050AE050EA010208BF70477F
:1013A00030B511F0004502D5404261EB41014FF4E8
:1013B000806404F132045FEA915C3FF4DCAE4FF0EC
:1013C00003025FEADC0C18BF03325FEADC0C18BFD3
:1013D000033202EBDC02C2F1200300FA03FC20FA24
:1013E00002F001FA03FE40EA0E0021FA02F1144471
:1013F000C1E600BF70B54FF0FF0C4CF4E06C1CEA86
:1014000011541DBF1CEA135594EA0C0F95EA0C0FFA
:1014100000F0DEF82C4481EA030621EA4C5123EA6D
:101420004C5350EA013518BF52EA033541F480119C
:1014300043F4801338D0A0FB02CE4FF00005E1FB4F
:1014400002E506F00042E0FB03E54FF00006E1FB99
:1014500003569CF0000F18BF4EF0010EA4F1FF04DC
:10146000B6F5007F64F5407404D25FEA4E0E6D411C
:1014700046EB060642EAC62141EA55514FEAC5202D
:1014800040EA5E504FEACE2EB4F1FD0C88BFBCF5A9
:10149000E06F1ED8BEF1004F08BF5FEA500E50F15A
:1014A000000041EB045170BD06F0004646EA010120
:1014B00040EA020081EA0301B4EB5C04C2BFD4EB52
:1014C0000C0541EA045170BD41F480114FF0000E4B
:1014D000013C00F3AB8014F1360FDEBF002001F0B9
:1014E000004170BDC4F10004203C35DA0C341BDC33
:1014F00004F11404C4F1200500FA05F320FA04F005
:1015000001FA05F240EA020001F0004221F0004138
:1015100010EBD37021FA04F642EB06015EEA430EAB
:1015200008BF20EAD37070BDC4F10C04C4F12005DB
:1015300000FA04F320FA05F001FA04F240EA02008E
:1015400001F0004110EBD37041F100015EEA430E5F
:1015500008BF20EAD37070BDC4F1200500FA05F27F
:101560004EEA020E20FA04F301FA05F243EA0203FE
:1015700021FA04F001F0004121FA04F220EA02000D
:1015800000EBD3705EEA430E08BF20EAD37070BD53
:1015900094F0000F0FD101F00046400041EB010133
:1015A00011F4801F08BF013CF7D041EA060195F015
:1015B000000F18BF704703F00046520043EB0303CF
:1015C00013F4801F08BF013DF7D043EA06037047BC
:1015D00094EA0C0F0CEA135518BF95EA0C0F0CD0C7
:1015E00050EA410618BF52EA4306D1D181EA03010D
:1015F00001F000414FF0000070BD50EA410606BF07
:101600001046194652EA430619D094EA0C0F02D14B
:1016100050EA013613D195EA0C0F05D152EA033690
:101620001CBF104619460AD181EA030101F00041AE
:1016300041F0FE4141F470014FF0000070BD41F0F7
:10164000FE4141F4780170BD70B54FF0FF0C4CF4D1
:10165000E06C1CEA11541DBF1CEA135594EA0C0FF0
:1016600095EA0C0F00F0A7F8A4EB050481EA030E3D
:1016700052EA03354FEA013100F088804FEA033324
:101680004FF0805545EA131343EA12634FEA0222F2
:1016900045EA111545EA10654FEA00260EF00041B3
:1016A0009D4208BF964244F1FD0404F5407402D205
:1016B0005B084FEA3202B61A65EB03055B084FEA96
:1016C00032024FF480104FF4002CB6EB020E75EB93
:1016D000030E22BFB61A754640EA0C005B084FEABB
:1016E0003202B6EB020E75EB030E22BFB61A754638
:1016F00040EA5C005B084FEA3202B6EB020E75EB83
:10170000030E22BFB61A754640EA9C005B084FEAFA
:101710003202B6EB020E75EB030E22BFB61A754607
:1017200040EADC0055EA060E18D04FEA051545EAF6
:1017300016754FEA06164FEAC30343EA52734FEA9F
:10174000C2025FEA1C1CC0D111F4801F0BD141EA18
:1017500000014FF000004FF0004CB6E711F4801F7D
:1017600004BF01430020B4F1FD0C88BFBCF5E06F5D
:101770003FF6AFAEB5EB030C04BFB6EB020C5FEA6D
:10178000500C50F1000041EB045170BD0EF0004EC2
:101790004EEA113114EB5C04C2BFD4EB0C0541EAF4
:1017A000045170BD41F480114FF0000E013C90E6F1
:1017B00045EA060E8DE60CEA135594EA0C0F08BFB5
:1017C00095EA0C0F3FF43BAF94EA0C0F0AD150EAB4
:1017D00001347FF434AF95EA0C0F7FF425AF104647
:1017E00019462CE795EA0C0F06D152EA03353FF46F
:1017F000FDAE1046194622E750EA410618BF52EAEC
:1018000043067FF4C5AE50EA41047FF40DAF52EABF
:1018100043057FF4EBAE12E74FF0FF3C06E000BF5C
:101820004FF0010C02E000BF4FF0010C4DF804CD69
:101830004FEA410C7FEA6C5C4FEA430C18BF7FEA29
:101840006C5C1BD001B050EA410C0CBF52EA430C57
:1018500091EA030F02BF90EA020F0020704710F1D7
:10186000000F91EA030F58BF994208BF90422CBF66
:10187000D8176FEAE37040F0010070474FEA410C5F
:101880007FEA6C5C02D150EA013C07D14FEA430C7D
:101890007FEA6C5CD6D152EA033CD3D05DF8040BEE
:1018A000704700BF8446104662468C461946634620
:1018B00000E000BF01B5FFF7B7FF002848BF10F1F7
:1018C000000F01BD4DF808EDFFF7F4FF0CBF01203C
:1018D00000205DF808FB00BF4DF808EDFFF7EAFFB8
:1018E00034BF012000205DF808FB00BF4DF808ED73
:1018F000FFF7E0FF94BF012000205DF808FB00BF68
:101900004DF808EDFFF7CEFF94BF012000205DF8F1
:1019100008FB00BF4DF808EDFFF7C4FF34BF0120FE
:1019200000205DF808FB00BF4FEA410212F50012EB
:1019300015D211D56FF47873B3EB625212D94FEA16
:10194000C12343F0004343EA505311F0004F23FA00
:1019500002F018BF404270474FF00000704750EA55
:10196000013005D111F0004008BF6FF00040704712
:101970004FF00000704700BF4A0011D212F500126C
:1019800011D20DD56FF47873B3EB62520ED44FEAD7
:10199000C12343F0004343EA505323FA02F0704757
:1019A0004FF00000704750EA013002D14FF0FF3095
:1019B00070474FF0000070474FEA4102B2F1E04338
:1019C00024BFB3F5001CDCF1FE5C0DD901F0004C26
:1019D0004FEAC0024CEA5070B2F1004F40EB830076
:1019E00008BF20F00100704711F0804F21D113F1A2
:1019F0003872BCBF01F00040704741F480114FEADB
:101A00005252C2F11802C2F1200C10FA0CF320FA63
:101A100002F018BF40F001004FEAC1234FEAD32380
:101A200003FA0CFC40EA0C0023FA02F34FEA4303EA
:101A3000CCE77FEA625307D150EA01331EBF4FF073
:101A4000FE4040F44000704701F0004040F0FE408E
:101A500040F40000704700BF80F0004002E000BF8B
:101A600081F0004142001FBF5FEA410392EA030F89
:101A70007FEA226C7FEA236C6AD04FEA1262D2EBD3
:101A80001363C1BFD218414048404140B8BF5B42D8
:101A9000192B88BF704710F0004F40F4000020F071
:101AA0007F4018BF404211F0004F41F4000121F087
:101AB0007F4118BF494292EA030F3FD0A2F10102D1
:101AC00041FA03FC10EB0C00C3F1200301FA03F10F
:101AD00000F0004302D5494260EB4000B0F5000F32
:101AE00013D3B0F1807F06D340084FEA310102F1F1
:101AF0000102FE2A51D2B1F1004F40EBC25008BFA3
:101B000020F0010040EA03007047490040EB00006C
:101B100010F4000FA2F10102EDD1B0FA80FCACF19B
:101B2000080CB2EB0C0200FA0CF0AABF00EBC2509A
:101B300052421843BCBFD0401843704792F0000F88
:101B400081F4000106BF80F400000132013BB5E7DB
:101B50004FEA41037FEA226C18BF7FEA236C21D051
:101B600092EA030F04D092F0000F08BF08467047B6
:101B700090EA010F1CBF0020704712F07F4F04D184
:101B8000400028BF40F00040704712F100723CBF97
:101B900000F50000704700F0004343F0FE4040F4C1
:101BA000000070477FEA226216BF08467FEA23637F
:101BB0000146420206BF5FEA412390EA010F40F46A
:101BC000800070474FF0000304E000BF10F00043B6
:101BD00048BF40425FEA000C08BF704743F096439D
:101BE00001464FF000001CE050EA010208BF7047B8
:101BF0004FF000030AE000BF50EA010208BF70473F
:101C000011F0004302D5404261EB41015FEA010C53
:101C100002BF84460146002043F0B64308BFA3F14B
:101C20008053A3F50003BCFA8CF2083AA3EBC2532D
:101C300010DB01FA02FC634400FA02FCC2F120024C
:101C4000BCF1004F20FA02F243EB020008BF20F083
:101C50000100704702F1200201FA02FCC2F12002E9
:101C600050EA4C0021FA02F243EB020008BF20EADE
:101C7000DC7070474FF0FF0C1CEAD0521EBF1CEA0C
:101C8000D15392EA0C0F93EA0C0F6FD01A4480EAFA
:101C9000010C400218BF5FEA41211ED04FF00063E3
:101CA00043EA501043EA5111A0FB01310CF000400F
:101CB000B1F5000F3EBF490041EAD3715B0040EA35
:101CC000010062F17F02FD2A1DD8B3F1004F40EB05
:101CD000C25008BF20F00100704790F0000F0CF0D8
:101CE000004C08BF49024CEA502040EA51207F3A9C
:101CF000C2BFD2F1FF0340EAC250704740F4000077
:101D00004FF00003013A5DDC12F1190FDCBF00F067
:101D100000407047C2F10002410021FA02F1C2F115
:101D2000200200FA02FC5FEA310040F1000053EAB1
:101D30004C0308BF20EADC70704792F0000F00F0FF
:101D4000004C02BF400010F4000F013AF9D040EA05
:101D50000C0093F0000F01F0004C02BF490011F499
:101D6000000F013BF9D041EA0C018FE70CEAD15397
:101D700092EA0C0F18BF93EA0C0F0AD030F0004C17
:101D800018BF31F0004CD8D180EA010000F00040CB
:101D9000704790F0000F17BF90F0004F084691F089
:101DA000000F91F0004F14D092EA0C0F01D14202C3
:101DB0000FD193EA0C0F03D14B0218BF084608D18C
:101DC00080EA010000F0004040F0FE4040F40000D6
:101DD000704740F0FE4040F4400070474FF0FF0C69
:101DE0001CEAD0521EBF1CEAD15392EA0C0F93EAB0
:101DF0000C0F69D0A2EB030280EA010C49024FEA02
:101E0000402037D04FF0805343EA111143EA1013BA
:101E10000CF000408B4238BF5B0042F17D024FF472
:101E2000000C8B4224BF5B1A40EA0C00B3EB510F4D
:101E300024BFA3EB510340EA5C00B3EB910F24BF36
:101E4000A3EB910340EA9C00B3EBD10F24BFA3EBBB
:101E5000D10340EADC001B0118BF5FEA1C1CE0D183
:101E6000FD2A3FF650AF8B4240EBC25008BF20F036
:101E7000010070470CF0004C4CEA50207F32C2BF8A
:101E8000D2F1FF0340EAC250704740F400004FF027
:101E90000003013A37E792F0000F00F0004C02BF58
:101EA000400010F4000F013AF9D040EA0C0093F022
:101EB000000F01F0004C02BF490011F4000F013B7C
:101EC000F9D041EA0C0195E70CEAD15392EA0C0FE4
:101ED00008D142027FF47DAF93EA0C0F7FF470AF1C
:101EE000084676E793EA0C0F04D14B023FF44CAF5F
:101EF00008466EE730F0004C18BF31F0004CCAD1F4
:101F000030F000427FF45CAF31F000437FF43CAF2F
:101F10005FE700BF4FF0FF3C06E000BF4FF0010C51
:101F200002E000BF4FF0010C4DF804CD4FEA400233
:101F30004FEA41037FEA226C18BF7FEA236C11D07D
:101F400001B052EA530C18BF90EA010F58BFB2EB30
:101F5000030088BFC81738BF6FEAE17018BF40F0B0
:101F6000010070477FEA226C02D15FEA402C05D164
:101F70007FEA236CE4D15FEA412CE1D05DF8040BE9
:101F8000704700BF844608466146FFE70FB5FFF77C
:101F9000C9FF002848BF10F1000F0FBD4DF808ED34
:101FA000FFF7F4FF0CBF012000205DF808FB00BF25
:101FB0004DF808EDFFF7EAFF34BF012000205DF87F
:101FC00008FB00BF4DF808EDFFF7E0FF94BF0120CC
:101FD00000205DF808FB00BF4DF808EDFFF7D2FFC9
:101FE00094BF012000205DF808FB00BF4DF808ED0C
:101FF000FFF7C8FF34BF012000205DF808FB00BFD9
:102000004FEA4002B2F1FE4F0FD34FF09E03B3EB05
:1020100012620DD94FEA002343F0004310F0004F45
:1020200023FA02F018BF404270474FF0000070479B
:1020300012F1610F01D1420205D110F0004008BF3A
:102040006FF0004070474FF00000704738B5012036
:10205000FF21074DA8474FF6FF740120FF21A84735
:10206000FF2803D014B1013CA4B2F6E738BD00BF8D
:10207000256F0108F8B504460F464FF6FF7501209D
:10208000FF21164EB047FF2803D115B3013DADB275
:10209000F5E7FE281FD1FF210120B047FF21207066
:1020A0000120B047FF2160700120B047FF21A070E0
:1020B0000120B047043FBFB2E070084D0434002F48
:1020C000E9D1FF210120A8470120FF21A8470120D5
:1020D000F8BD2846F8BD0020F8BD00BF256F0108F7
:1020E000F8B5174B06460C469847FF2823D1FE3813
:1020F0002146144FB847FD2C1FD00024315D01202C
:10210000B8473319012059780234B847B4F5007F35
:102110000C4DF3D1FF210120A847FF210120A84742
:102120000120FF21A84700F01F00A0F1050358423D
:1021300040EB0300F8BD0020F8BD0120F8BD00BF52
:102140004D200008256F010810F0800F70B504467F
:102150000E4607D0772000211F4B984701283AD818
:1021600004F07F0401201D4B984701201C4B984729
:102170001C4B9847FF282DD11B4DFE382146A84700
:10218000310E0120A847310C0120C9B2A847310AFD
:102190000120C9B2A8470120F1B2A847402C04D0C1
:1021A000482C0CBF8721012100E095210120A84780
:1021B0004C2C03D10120FF210B4B98470A2401200E
:1021C000FF21A84710F0800F05D0013CE4B2002C9D
:1021D000F5D170BDFF2070BD49210008296F0108AD
:1021E0002B6F01084D200008256F01082DE9F347EA
:1021F000002840F0B9805E4B1A681D4612F0020FAD
:1022000001D01868B1E05B4BFA2098475A4E012084
:10221000B0470120594B9847FA24B146584E013C2B
:102220000120FF21E4B2B047B046002CF6D1402097
:102230002146544EB047012882466BD148204FF4C6
:10224000D571B0470128504F39D120464F49B84782
:102250000120FF21C04701AB18550134042CF7D1F0
:102260009DF80630012B52D19DF80730AA2B4ED194
:102270004FF6FF74013CA4B24FF6FF739C4207D0A7
:10228000E9204FF08041B0470028F3D1002C41D025
:102290007A200021B047002839D104460120FF21CF
:1022A000C04701AB18550134042CF7D19DF8044008
:1022B00004F04004002C0CBF04240C242AE0E92084
:1022C0002146B047012806D820463149B8470224A4
:1022D0004FF0E90A05E020462E49B84754464FF032
:1022E000410A4FF6FF77013FBFB24FF6FF739F429F
:1022F00005D050460021B0470028F4D14FB15020FE
:102300004FF40071B047002818BF002402E00024F9
:1023100000E03C46204B01201C70C8470120FF21F3
:10232000C0473CB12B68012023F001032B601B4BFD
:10233000984717E0144B2046194998472B6813F02B
:10234000010F0BD10120174B9847174B98470120DD
:10235000094B98470120FF21094B98472B6843F010
:1023600001032B60286800E00120BDE8FC8700BF66
:1023700000000020896B0108296F0108236F010804
:10238000256F010849210008917001086C8401083B
:102390007C8401088C8401082C030020216F010833
:1023A0009B8401082B6F01084D20000810B9024BD7
:1023B00018687047012070470000002070B50C4677
:1023C0001D461146002839D1002B37D01D4B1B6804
:1023D00013F0010F34D11C4B1C4E1B7813F0080F67
:1023E00008BF5102012D0CD15120B047D8B9204669
:1023F0004FF40071164B9847D0F1010538BF002506
:1024000011E05220B04770B920464FF40071104BD4
:10241000984728B1013DEDB215B104F50074F3E71A
:102420004C200021B04701200A4B98470120FF2192
:10243000094B9847281E18BF012070BD042070BDAD
:10244000032070BD000000202C030020492100085B
:1024500075200008296F0108256F0108F8B50C46A2
:1024600015461E46002846D1002B44D0254B1A683D
:1024700012F0010F41D11B6813F0040F3FD1224B22
:10248000224F1B7813F0080F08BF6D02012E0CD1EC
:1024900058202946B84718BBFE2120461C4B9847B8
:1024A000D0F1010638BF00261AE013F0060F02D063
:1024B000D7203146B84759202946B84780B9204629
:1024C000FC21134DA84728B1013EF6B216B104F520
:1024D0000074F4E70020FD21A847002808BF01266A
:1024E00001200C4B98470120FF210B4B9847301ED1
:1024F00018BF0120F8BD0420F8BD0320F8BD02205C
:10250000F8BD00BF000000202C0300204921000876
:10251000E1200008296F0108256F0108F0B5154674
:1025200085B0002840F0F780042905D11478022CEA
:102530008CBF04240024F1E07A4B1B6813F0010FD8
:1025400040F0EB80784E0E2900F2DB80DFE811F0DE
:102550000F00190055005900D900D900D900D90041
:10256000D900D900AA00AF00B100B900C80001200D
:102570006E4B98476E4B9847B0F1FF0418BF01248B
:10258000C2E0492000216B4B98470446002840F0E8
:10259000BA8068461021684B9847002800F0B38045
:1025A0009DF800309B09012B9DF8083007D19DF85C
:1025B00009201B020132D3189BB29B0270E09DF8E8
:1025C00007209DF80510920002EB93139DF806205A
:1025D000013302F0030292029B189DF80A2001F0D9
:1025E0000F0101EBD2119DF80920023102F0030224
:1025F00001EB4202093A934052E04FF4007313801A
:1026000053E04E4C4B4B217811F004011CD0CD20EF
:1026100000219847002876D1FF210130B047684655
:102620001021454B984700286DD03024013C0120F3
:10263000FF21E4B2B047002CF8D19DF80A301022F7
:102640001B0912FA03F32BE049209847074600289C
:1026500059D168461021384B9847002853D0247828
:102660009DF80A2014F002049DF80B300DD09DF85F
:102670000D10DB09013302F03F02890903EB42022E
:1026800001398A403C462A603EE0590902F07C024A
:102690009208013103F00303013201EBC3035343FA
:1026A0002B6031E0254B1B78137000242CE049206F
:1026B00000E04A2000211F4B984720BB28461021EC
:1026C00018E07A2000211B4B9847E0B9044601200E
:1026D000FF21B04728550134042CF8D1043C13E005
:1026E000CD200021134B984768B9FF210130B04736
:1026F00028464021104B9847D0F1010438BF0024F0
:1027000002E0042400E0012401200D4B9847012041
:10271000FF21B04702E0042400E00324204605B076
:10272000F0BD00BF00000020256F01082B6F0108DD
:102730004D20000849210008752000082C030020C6
:10274000296F010808B500200349044B9847003859
:1027500018BF012008BD00BFD40600208D3D000831
:1027600030B5ADF5137D81A81549164B984708BBC8
:10277000012401AB90934FF40073919381A88AA92F
:10278000114B9847B8B99DF83132A3B18CA80130EC
:102790000E490F4DA84750B98CA801300D49A847E4
:1027A00028B98CA801300C49A8470028E1D0013491
:1027B000E4B2DEE7012420460DF5137D30BD00BFF5
:1027C000EA8401086D430008E5430008B08401086D
:1027D00075080008B5840108BA8401082DE9F041A4
:1027E0009846ADF5127D00230C46137081A81E4952
:1027F0001E4B1546984700282BD1064601AB9093F7
:102800004FF40073919381A88AA9194B984700BB94
:102810009DF83132EBB18CA801301649164FB847FC
:1028200050B98CA801301549B84728B98CA8013097
:102830001349B8470028E1D0B44207D18CA92846F3
:10284000013142460F4B9847022008E00136F6B2AC
:10285000D4E728460C4942460A4B984704200DF518
:10286000127DBDE8F08100BFEA8401086D430008D5
:10287000E5430008B084010875080008B584010824
:10288000BA84010811050008BF8401082DE9F04150
:102890000020ADF50E7D0D46224C23491746984683
:1028A000A04700202946A04700202049A04702A8B1
:1028B000294601221E4B98470646002829D11D496A
:1028C000A0478CAB39461C4D02A842460633A847A8
:1028D0001A4F054630B130461949A04702A8B847FB
:1028E00030461AE002A8B84701232A46BDF936123D
:1028F00000938BA82B46134EB04728461249A04799
:1029000028468BA9A04728460849A047BDF83602AB
:1029100003E000200D49A04700200DF50E7DBDE825
:10292000F08100BF91700108C7840108E8840108A4
:10293000AD3D0008DC840108293F00085943000828
:10294000EB84010865520008FF8401080C8501082A
:102950002DE9F0431D46ADF52B7D002306460F46BD
:10296000137099A82649274B1446984700283CD154
:10297000804600ABA8934FF40073A99399A8A2A92D
:10298000214B9847002830D19DF89132002B2CD054
:10299000A4A801301D49DFF89090C84750B9A4A8F9
:1029A00001301B49C84728B9A4A801301949C847B4
:1029B0000028DED0474513D10A20174B9847A4A919
:1029C00001312923304680AA144EB047204686A9FB
:1029D0002A46134B98479DF828023C280BD104E067
:1029E00008F101085FFA88F8C3E720460D492A4636
:1029F0000B4B98473C200DF52B7DBDE8F08300BFC5
:102A0000EA8401086D430008E5430008B08401082A
:102A1000B5840108BA840108896B01088D28000873
:102A200011050008BF840108750800082DE9F0436E
:102A30000020ADF50B7D0F46254C264916461D4658
:102A4000A04700203946A04700202349A047DFF8CF
:102A5000B090684639460A22C847804648B10020EF
:102A60001E49A047684639460A22C84780460028C2
:102A700025D11B49A04788AB684631462A46063314
:102A8000184FB847814618B91749A0474D460FE07F
:102A900040461649A04788AB2A4668463146063369
:102AA000B847054608B9104901E011494046A0471A
:102AB0006846104B984768460F4B984703E0002044
:102AC0000E49A047012528460DF50B7DBDE8F08392
:102AD000917001081E850108E88401085A850108E3
:102AE00026850108CD400008318501083E85010892
:102AF0004A850108A1420008594300086B85010876
:102B0000AD3D000838B500200D460A4C0A49A047E3
:102B100029460020A04700200849A0472846084B26
:102B20009847054618B90749A047284638BD0120EF
:102B300038BD00BF9170010879850108E88401085B
:102B4000554400088285010803E011F8013B00F8B4
:102B5000013B013AF9D2704701E000F8011B013A4C
:102B6000FBD2704710F8013B0BB18B42FAD11846EB
:102B70007047002302461846410841EAC010D15C64
:102B8000013340180B2B00F0FF00F5D17047000017
:102B9000F8B503690D460931002B4DD043690C4649
:102BA0001F7B00269A5D2146202A12D0052A08BFE5
:102BB000E52217F0080F06D0A2F14101C9B2192988
:102BC00001D82032D2B2013604F8012B082E21465A
:102BD000E8D11A7A202A18D022462E2102F8011BA9
:102BE00008269C5D1146202C0FD017F0100F06D040
:102BF000A4F14101C9B2192901D82034E4B2013647
:102C000002F8014B0B2E1146EBD1DA7A2A729A7F29
:102C1000DC7F120442EA04621C7F22435C7F42EAAA
:102C200004222A605C7E1A7E42EA0422AA80DA7DAF
:102C30009B7D43EA0223EB8000240C70AE69F6B161
:102C40000369ABB1028C4FF6FF739A4215D0C76986
:102C500009E000210A4B984760B1EB69013B9C42B7
:102C60000ADA3055013437F8020B0028F1D104E0BC
:102C70001C4602E0044600E0002400233355F8BD62
:102C8000254500082DE9F843C56A04468D420E46E5
:102C90002AD00379E3B100F13008194F407841465A
:102CA0002A460123B847B94608BBA269236A2071A6
:102CB000D3189D420CD2E77808E0A3696078ED183C
:102CC00041462A460123C847013FFFB2012FF4D8ED
:102CD00086B1607804F1300132460123094DA847DE
:102CE00058B9E662BDE8F8830020BDE8F88301200A
:102CF000BDE8F8833046BDE8F8830120BDE8F883DD
:102D00005D240008BD23000838B504460A46407813
:102D100004F1300101231C4DA84780BB94F82E32EA
:102D200094F82F2243EA0222184B12B29A4228D179
:102D300094F8682094F86930120442EA036294F827
:102D400066301A4394F8673042EA0322104B22F0AF
:102D50007F429A4216D094F8840094F885200004AB
:102D600040EA026094F88220104394F8832040EAFD
:102D7000022020F07F40C01A18BF012038BD032078
:102D800038BD022038BD00BFBD23000855AAFFFF93
:102D90004641540070B500212B4B04469847054628
:102DA00000284FD12378032B44D16379002B41D0E5
:102DB00004F13006E062294630464FF40072234B9E
:102DC0009847552384F82E32DB1884F82F32583B6D
:102DD00084F8303084F831300F3384F8323084F89E
:102DE00017322369412284F8332084F816221A0A04
:102DF00084F8183284F819221A0C1B0E84F81B323E
:102E0000E36884F81A221A0A722184F81C3284F8C2
:102E10001D221A0C1B0E84F8141284F8151284F863
:102E20001E2284F81F323146607862690123084E01
:102E3000B0476571002160780A46064B9847003814
:102E400018BF012070BD00BF852C0008592B000859
:102E50005D2400081D25000808B560B1037853B152
:102E6000C3888B4209D14078054B984710F0010088
:102E700018BF032008BD092008BD092008BD00BFF8
:102E8000AD23000801292DE9F84304460D465DD91C
:102E9000C36999425AD20378066A022B2CD0032BBD
:102EA0003AD0012B55D18FB207EB5707BFB206EBD3
:102EB0005721DFF8B080C04700284AD1FB05013711
:102EC000DB0DBFB2E318204606EB572193F8309094
:102ED000C04700283DD1FF05FF0DE71997F83000E6
:102EE00015F0010F49EA002002D00009BDE8F8837F
:102EF0000005000DBDE8F88306EB1121194B98473A
:102F000038BB2D0604EBD55494F8310094F83030DA
:102F100043EA0020BDE8F88306EBD111114B984736
:102F2000D8B96D0604EBD55494F8320094F83330D8
:102F3000000440EA036094F8303094F8319018436C
:102F400040EA092020F07040BDE8F8830120BDE888
:102F5000F8834FF0FF30BDE8F8834FF0FF30BDE855
:102F6000F88300BF852C000801292DE9F8430446A9
:102F70000D46164673D9C369994273D20378076A1E
:102F8000022B45D0032B51D0012B63D11FFA81F8BE
:102F900008EB58081FFA88F8DFF8D09007EB5821A3
:102FA000C8474B46002856D14FEAC852D20D15F0FB
:102FB0000105F1B206D0A01890F8300000F00F0023
:102FC00040EA0111A21808F1010882F830101FFA36
:102FD00088F801222271204607EB582198470028E3
:102FE00039D14FEAC8584FEAD8580DB136090AE02E
:102FF00004EB080393F83030360A23F00F0306F091
:103000000F0643EA060604EB080383F8306022E06B
:1030100007EB1121154B9847E8B92D0604EBD55560
:1030200085F83060360A85F8316014E007EBD1117D
:103030000E4B984778B96D0604EBD555330A85F8E1
:10304000306085F83130330C360E85F8323085F833
:10305000336000E0022001232371BDE8F8830220E1
:10306000BDE8F8830220BDE8F88300BF852C000886
:103070002DE9F0410546D0F81C800E4629B9C768F5
:103080005FB1474528BF012708E0214B9847012839
:1030900031D940453AD3374600E001273C46013458
:1030A000444502D3012F29D9022428462146184B32
:1030B000984738B1B0F1FF3F28D0012826D0BC4254
:1030C000EDD11BE0284621466FF07042114FB84702
:1030D000B8B926B1284631462246B84788B92B6987
:1030E000EC60B3F1FF3F10D0013B2B6101236B710A
:1030F0002046BDE8F0810120BDE8F0810020BDE858
:10310000F0814FF0FF30BDE8F0812046BDE8F0814E
:10311000852E0008692F0008012970B504460E4667
:1031200023D9C36999421AD31FE020463146114B77
:1031300098470546C0B1012817D0B0F1FF3F16D01F
:103140002046314600220C4B984788B92369B3F1D9
:10315000FF3F03D001332361012363712E46E369EE
:103160009E42E2D3002070BD70BD022070BD0120E0
:1031700070BD00BF852E0008692F0008C3690239A1
:10318000023B994204D28278836A02FB0130704785
:103190000020704770B50D46C18081680446012942
:1031A00039D00368DA69914235D271B91A78032AA5
:1031B00001D1596A49B90022E2601A89AA422AD982
:1031C0005B6A03EB151323611AE09E7836010EE06B
:1031D0002068134B9847B0F1FF3F014619D00128F2
:1031E00019D92368DB69984217D2AD1BADB2B5423D
:1031F000EED2E16020680B4B984700EB1510206180
:10320000236805F00F0530336D015D1965610020FD
:1032100070BD012070BD022070BD022070BD00BFD6
:10322000852E00087D3100082DE9F843C688044644
:103230000136B6B20F46002E6BD00369002B68D062
:1032400016F00F0F5AD1C16801330361006819B934
:103250000389B34252D85CE08378013B13EA16132A
:103260004CD1334B98470128054658D9B0F1FF3F60
:1032700058D02068C3699D423AD3002F49D0E168F5
:103280002C4B98470546002846D0012847D0B0F17E
:10329000FF3F47D020680021DFF8A480C0470746E1
:1032A00000283FD12068394630304FF40072224B5D
:1032B0009847D4F8009029464846204B9847C9F8CB
:1032C0002C000EE04FF0010983F8049020680021E3
:1032D000C047002829D123684F44DA6AFFB24A4424
:1032E000DA6223689A78BA42ECD8DA6AD71BDF62CE
:1032F000E56020682946114B984720612368E680E5
:1033000006F00F06303376019E1966610020BDE895
:10331000F8830420BDE8F8830720BDE8F883022085
:10332000BDE8F8830120BDE8F8834846BDE8F8838E
:10333000852E000871300008592B00087D310008E7
:10334000852C00082DE9F74F4D4B00210546984785
:103350008046002840F08D80FF2634462868296981
:10336000484B98478046002840F083806F693B783F
:10337000002B7CD0E52BFA7A6FD002F03F0212F0DE
:10338000080F02D00F2A68D101E00F2A4FD1D5F8DB
:103390001CB0BBF1000F61D013F0400F05D0EA88DC
:1033A0007E7B03F0BF042A8401E0A34255D17B7BDE
:1033B000B34252D197F800800D2308F0BF0808F1FE
:1033C000FF3803FB08F84FF001094FF0000A2E4BBD
:1033D00013F80A30FA185078FB5C43EA0020B9F180
:1033E000000F0FD0294B01939847B8F1FE0F81468B
:1033F000019B32DC3BF81800984781452DD108F13C
:10340000010803E04FF6FF73984226D10AF1010A42
:10341000BAF10D0FDBD13B7813F0400F2CD0B9F18E
:10342000000F29D03BF81830002B25D015E024B927
:103430003846174B984786421BD04FF0FF33AA6996
:103440002B84D37A13F0010302D006E00B2B10D0AB
:10345000F85CD15C01338842F8D0FF242846002173
:103460000C4B9847804600283FF478AF01E04FF0BE
:1034700004084046BDE8FE8F013CE4B2EEE700BF21
:1034800095310008852C0008B685010861450008C3
:10349000732B0008293200082DE9F04F0B7885B016
:1034A0002F2B06460F4601D05C2B00D1013700249C
:1034B000B4603B781F2B05D8304621468B4B98478C
:1034C00074610FE10297D6F81CB000255F46D8461C
:1034D000029905F10109485D1F281BD92F281DD02D
:1034E0005C281BD0B9F5807F00F0F9800121804B6A
:1034F00098470446002800F0F2807F2806D87D48CF
:1035000021467D4B9847002840F0E98028F8024B7F
:103510004D46DDE7CDF80490042402E0CDF8049098
:1035200000240BEB450306E033F8022D202A01D0DE
:103530002E2A03D1013D002DF6D1D0E000222BF838
:103540001520B06920210B226C4B98474FF00009E1
:1035500001E009F1010937F8023B202BF9D02E2BAD
:10356000F7D0B9F1000F01D044F003040BEB450391
:103570000AE0013D08D108224FF0000ACDF80CB056
:10358000D0461746B34604E033F8022D2E2AF0D178
:10359000F1E7039B33F81960002E53D0202E09F178
:1035A000010903D02E2E04D1A94502D044F0030412
:1035B000EFE7BA4501DAA94514D10B2F04D13A46F9
:1035C0005E4644F003043FE0A94502D044F0030402
:1035D00038DC4FEA88085FFA88F8A9460B274FF0D5
:1035E000080AD6E77F2E0CD930460021404B984779
:1035F000064618B1424B1E1816F8806C44F00204BF
:1036000026B1404831463C4B984718B144F003047A
:103610005F2610E0A6F141039BB2192B02D848F0B7
:10362000020808E0A6F161039BB2192B03D8203EE3
:1036300048F00108B6B2DBF8183003F80A600AF166
:10364000010AA6E73A465E46B3691978E52901D131
:10365000E0391970082A04BF4FEA88085FFA88F831
:1036600008F00C030C2B03D008F00302032A01D14D
:1036700044F0020414F0020F0AD108F00308B8F174
:10368000010F08BF44F01004042B08BF44F00804E5
:10369000B3693046DC721C4B9847B369DB7A03F0A0
:1036A0000403DBB228B104281CD1002B08BF05207D
:1036B00018E0BBB97369DA7A12F0100F11D00299D1
:1036C000019A89180291597D1A7D42EA0122D97E18
:1036D0009B7E43EA012343EA0243B360F3E60620FC
:1036E00000E0052005B0BDE8F08F00BF953100086F
:1036F00025450008A6850108652B0008592B000800
:10370000C3850108AF8501084533000838B5018C31
:10371000C5884FF6FF73994208BF29460F4B0446F0
:1037200098470146B8B9216920680D4B9847014672
:1037300070B96369E5221A702368E43A1A71E38864
:10374000AB4208D22046074B984701460028EAD0F2
:10375000042908BF0221084638BD00BF9531000882
:10376000852C0008293200082DE9F041FF26054686
:103770003446042766E02868394B984707460028F6
:1037800064D168690378002B68D0E52BC27A52D0E7
:103790002E2B50D002F03F0212F0080F02D00F2A59
:1037A00049D101E00F2A3DD113F0400F05D0EA883E
:1037B000467B03F0BF042A8401E0A3423BD1437B54
:1037C000B34238D103780D2203F03F03013BEF6988
:1037D00053434FF0010E0D3A224911F802C000EB9D
:1037E0000C0191F8018010F80C1041EA0821BEF19B
:1037F000000F06D0FE2B1EDC27F813108E46013377
:1038000003E04FF6FF7C614515D101320D2AE3D16B
:10381000027812F0400F1ED0FE2B0CDC002227F89D
:10382000132018E01CB9104B9847864210D04FF077
:10383000FF332B840CE0FF24284600210B4B9847D4
:10384000074618B92969002995D10FB100232B61CA
:103850003846BDE8F081013CE4B2EDE70427F5E726
:10386000852C0008B6850108732B00082932000852
:1038700073B51E4615461C4B0B2204469847052E71
:103880000AD9730843EAC6362B4635F8022B5B8803
:10389000B618B6B2002BF4D107230A21B6FBF1F219
:1038A00001FB126196B230310DF80310013B002E7E
:1038B000F3D102A9CA187E2102F8081C00E00136E3
:1038C0009E4202DAA25D202AF9D1072B05DC02A96B
:1038D000CA1812F8082C013300E02022A255013644
:1038E000072EF2DD7CBD00BF492B00082DE9F04F0B
:1038F000856985B0D0F81C800C226D4E044629469F
:1039000001A8B0479DF80F30B14613F0010F1CD04D
:103910000023EB720126E361284601A942463346A3
:10392000644FB8472046644B9847074628B901368C
:10393000B6B2642EF0D1C71DACE0042840F0AA80D6
:103940009DF80F30EB72C4F81C809DF80F3013F017
:10395000020F12D04FF0000A03E00AF1010A1FFA29
:103960008AFA38F81A30002BF7D10AF1190A0D3308
:103970009AFBF3FA1FFA8AFA01E04FF0010A4F4D61
:1039800020460021A847AB460746002840F0828029
:103990000646054620682169DFF83081C0470746A2
:1039A000002877D163691B78E52B00D033B905B9BE
:1039B000E6880135ADB2554501D16FE00546204698
:1039C00001213F4B984707460028E3D062E020469C
:1039D0003146D847074600285CD1A069394B984743
:1039E000013D0646ADB220682169C0470746002860
:1039F00050D163690F21EAB2D4F81CE00D27D972C7
:103A0000511E79435E7318739876D87607464FF641
:103A1000FF7C6045DFF8B8C018BF3EF811001CF805
:103A200007C04FEA102A03F80C009C4418BF01316C
:103A30008CF801A001374FF6FF7C002808BF6046D4
:103A40000D2FE4D1604502D03EF8111009B942F0C3
:103A500040021A70236801221A7120460021184B77
:103A600098470746B0B9013DADB2002DBBD117E074
:103A70006569154B28463946202298470B2228466F
:103A8000A169C847A3690122DB7A03F018032B73ED
:103A900023681A71384605B0BDE8F08F012D96D124
:103AA00020682169C04707460028F3D1E0E700BF3E
:103AB000492B00087138000845330008953100088B
:103AC00029320008732B0008592B0008852C0008A8
:103AD000B6850108F8B5036815461A78303A92B2EF
:103AE000092A07D85C783A2C04D102330360002AF3
:103AF00040F018819C4B1C680C60002C00F0148175
:103B000023786BB16078994B984710F0010F07D17B
:103B1000002D00F00B8110F0040018BF0A20F8BD42
:103B2000002020706070924B984710F0010F40F019
:103B3000FF801DB110F0040F40F0FC8000212046F2
:103B40008C4DA847012816D194F8F231002B00F0D3
:103B5000F58094F8F86194F8F931360446EA036682
:103B600094F8F63120461E4394F8F73146EA0326CE
:103B70003146A84700E00026032800F0DD80002839
:103B800040F0DC8094F83C2094F83B3043EA022378
:103B9000B3F5007F40F0D48094F8472094F8463085
:103BA00053EA02230DD194F8563094F857201B04A1
:103BB00043EA026394F85420134394F8552043EAEF
:103BC000022394F8402094F8427094F84100A361D5
:103BD000E270534394F83F1094F83E2040EA0720E7
:103BE00094F844C094F8437042EA012194F83D509F
:103BF000721857EA0C272262A57020810ED194F822
:103C0000527094F853C03F0447EA0C6794F850C0D0
:103C100047EA0C0794F851C047EA0C27791A0009C3
:103C2000C91A091AB1FBF5F1023140F6F675A9423D
:103C3000E16106D94FF6F675A94200F283800225AC
:103C400000E00125991861621218D318A3624FF0A1
:103C5000FF3323610133032D23715AD1637194F82B
:103C6000612094F86030607843EA0222B218626101
:103C700004F130010123404EB047002849D194F8A7
:103C80002E3294F82F2243EA02223C4B12B29A427F
:103C90003FD194F8322094F83330120442EA0362A0
:103CA00094F830301A4394F8313042EA0322344B0E
:103CB0009A422ED194F8162294F81732120442EA4E
:103CC000036294F814321A4394F8153242EA03223C
:103CD0002C4B9A421DD194F81E3294F81F221B04DB
:103CE00043EA026394F81C22134394F81D2243EA2A
:103CF0000223E36094F81A3294F81B221B0443EA6F
:103D0000026394F81822134394F8192243EA022319
:103D100023611D4A2570138800200133E06213805F
:103D2000E380F8BD0B20F8BD0C20F8BD2846F8BD97
:103D30000320F8BD0A20F8BD0120F8BD0D20F8BD14
:103D40000D20F8BD94F85E1094F85F50090441EA24
:103D5000056194F85C50294394F85D5041EA0521CF
:103D60006162032570E700BF30050020AD23000825
:103D7000ED210008092D0008BD23000855AAFFFF0A
:103D800052526141727241612E03002048B9064AC5
:103D9000136803B1187009B100230B701160002083
:103DA00070470B20704700BF300500202DE9F0411F
:103DB0008EB0044600230EA802F01F0540F8341D03
:103DC000236002A905F01E02504B9847002840F0DE
:103DD00099800BAB08934E4B02A8099301994D4B68
:103DE000984715F01C0F54D060B1042840F08A8029
:103DF00002A8494B9847002840F0848045F0080508
:103E0000079E32E015F0040F77D1079E002E78D080
:103E1000F37A13F0110374D115F0080F25D0327D19
:103E2000777DF17E42EA0727B27E33757375B376EC
:103E3000F37633777377B377F377029842EA012208
:103E4000012352EA07470371D0F82C8007D0394686
:103E5000324B9847002855D1029B013FDF60029802
:103E600041462F4B984700284CD115F0080F1FD022
:103E70000023F3722B4B9847030AB073F373030CC0
:103E8000000E33747074029B01221A7145F02005F4
:103E90000EE0002836D1079E002E30D0F37A13F0C2
:103EA000100F2CD115F0020F02D013F0010F28D102
:103EB000029BDA6AA571E261079A2262327D717D06
:103EC000F07E42EA0121B27E42EA002242EA014249
:103ED0002261B27FF17F120442EA0162317F002049
:103EE0000A43717F236042EA0122E260FF22E2710D
:103EF000DB88A060A061A38004E0082002E0042029
:103F000000E007200EB0BDE8F08100BFD53A000800
:103F10003003002099340008ED38000819310008FA
:103F2000852C00081D4500082DE9F84F9B4600230D
:103F3000ABF8003004468A460068A1885D4B1646FF
:103F400098470546002840F0B280A37913F0800F0F
:103F500040F0AA8013F0010F00F0A880E268A36887
:103F6000D31A9E4240F29C809EB299E0A268D3058B
:103F7000DB0D002B77D12068E179837899420DD34E
:103F80000AB9206902E061694B4B984701280BD9B7
:103F9000B0F1FF3F5CD000236061E3712768616985
:103FA0003846464B984720B9A37963F07F03A37145
:103FB0007AE0E3795FEA562800EB03092CD0BA785F
:103FC00008EB03019142C4BFC3EB02081FFA88F853
:103FD00078785FFA88F351464A46394FB847A37953
:103FE000002836D113F0400F0ED0A369C9EB0309A6
:103FF000C14509D24FEA49290AEB090004F124011D
:104000004FF400722F4B9847E37943444FEA482816
:10401000E3711FFA88F837E0A37913F0400F0BD053
:104020007878012304F12401A269274FB847A379C6
:1040300078B923F04003A371A3694B450ED0214604
:1040400051F8243B4A4658781D4F0123B84728B100
:10405000A37963F07F03A371012528E0E379C4F815
:1040600018900133E371A36804F12401DB05DB0D33
:10407000C3F500781FFA88F8464538BFB046C9181E
:10408000504642460F4B9847A368C8EB0606434488
:10409000A360BBF80030C2444344ABF80030B6B272
:1040A000002E7FF463AF02E0022500E007252846DA
:1040B000BDE8F88F592E0008852E00087D310008D4
:1040C000BD230008492B00085D2400082DE9F84FA6
:1040D0009B460023ABF8003004468A460068A1885E
:1040E000694B164698470546002840F0C980A379D9
:1040F00013F0800F47D113F0020F00F0C080E36887
:10410000DE4228BF0026ADE0A268D305DB0D002B00
:1041100040F087802068E1798378994217D332B9DB
:10412000216959B9594B98470146206103E06169FB
:10413000564B98470146002900F097800129A37942
:104140001ED0B1F1FF3F62D000236161E371A3791A
:1041500013F0400F0DD0214651F8243BA269587846
:104160004B4F0123B847A379002850D123F04003D7
:10417000A371276861693846464B984728B9A379E7
:1041800063F07F03A37102257AE0E3795FEA5628A2
:1041900000EB03092BD0BA7808EB03019142C4BFAE
:1041A000C3EB02081FFA88F8787851464A465FFA4E
:1041B00088F3374FB84748BBA369C9EB0309C1452A
:1041C0000DD24FEA4929344B04F124000AEB0901CE
:1041D0004FF400729847A37923F04003A371E37969
:1041E00043444FEA4828E3711FFA88F82EE0A36998
:1041F0004B4511D0A268E3689A420DD2787804F159
:1042000024014A460123254FB84728B1A37963F01A
:104210007F03A371012533E0E379C4F818900133DB
:10422000E371A36804F12400DB05DB0DC3F500781E
:104230001FFA88F8464538BFB046C0185146164B9D
:1042400042469847A37943F04003A371A368C8EBA3
:1042500006064344A360BBF80030C2444344ABF8B5
:104260000030B6B2002E7FF44FAFA368E2689342ED
:1042700088BFE360A37943F02003A37100E0072522
:104280002846BDE8F88F00BF592E0008713000089D
:104290005D2400087D310008492B0008BD2300087B
:1042A00038B50446A1880068264B9847002847D1B6
:1042B000A37913F0200F43D013F0400F0DD0214607
:1042C00051F8243BA26958781F4D0123A8470028C4
:1042D00035D1A37923F04003A3712068E1691B4B1A
:1042E000984700282CD1256AEB7A43F02003EB7223
:1042F000E3682B77A3891B0A6B77E389AB77E37BB2
:10430000EB772369AB76238A1B0AEB76638A2B75DE
:10431000638A1B0A6B750E4B9847030AA875EB75E9
:10432000030C000E2B766876A379012223F020037C
:10433000A37123681A712068064B984738BD012085
:1043400038BD00BF592E00085D240008852C0008E8
:104350001D450008952D000810B5034B04469847ED
:1043600000B9206010BD00BFA142000810B586B0A2
:10437000044606A840F8141D00222146154B984714
:1043800028BB03ABA361144B2046E3610199134B97
:104390009847B8B9636973B1DA7A12F0100F15D083
:1043A000597D1A7D42EA0122D97E9B7E43EA012390
:1043B00043EA0243A36023682046DB880021A380F0
:1043C000074B9847042808BF052000E0052006B0E9
:1043D00010BD00BFD53A0008300300209934000812
:1043E000953100087FB504460E460068A188134B3E
:1043F00098470546F8B901ABA361114BE36126B9B3
:10440000204629460F4B984714E020460E4B98470C
:10441000042801D1256100E060B9204631460B4BEC
:104420009847002120460A4B9847042802D10023D0
:10443000236100E00546284604B070BD592E0008EF
:10444000300300209531000869370008912B0008DF
:104450002932000810B598B018AB43F85C0D184627
:104460000CA90122244B9847002843D115AB129385
:10447000224B0CA813930199214B9847002839D15E
:10448000119B002B31D0DA7A12F0010F31D1197D56
:104490005C7D12F0100F41EA0424D97E9B7E43EA32
:1044A000012343EA044412D0012C20D903A80CA90B
:1044B000144B24229847059403A80221124B9847D5
:1044C000C0B903A8114B984798B1042812D10CA881
:1044D0000F4B984770B924B10C9821460D4B984763
:1044E00040B90C980C4B984704E0062002E00220EB
:1044F00000E0072018B010BDD53A000830030020B6
:1045000099340008492B00089531000869370008E4
:104510000D37000819310008952D00080048704734
:104520000050473C7F2815D931B1FF2811D80A4BDC
:10453000803833F810007047084B33F8022F82425E
:1045400003D0013189B28029F7D101F18000C0B2D6
:1045500070470020704700BF44860108428601086A
:10456000064A002300E0013332F8021F21B18842DD
:10457000F9D1034A32F81300704700BF22890108BD
:1045800044870108FF230370FF3B8370643343704B
:104590007047FF230370F53B83705A334370643BCD
:1045A000C370704738B50025044645700E4B043083
:1045B00098470E4B04F108009847FF2364222370AC
:1045C00023736273A373E27323746274A374E2743B
:1045D000072395FBF3F3643BC835237563750434F7
:1045E000B5F5C86FF4D138BD93450008854500087E
:1045F00037B50D4B04460D4998470D4B204698475B
:104600000C4B201819780C4D4A1C1A7001230022FB
:1046100000931346A847002323826382A382A375D5
:10462000E3750023A3613EBDF5030008048B010878
:10463000B1040008350500206552000837B5114B5C
:104640000446114998472046104B9847104B2018B4
:104650001978104D4A1C1A7000220123009313464A
:10466000A84700222282A274E27422756275A275A4
:10467000E27522766276A276E27604F11C00064BA1
:1046800098473EBDF5030008108B0108B1040008EF
:104690003805002065520008854500080023037096
:1046A00043708370C370704770B5FF2300250446C4
:1046B00043700570074B8570C57004309847064EEF
:1046C00004F10800B04704F10C00B0472582658270
:1046D00070BD00BF9345000885450008FF2310B555
:1046E0000370FF3B044643708370C3700430034B78
:1046F000984704F10800024B984710BD9345000805
:1047000085450008FF2310B50370FF3B0446437046
:104710008370C3700430034B984704F10800024BC8
:10472000984710BD934500088545000838B5FF231C
:104730000370FF3B044643708370C3700430054B25
:104740009847054D04F10800A84704F10C00A8475C
:1047500038BD00BF934500088545000838B5FF23E4
:104760000370FF3B044643708370C3700430054BF5
:104770009847054D04F10800A84704F10C00A8472C
:1047800038BD00BF934500088545000837B50D4B7F
:1047900004460D49984720460C4B98470C4B20186F
:1047A00019780C4D4A1C1A700123002200931346FD
:1047B000A84700232382A374E37404F11400064B7A
:1047C00098473EBDF5030008178B0108B1040008A7
:1047D0003605002065520008854500080023037057
:1047E00043708370C3708380C3800381438100F171
:1047F00020030022828102309842FAD170470023C0
:1048000043708370C370C21802330021202B918043
:10481000F9D170470023037043708370C3707047F1
:1048200038B50446124DA847201DA84704F10800DA
:10483000A84704F10C00A847002525746574A574E9
:10484000E57425756575A575E57504F11800094BC6
:10485000984725776577A577E5772584658484F87B
:10486000245084F8255084F8265084F8275038BD09
:1048700015480008854500082DE9F74F0024064635
:1048800046F8044B05463A4F3A493046B847DFF8F8
:10489000EC803046C047384E281831784FF0010977
:1048A0004B1CDFF8DCA02246337005F1140B2346C5
:1048B0000430CDF80090D0472E495846B8475846A6
:1048C000C0473178281801EB09032246337005F1FF
:1048D000240B23461430CDF80090D0472549584684
:1048E000B8475846C0473178281801EB09032246DB
:1048F000337005F1340B23462430CDF80090D047B7
:104900001C495846B8475846C0473178281801EB2B
:1049100009032246337005F1440B23463430CDF8A9
:104920000090D04713495846B8475846C047317899
:10493000281801EB09032246337005F5A27B2346B4
:104940004430CDF80090D0470A495846B8475846F9
:10495000C0473178281801EB0903337022462346FB
:1049600000F5A270CDF80090D047BDE8FE8F00BFE3
:10497000F50300081F8B010837050020B10400086B
:10498000655200080023038043808380C380704702
:1049900038B50546002405EBC400034B01349847A5
:1049A000042CF8D138BD00BF8549000800234370AE
:1049B000C3704371C371704770B50025044605602C
:1049C000057145718571C571A81C04EB80002E4BE3
:1049D00001359847102DF7D1103D0C2000FB054004
:1049E0002A4B483001359847102DF6D1103D0C2048
:1049F00000FB0540264B00F5847001359847102DCB
:104A0000F5D1103D142000FB0540224B00F5E47069
:104A100001359847102DF5D1103D342000FB05409D
:104A20001D4B00F5427001359847402DF5D1403DB2
:104A3000280100F5805008302018184B01359847A0
:104A4000102DF5D1103D280100F5885008302018B0
:104A5000134B01359847102DF5D104F5905606F10A
:104A60000800104DA84706F13400A84704F59350FC
:104A70000D4D04F59454A847201DA84704F12800C3
:104A80000A4B984770BD00BF9D460008DD460008F0
:104A900005470008A9460008A54500082D4700085D
:104AA0005D470008DD470008FF470008AD490008E2
:104AB0000023037043708370C370704710B5054BBB
:104AC000044698470022A280E28022726272A2729B
:104AD000E27210BD93450008002208B50260828092
:104AE000C280027242728272C272024B0C309847CC
:104AF00008BD00BF934500082DE9F347044631493E
:104B0000314FB847314E2046B047314D0022297809
:104B10004FF001084B1C2B70DFF8D090134604F1C6
:104B2000180A2018CDF80080C84726495046B847D3
:104B30005046B0472978002201EB080318302B704B
:104B4000201800251346CDF80080C84784F8285067
:104B500084F8295084F82A5084F82B5068012018D2
:104B60002C301C4B01359847402DF7D1403D182083
:104B700000FB054000F502600C30174B01359847EB
:104B8000402DF4D1403D1C2000FB054000F5626043
:104B90000C30124B01359847202DF4D104F58C5080
:104BA0000F4B04F510542C3098470E4D04F15C0067
:104BB000A84704F16C00A84704F17C000A4B984711
:104BC000BDE8FC87288B0108F5030008B104000844
:104BD000340500203D4600088D470008F1450008D7
:104BE000B9490008D94A0008BD4A000865520008C2
:104BF00010B5064B0446984704F12000044B984733
:104C000004F14800034B984710BD00BF91490008CC
:104C100021480008794800080C4A002310B5137099
:104C20000B4A044613700B4A04F5125413700A4AD7
:104C300013700A4A13700A4B984704F10800094B95
:104C4000984704F10C00084B984710BD350500202B
:104C500038050020360500203705002034050020E7
:104C6000F94A0008B14A0008F14B00082DE9F0416B
:104C700093F900406425E602361B96FBF5F6541EB8
:104C8000B04213F8244001DC30B207E064B2E6021F
:104C9000341B94FBF5F4A042A8BF20B200262AE002
:104CA00093F90040E5022D1B642495FBF4F5A8421E
:104CB0001FDB93F9047003F1040C4FEAC728C7EB1C
:104CC000080797FBF4F7B84213DC93F90130401B57
:104CD000DA02D31A9CF9012093FBF4F3D602B21A3C
:104CE00092FBF4F4E41A60437F1B90FBF7F5ED1898
:104CF00005E001360433541EA642D1DB002569438A
:104D0000642391FBF3F000B2BDE8F0810378FF2B40
:104D10001AD0FE2B1AD0FD2B01D1407817E03F2B83
:104D200005D80C4A5B019B189A7952B200E0002228
:104D300090F9023090F901006432C01A5043C82142
:104D400090FBF1F0C01802E0002000E0642040B2C7
:104D5000704700BF1C18002002780346FF2A17D0B6
:104D6000FE2A13D03F2A13D80E49520152189179C6
:104D700090F9020049B288420ADC907993F9012047
:104D800040B28242B4BF0020012002E0012000E0D6
:104D9000002093F90330012B04BFC0F10100C0B221
:104DA000704700BF1C18002008B51648164B9847DE
:104DB0001448164B00F59A51083198471148144B86
:104DC00000F58E51083198470E48124B00F594516A
:104DD000083198470B48104B00F5A452083200F5F3
:104DE000006198470D480E4B00F5CC5108319847AB
:104DF0000A480C4B00F5D4510831984707480A4B34
:104E0000984708BD10180020155300085157000896
:104E1000A15500080957000871580008102000200B
:104E2000F5590008615A0008D95A000810B5002346
:104E30000D4A342101FB0322FE2402F5A452FD2178
:104E400082F8343082F8384082F83C10FD3982F81C
:104E50003E10643182F83D1082F840300133402B1F
:104E600082F84110E4D110BDE4170020F8B59D4947
:104E70009D4C9E48A0479E499E48A0479E499F48FA
:104E8000A0479F499F48A0479F49A048A047A04BE3
:104E900042F2B962DA62012003F594534FF496723C
:104EA00083F865003C21A3F860204FF41675FF22BB
:104EB0004FF49676A3F86250274683F8641083F87F
:104EC000682083F87500A3F870600138A3F8725069
:104ED00083F8741083F878201946844B142202FB5F
:104EE0000032FE2502F59A52013082F83850002433
:104EF0006426013D102882F83E4082F83D6082F829
:104F00003C5082F8424082F8416082F84050E4D13F
:104F100022460C2404FB0234FE2504F58E5484F84A
:104F200038500020D13D013284F83E0084F83D50D5
:104F3000D035102A84F83C50EBD10C2404FB00340B
:104F4000FE2504F5945484F838500022B33D013016
:104F500084F83E2084F83D50B235102884F83C5047
:104F6000EBD1342000FB0230FE2500F5A45080F880
:104F7000385000249A3D013280F83E4080F83D5080
:104F80009935402A80F83C50EBD104F50672033283
:104F9000FE2003EB0212107204F58072013203EB63
:104FA0000212013402F58C52FE386426FD25102CC5
:104FB00082F82E0082F82D6082F82C5082F83200A0
:104FC00082F8316082F83050DFD100F50A72033286
:104FD000FE2403EB0212147200F58872013203EB17
:104FE0000212013002F58C52FE3C6426FD25102889
:104FF00082F82E4082F82D6082F82C5082F83240E0
:1050000082F8316082F83050DFD122462C2505FB32
:105010000235082405F50E5585F834400126083C74
:1050200085F8354085F836604FF496762E8740F245
:10503000DC56AE874FF47A7605F13000EE8742F603
:10504000E06545812046162404FB020404F58E54D5
:105050001C340130002603EB440410282681F2D1D1
:105060000132022AD2D1023A242000FB0230082465
:1050700000F51050C473F7344473FF3C847320462A
:10508000122404FB020404F590540434013000257A
:1050900003EB440410282581F2D10132022AE3D126
:1050A0000024182000FB043001340022FD25402C90
:1050B00080F8422880F8412880F84058F1D150010A
:1050C0001818383001240472941C640100251C193E
:1050D0004572A5726572FD35257254B2042C19DC37
:1050E000262418E0B88B0108F5030008E417002017
:1050F000C98B0108BC3C0020CE8B0108CC3C0020B1
:10510000EA840108FC3C0020D48B0108FC17002035
:105110006429002027240132402AC471CFD12B3AC0
:1051200083F83F20013283F85F20013283F87F202B
:10513000013283F89F20FD20183A83F84A2083F833
:10514000492083F8480083F86A2083F8692083F8AF
:10515000680083F88A2083F8892083F8880083F820
:10516000AA2083F8A92083F8A8002F3881F85500D9
:1051700081F8570081F8590081F85B00CD3881F83B
:10518000542081F85600013081F85800013081F830
:105190005A00911C4901002559188D7151010132A5
:1051A0005918402A81F83E508D87F2D12A4C2B4B5A
:1051B00098470123237284F8533084F85130033325
:1051C00084F85230FB3384F82C5084F8345084F83F
:1051D0002D5084F8355084F82E5084F8365084F8D9
:1051E000383084F8393084F83A3084F8303084F834
:1051F000313084F83230F73B84F83C301A3384F88D
:105200004B30183B84F84930013B84F84A30322651
:105210000D3384F8483004F1880084F85060104958
:10522000B8472623A0207822A4F84C00A4F84E20EA
:1052300084F8406084F842303E3384F8415084F86A
:10524000465084F84530993384F844307D3B84F8E7
:105250003D3084F83E50F8BD643C00202D4E0008DF
:10526000DC8B0108F0B5002985B005DA2D24494210
:10527000047009B22C3C00E0002400250BE04FF044
:105280000A0C91FBFCF70CFB17110135303106F8C5
:105290000C1CEDB239B204AF092907EB0506EEDCB0
:1052A000303106F80C1C691C03E0302605F80C6C44
:1052B0000131C9B204AE994206EB0105F5D991421C
:1052C000F3D3002205F80C2C0A460DE09A4203D1D4
:1052D0002E2101550134E4B204AFB91811F80D1CA8
:1052E000013A01550134E4B2002AEFD1025505B06C
:1052F000F0BD000010B50024E0B2044B9847044B09
:1053000023F814000134202CF6D110BDD96E010809
:1053100008090020F0B5002585B004462F4694F911
:105320001530EEB2042B24D1043B2375A37D013B41
:10533000DBB2632B01D90123A375E17DA37DA27CA0
:1053400051B958B251B24118632901DC9B183DE0B4
:105350006423A374633B0AE050B259B2411A11F1BD
:10536000630F01DBD31A31E09C23A3749C3BE375EC
:1053700063E094F914208AB9022B5ED194F91630B7
:10538000002B5ED1A37C5AB2632A04DC14270133BC
:105390005743A37455E00123A37552E0774A012BCC
:1053A00032F815703FB213D117F5027F01DA9B3343
:1053B0000CE0B7F5027F01DD642307E007F5F8771D
:1053C000033740F2E6339F4237D80023A37434E01A
:1053D000022B14D117F1640F05DAA37C5AB212F133
:1053E000630F2ADB05E0642F27DDA37C5AB2632A12
:1053F00023DC4FF4FA7297FBF2F7FB18E6E7032B76
:105400001FD1642F07DD94F916308BB994F912205F
:105410005AB9643309E017F1640F09DA94F91630C8
:1054200033B994F9122002B99C33A374012303E029
:105430006337C62F01D80023A37594F912301427BF
:105440005F43032E1DD84E4A05F59263013302EBEC
:10545000C303DA8812B2BF1A002F07DD1A8912B20D
:10546000002A0EDDFA02D71B1B8907E009D09A88B3
:1054700012B2002A05DA434A9B8857431BB297FBB6
:10548000F3F7237F3F2B03D9FE2B01D0FD2B24D133
:105490003D4B04F11C00984794F91B30012B15D1AA
:1054A0009B3364218DF804308DF805309C3B8DF8DA
:1054B00008308DF809008DF80C1038B28DF80D10F9
:1054C000324F032201ABB847074606E0C302181A61
:1054D000642390FBF3F000B23F1894F91A30012BCB
:1054E000284B08BF7F429F42B8BF1F4640F2FF7360
:1054F0009F42A8BF1F46264B33F8152012B2974291
:1055000021D0042E09D9234A1670234A1278C2B139
:1055100094F91520042A12D113E033F8150028223B
:1055200000B297FBF2F190FBF2F2914209D0194AD6
:105530001670194A1278012A03D9042E01D1174A8C
:10554000167023F8157094F9143027827BB194F902
:10555000153063B9143397FBF3F31BB2642BA8BF68
:1055600064236FF063029342B8BF1346A3740135FE
:105570002034402D7FF4D3AE05B0F0BD08090020E3
:10558000E417002001F8FFFF0D4D00086D4C0008E6
:105590003A05002016020020B53C00201802002029
:1055A0002DE9F04F0D4685B000242B5D2E193F2BC1
:1055B00079D8301D424B9847012874D106F1080074
:1055C000404B9847824600286DD02E5DDFF8209131
:1055D00073014B44988F3C4F00B2B8473B493C4B5A
:1055E00098474FF07E513B4B8046984728B940463C
:1055F00039493A4B984718B904E04FF07E5801E01A
:10560000DFF8D4802B195B78DFF8EC90013BDBB23C
:10561000012BDFF8E8B0324F05D84046C847CDE946
:105620000001404606E04046C847CDE9000140463B
:105630004146D8474146D8472A4A01464046904706
:10564000C847214BCDE9020150469847C847002280
:10565000DFF8ACC0244BE04702460B46DDE902010F
:10566000B847DFF8A0C002460B46DDE90001E0477D
:1056700011A3D3E90023B8471C4A90471C4ADFF81E
:1056800070C0730176016344961998873836B288E2
:1056900040F2FF7312B29A4204DCB288154B12B288
:1056A0009A4200DAB3800C34C02C7FF47EAF05B090
:1056B000BDE8F08FAFF300800000000000FC9F40C9
:1056C000594D00080D4D0008CD1B000800E0FF44B7
:1056D000DD1D0008ED1F0008000080BFB11F00089D
:1056E000F5130008611A0008000059402919000844
:1056F000E417002001F8FFFF4D130008751C000897
:10570000491600088D100008F8B504460E4600251D
:10571000735D77193F2B12D8381D0B4B9847012822
:105720000DD10A4B07F108009847735D64215B01B6
:10573000E318B3F91020424392FBF1F21A820C35C0
:10574000C02DE5D1F8BD00BF594D00080D4D000832
:105750002DE9F047044688460D46002708EB07066A
:1057600073783F2B76D8281D3E4B984701286CD183
:10577000DFF8F8A005F10800D047814605F10C00DC
:10578000D04718F80720737892B95B01E318B3F992
:1057900010202B8A19B209EB010C624503DD9944F4
:1057A000A5F810904BE0091A8A4248DA1B1A45E026
:1057B0005B01E318B3F91030142B10DD03FB09F380
:1057C00040F2FF7293FBF2F3B2785BB2002A28D06A
:1057D000698A08B21018984224DA521810E013F1BE
:1057E000140F11DA4343204A93FBF2F3B2785BB211
:1057F00042B1698A5B4208B2801A984212DD8A1A65
:105800006A820FE05B420CE0B37853B16A8A11B24E
:10581000C81A002801DDD31A03E0CB424CBF9B1805
:1058200000236B822B8A6A8AD2180F4B2A8212B20B
:105830009A4203DB40F2FF739A4200DD2B827378B9
:105840002A8A5B01E3181A8204E073785B01E3188B
:105850001B8A2B8214371435B7F5A07F7FF47EAFF7
:10586000BDE8F087594D000801F8FFFF0D4D000815
:105870002DE9F74F0B46904682460E4601F5C06271
:105880000021198218339342FAD14446002518F8B2
:1058900005303F2B00F29F80201D534B9847012875
:1058A00040F09980514B04F108009847237B8146D2
:1058B0003F2B21D894F90D20F2B14FF0180B0BFBC0
:1058C000036B18F80530BBF810C05B015344B3F903
:1058D0001000082204F11403CDF804C04946444FD7
:1058E000B84794F90D30DDF804C04343642293FBBC
:1058F000F2F39C44ABF810C0A37B3F2B21D894F962
:105900000F20F2B14FF0180B0BFB036B18F80530AA
:10591000BBF810C05B015344B3F91000082204F136
:105920001403CDF804C04946314FB84794F90F30FD
:10593000DDF804C04343642293FBF2F39C44ABF8CC
:1059400010C0237C3F2B21D894F91120F2B14FF0E5
:10595000180B0BFB036B18F80530BBF810C05B018C
:105960005344B3F91000082204F11403CDF804C025
:1059700049461F4FB84794F91130DDF804C043433E
:10598000642293FBF2F39C44ABF810C0A37C3F2B42
:1059900021D894F91320F2B14FF0180B0BFB036BD5
:1059A00018F80530BBF810C05B015344B3F9100080
:1059B000082204F11403CDF804C049460C4FB8473F
:1059C00094F91330DDF804C04343642293FBF2F3EF
:1059D0009C44ABF810C034353434B5F5506F7FF4C7
:1059E00056AFBDE8FE8F00BF594D00080D4D0008B1
:1059F0006D4C00082DE9F04104460E460025735D0C
:105A000006EB05083F2B21D808F10400124B9847FC
:105A100001281BD1725D182707FB0242138A19B2B5
:105A2000002902DD08F1080002E073B108F10C0062
:105A30000A4B9847735D642207FB0347B7F91030A0
:105A4000434393FBF2F33B8200E013821035B5F53C
:105A5000807FD4D1BDE8F081594D00080D4D00087C
:105A60002DE9F04104460E460025735D77193F2B62
:105A700028D8381D164B9847012823D1DFF85480C9
:105A800007F10800C047735D182202FB0342C302FE
:105A90006421181AB2F9103090FBF1F08342C8BFAC
:105AA000108207F10C00C047735D182202FB03430C
:105AB000C2026421821A92FBF1F2B3F910109142F2
:105AC000B8BF1A821035B5F5807FCED1BDE8F08120
:105AD000594D00080D4D000870B5044600F5C0662C
:105AE000237DB4F910503F2B03D9FE2B01D0FD2BA1
:105AF0000AD10F4B04F114009847C3021B1A642209
:105B000093FBF2F31BB2ED1894F91230012B094B01
:105B100008BF6D429D42B8BF1D4640F6FE139D4230
:105B2000A8BF1D4625821834B442D9D170BD00BF2C
:105B30000D4D000802F6FFFF10B528230A4C0B4953
:105B40000B4A0C48A04720230B490C4A0948A047A0
:105B50000B490C4A4FF411730648A0470A490B4AF7
:105B600004230448A04710BD8D280008E08B0108DD
:105B7000903C0020EA840108E88B0108703C00207A
:105B8000F08B0108B83C0020F88B01086C3C002029
:105B900010B50B490B4C0C4A4FF411730B48A0473E
:105BA00020230B490B4A0948A04728230A490B4ADE
:105BB0000648A0470A490B4A04230448A04710BDE1
:105BC000F08B01082D2A0008B83C0020EA84010867
:105BD000E88B0108703C0020E08B0108903C00201D
:105BE000F88B01086C3C00202DE9F047274CB4B03D
:105BF000A0420746884645D32549264B02A8984728
:105C0000254E02A8B0470022391B02AB0124234DC8
:105C10000094181809B21346A847DFF89890204955
:105C200002A8C84702A8B04702AB00220094181887
:105C30000FFA88F11346A847B246013C2E464D465E
:105C40000EE0174902A8A84702A8D0470123395DF2
:105C50000022009302AB18181346B0470134E4B297
:105C60004445EED30E4902A8A8470E4B00209847A2
:105C70000D4C02A90020A04700200C4B98470020A3
:105C80000B49A047002034B0BDE8F087E41700209E
:105C9000788E0108F5030008B10400086552000879
:105CA00079A1010845700108917001083D71010852
:105CB000E8840108D1010008084B00221A70084B43
:105CC0000849FF2050540021013223F8021C19809A
:105CD000598099800833642AF2D17047DD0500208D
:105CE000AA090020C80C0020F0B50A4DBDF81460C8
:105CF0002C78622C0BD8084F3855084820F83410FF
:105D000000EBC4018B80631C4A80CE802B70204640
:105D1000F0BD00BFDD050020C80C0020A809002050
:105D200038B5084B9847084D0446A847844206D228
:105D3000A847041B04EBD4746010C0B238BD002027
:105D400038BD00BF195E01085F61010838B5084B16
:105D50009847084D0446A847844206D2A847041B2A
:105D600004EBD4746010C0B238BD002038BD00BF51
:105D70003D5E01085F61010838B5054B054698474F
:105D8000044B044628469847201AC0B238BD00BFCD
:105D90005F610108195E010808B592F900300BB186
:105DA000002300E00123137010460121014B9847A6
:105DB000012008BDE95B00082DE9F04FDFF858929B
:105DC0008FB014468846C847894D0646A84701212A
:105DD000A6F10A02A0F10A0300260A20D2B2DBB221
:105DE0000091844F0146019602960396B847C84732
:105DF0008146A847FF21A9F10A02A0F10A030A205F
:105E0000019102910391D2B20146DBB20096B847EC
:105E1000DFF808A22046D047DFF8E491013099F876
:105E200000B0834502D8BBF10F0F01D989F800609B
:105E3000DFF8D4C1FF26CDF814C02046E0476E4FEE
:105E400022463346009601960F21B8476B4ADDF88B
:105E500014C013789346002B7FD1B8F1010F0DD1F8
:105E6000204699F800800693D0478045644E069BF3
:105E70000CD208F1010886F800803AE0B8F1020F70
:105E80000AD199F800305E4E13B1013B337030E017
:105E90002046D04730702CE0A8F103085FFA88F85C
:105EA000B8F1010F25D899F8006046B92046D047CF
:105EB000411C89B22046534B9847012069E106F105
:105EC000FF3814F808202B2A01D12D2302E02D2AB7
:105ED00003D12B2304F808300BE020460693D0476B
:105EE0008642069B03D9202204F80820A3558BF88C
:105EF000006099F800606EB9434A444890470646EE
:105F0000A847FF23A0F11301009301933046C9B2C3
:105F10003E4A10E02046D04786420FD93A4B3C48D3
:105F200098470646A847FF23A0F11701384A009377
:105F300001933046C9B2B847002623E1DFF8C8C054
:105F40003448E0470646A847FF23A0F11701009315
:105F500001933046C9B22F4AEDE72E48E04706903C
:105F6000A847069BA0F11701009618460196C9B2F2
:105F7000284A3346B847B8F1010F0DD19BF80030DD
:105F8000013BE25C2B2A10D02D2A12D0382A01D8EE
:105F9000013215E0302213E0B8F1020F12D19BF864
:105FA0000030013BE25C2B2A01D1023208E02D2AAD
:105FB00001D1023A04E0302A01D9013A00E0392245
:105FC000E254B9E7A8F103085FFA88F8B8F1010FC5
:105FD000B2D89BF800305A1EA15C202901D120398B
:105FE000A15489F8003000238BF80030A4E700BFEB
:105FF00063610108AD5B0108B55E0108120600206F
:106000000C060020E95B0008215D0008808E010875
:10601000858E0108898E01085F610108B1040008BE
:10602000A35D0022A01908908DF82C308DF82D204A
:10603000594B5A489847831CDBB2079399F80030B4
:106040000990013B9E4240F08E80A35DDDF81CC0AC
:10605000202B06FB0CF80CD1A84708F10F084108CB
:10606000FF23009301935FFA88F0C9B24C4AB84706
:1060700036E00EAA08F10F0C02F80C3D5FFA8CFC1A
:106080000692CDF814C0A847DDF814C04FF0FF0801
:106090004108C9B26046069A4346CDF80080CDF863
:1060A0000480B847A8470690A847069BDDF814C0AF
:1060B0005B08991E099BACF102029C4443080B3318
:1060C00000200090CDF80480D0B2CDF808805FFAAF
:1060D0008CF2CDF80C80C9B2DBB2DFF8C8C0E04763
:1060E0009BF80030002B4BD0089803785A1ED2B290
:1060F0002B2B8DF82C2001D1023306E02D2B01D162
:10610000023B02E02F2A02D839238DF82C30079A5F
:1061100006FB02F8A84708F10F084108FF230839D9
:106120005FFA88F8009301930BAA4046C9B2B847BA
:10613000089803785A1CD2B22B2B8DF82C2001D151
:10614000023306E02D2B01D1023B02E0392A02D9AD
:1061500030238DF82C30A847FF23410808310093E5
:106160000193404609E0A847079B410806FB03F25C
:10617000FF230F3200930193D0B2C9B20BAAB847E4
:106180000136F6B22046D04701308642FFF448AFD0
:1061900000200FB0BDE8F08F195E010836930108AA
:1061A0008E8E0108AD5B0108F0B5012387B006466D
:1061B0000D461446B2F9001002A800930922013BD3
:1061C000084FB847294602AAFF233046064DA84784
:1061D000064D064602A8A84702A8A84720603046F8
:1061E00007B0F0BD65520008B95D00080D01000858
:1061F000F0B5012387B006460D461446B2F90010EB
:1062000003A8052200930C4F013BB8472946FF2302
:10621000304603AA094DA847094D064603A8A847DA
:10622000B0F5803F02DB0023238002E003A8A847EB
:106230002080304607B0F0BD65520008B95D000807
:106240000D010008F0B50E46B2F9001087B0002924
:10625000074614464FF00103174D04DA009303A8D4
:106260000622013B07E02B228DF80C2000930DF154
:106270000D00253A0023A8473146FF2303AA0F4DFE
:106280003846A8470E4D064603A8A847B0F5FA4F72
:1062900002DD4FF4FA4306E003A8A84710F5FA4FD1
:1062A00003DA48F20033238002E003A8A8472080E5
:1062B000304607B0F0BD00BF65520008B95D000868
:1062C0000D0100082DE9F04FDFF884928FB01446DD
:1062D0008846C847914D0646A8470121A6F10A0203
:1062E000A0F10A0300260A20D2B2DBB200918C4F43
:1062F0000146019602960396B847C8478146A847CB
:10630000FF21A9F10A02A0F10A030A2001910291DA
:106310000391D2B20146DBB20096B847DFF80CB267
:106320002046D847DFF808A201309AF8009081454E
:1063300002D8B9F10F0F01D98AF80060FF26DFF803
:1063400014922046C847774F22463346009601965E
:106350000F21B847744ACB461378002B77D1B8F198
:10636000010F0FD105932046704A90479AF800809C
:10637000013080456E4E059B0CD208F1010886F86D
:10638000008032E0B8F1020F0CD19AF80030684E6C
:1063900013B1013B337028E02046644B984701302D
:1063A000307022E0A8F103085FFA88F8B8F1010F15
:1063B0001BD89AF8006056B9DFF870C12046E04754
:1063C000411C89B220465B4B984701208EE1059322
:1063D0002046564A90478642059B04D9A21920219F
:1063E00002F8011CA355504B1E709AF8006066B964
:1063F0005148D8470646A847FF23A0F1170100934C
:1064000001933046C9B24C4A11E02046DFF81CC166
:10641000E04786420ED94948D8470646A847FF2399
:10642000A0F11701454A009301933046C9B2B8471D
:10643000002653E14248D8470646A847FF23A0F16B
:106440001701009301933046C9B23D4AEFE73C483B
:10645000C8478146A847A0F1170100960196484613
:10646000C9B2374A3346B847B8F1010F09D12E48AF
:106470000378013BE25C7E2A01D801320DE0202244
:106480000BE0B8F1020F0AD1274A1378013BE25C16
:10649000202A01D9013A00E07F22E254C8E7A8F19E
:1064A00003085FFA88F8B8F1010FC1D81E480378D5
:1064B0005A1EA15C202901D12039A1541A4A8AF818
:1064C000003000231370B3E7A3190793A35D4FF0C7
:1064D000000C8DF82C308DF82DC01A4B1A489847B7
:1064E0009AF8003000F10209013B9E4206905FFAE3
:1064F00089F940F0E380A35D06FB09F8202B2BD13E
:10650000A84708F10F084108FF23009301935FFAA1
:1065100088F0C9B20D4AB84756E000BF6361010870
:10652000AD5B0108B55E0108BB050020B1040008A1
:10653000D6050020E95B0008808E0108858E0108E1
:10654000898E0108195E0108369301088E8E0108B4
:106550005F610108215D00080DF1380B08F10F0C97
:106560000BF80C3D5FFA8CFCCDF814C0A847DDF8A1
:1065700014C04FF0FF0841085A466046C9B243466E
:10658000CDF80080CDF80480B847A8478346A847D7
:10659000DDF814C0069BACF102024FEA5B0B9C4491
:1065A0004308ABF1020100200B330090CDF80480CA
:1065B000D0B2CDF808805FFA8CF2CDF80C80C9B269
:1065C000DBB2DFF838C1E0474A480378002B00F01F
:1065D0008380C9F10003DBB2089306FB09F30F3394
:1065E000DBB2099406934FF000081C4616E0023B0C
:1065F000C8EB03030DF1380B0BF80C3DA84741081D
:10660000FF2304EB09021039D0B200930193C9B201
:106610005A46B84708F101085FFA88F8089A0798BF
:10662000A418B045E4B20378E1D10DF1380B013B79
:106630000BF80C3D099CA84741084FF0FF080839AA
:10664000C9B25A464346CDF80080CDF8048006987A
:10665000B847079A137801338DF82C30A8474108C2
:106660000831CDF80080CDF804805A46434606989C
:10667000C9B2B847A8F1FF08A34619E007980EACC5
:1066800003780233434404F80C3DA84708EB0602A4
:1066900002FB09F24108FF230F321031D0B2009300
:1066A0000193C9B22246B84708F101085FFA88F899
:1066B000C6F10E039845E1DB5C460DE0A84706FBFA
:1066C00009F94108FF2309F10F09009301935FFACB
:1066D00089F0C9B20BAAB8470136F6B22046064A7D
:1066E000904701308642FFF4EFAE00200FB0BDE8C6
:1066F000F08F00BFBB050020B1040008AD5B0108AE
:1067000037B5064B0D461978054C4118FF2302207A
:10671000C9B22A4600930193A0473EBD0001002064
:10672000B55E01082DE9F3410C4B064608460D46BF
:106730009847DFF834800A4F98F800206FF0030381
:106740009B1AC0183B78074CF618F1B2FF232A4673
:10675000C0B200930193A047BDE8FC81795D0008B9
:1067600000010020B55E01088801002070B50123FA
:1067700086B0144600220546009303A8134609B2CA
:10678000044EB047284603A92246034B984706B05B
:1067900070BD00BF655200082567000837B50E4B75
:1067A0000C46054698470D4B013593F848200C4B95
:1067B000083A19786FF012035B1A02EBD27205EBFC
:1067C0006201C01800230093E2B2C9B20133054C44
:1067D000C0B2A0473EBD00BF5F610108643C00201D
:1067E000880100209557010870B5054686B01C4603
:1067F000002922D1012A3E4B05D13E4903A89847E2
:106800002846242162E0022A02D103A83A4923E063
:10681000032A02D103A8394955E0042A02D103A86A
:10682000374906E0052A02D103A8364914E0364963
:1068300003A8984728462B2148E0012926D1012AA0
:106840002B4B05D1314903A89847284625213DE027
:10685000022A03D12E4903A8984741E0032A05D113
:106860002C4903A89847284627212FE0042A02D163
:1068700003A8294906E0052A02D103A82749EBE726
:10688000274903A8984728462A211FE0022908D152
:10689000032A25D1234903A8154B984728462821C8
:1068A00014E0032908D1032A1AD11F4903A8104B69
:1068B00098472846292109E004290AD1032A0FD143
:1068C0001A490B4B03A89847284626212246184B05
:1068D0000AE001230022009303A81346154EB04797
:1068E000154B284603A92246984706B070BD00BF45
:1068F000F5030008948E01089B8E0108A38E010801
:10690000AA8E0108AD8E0108BE9501089294010877
:10691000B58E0108E4970108BA8E0108BE8E010801
:10692000B6950108C58E0108CC8E0108D38E0108EA
:106930009D670008655200082567000870B50123AF
:1069400086B0144600220546009303A8134609B2F8
:10695000064EB04703A80649064B9847284603A9A8
:106960002246054B984706B070BD00BF655200082F
:10697000E68E0108D10100082567000837B5064BEF
:106980000D461978054C4118FF230320C9B22A4649
:1069900000930193A0473EBD00010020ED5E010879
:1069A00037B5064B0D461978054C4118FF230320D7
:1069B000C9B22A4600930193A0473EBD00010020C2
:1069C000B55E01082DE9F0410E46097888B03F29EF
:1069D00005469046174C04D8174B490102A8C91820
:1069E00005E00331C9B202291ED8144902A8144B8C
:1069F0009847144B30469847134E0746134902A850
:106A0000B047134B02A8984701230022009302AB22
:106A100039B218180F4F1346B8470F4902A8B047AC
:106A2000284602A9424600E00C49A04708B0BDE84C
:106A3000F08100BF2567000810180020D88E0108DB
:106A4000F50300080D4D0008D1010008EA8F010888
:106A5000B104000865520008E68E0108DF8E0108C7
:106A60002DE9F0410E46097886B03F2905461746C4
:106A7000DFF86480104C12D8104B4901C9186846E1
:106A80000F4B98473046C0470E4B10B168460E4931
:106A900001E00E49684698472846694607E03046B7
:106AA000C04710B128460A4901E00A4928463A463B
:106AB000A04706B0BDE8F081256700081018002047
:106AC000F5030008D1010008E88E0108EE8E0108E8
:106AD000F58E0108FE8E0108594D0008F0B5DFF86B
:106AE00074C085B00546194EF9B1327800F115072A
:106AF0000024FFB20123C2F12E0200932046294652
:106B00003B46D2B2019402940394E0473278FF23CB
:106B1000C2F12E020094019302930393204629466A
:106B2000D2B23B460A4CA0470EE0327800F1150382
:106B3000C2F12E02012000900191029103910846BA
:106B4000D2B22946DBB2E04705B0F0BD8801002093
:106B5000AD5B0108FD5901082DE9F043054685B0FC
:106B60000C461D4F1D4EDFF87C9011B3B8473278AC
:106B700005F11508D24300245FFA88F80123821832
:106B80002946009320464346D2B2019402940394CE
:106B9000C847B8473278FF23D24382180094019344
:106BA0000293039320462946D2B243460C4CA04799
:106BB0000FE0B84732780121D243821805F115035E
:106BC000009120462946D2B2DBB20194029403948C
:106BD000C84705B0BDE8F0835F6101088801002067
:106BE000AD5B0108FD59010838B50C460546224643
:106BF0000449054B984728463D212246034B9847B8
:106C000038BD00BF808E0108016700089D6700083D
:106C100008B50A46014B0249984708BD01670008BC
:106C2000808E0108012809D11848002303701078CC
:106C3000013988420ADA0130107025E002280AD1B1
:106C4000124B02381870137813B1013B13701BE01C
:106C50000139117018E0032807D11978FF290CBFFA
:106C60001278FF221A7001220CE0632805D91A78E5
:106C7000FF2AF8D164381870F5E7042804D10022FF
:106C80001A700132024B1A7000207047FF05002075
:106C9000460000202DE9F04315463E4A89B012789F
:106CA0000446012A8E463C4F3C4E20D1B7F8008066
:106CB00040F6736C1FFA88F8E04512D8DFF8E0C0A0
:106CC000DCF854804FF47A7CB8FBFCF90CFB198C8F
:106CD000BCF5FA7F05D9009205EB000C5B18FE327B
:106CE0001FE0012100912A197344013924E0B7F80B
:106CF00000C041F218021FFA8CFC944517D9284AAB
:106D0000D2F854C04FF47A72BCFBF2F802FB18C2FE
:106D1000B2F5FA7F0BD90122009205EB000C5B184B
:106D2000013A0192029203925FFA8CF20AE0012189
:106D300000912A197344FE3101910291039120467A
:106D40007146D2B2DBB2B0473988642389B2B1FB55
:106D5000F3F1633B0022009309B205A8114EB0473E
:106D600005A8114B9847114B2D1A197805EBD575CD
:106D7000C1F10A0101EBD17104EB6504FF23491055
:106D800000930193E0B2C9B205AA094CA04709B02B
:106D9000BDE8F0831C020020CE060020FD5901084A
:106DA000643C002065520008195E0108380100208B
:106DB000B55E010810B50146054B06489847064CDC
:106DC00006490448A04706490248A04710BD00BF35
:106DD000F503000888090020D1010008EA8F0108A6
:106DE000FC1700202DE9F04F4B1EDBB2012B14469F
:106DF00085B08246874B884A0BD81878884208D1DC
:106E0000864805786EB2022E01DC01350570062039
:106E100009E0127850B2002803DD7F48013A027081
:106E200002E07E4A00201070012919700CD17B4BC2
:106E300022781B7859B2C1F156018A4201DA013336
:106E40000BE08BB156230FE0022911D1734B22784E
:106E50001B7859B28A4203DDDB43D218227004E06A
:106E60000BB9563300E0002323702046012106E0D1
:106E7000042907D1237820465B4223700339684BED
:106E8000984707E0032905D120460239644B98470B
:106E90000120BBE0DFF89881C047624E0546B0474D
:106EA0004FF0010B6A1F431F00250A21D2B2DBB24B
:106EB0000520DFF88891CDF800B001950295039583
:106EC000C847C0470746B0477A1F431FFF270A211C
:106ED000D2B20520019702970397DBB20095C8470D
:106EE000514B504698478146B04781083B46009732
:106EF000019748464D4FC9B25246B8472378474696
:106F00005B45DFF8308117D9B8478146B047062383
:106F1000B9FBF3F90521B0FBF3F359432378A9F149
:106F20000F090139023BCDF800B001955FFA89F0F5
:106F3000C9B20222DBB2C0472378B3B1B8470546D5
:106F4000B0470623B0FBF3F1B5FBF3F5237801223C
:106F50006D0089000F3D0139013B0092013A019219
:106F6000E8B2C9B20232DBB2C047B8470546B04703
:106F70006D084108A5F116020F3901254FF00009EF
:106F80002378D0B200950322CDF80490C9B2C0474F
:106F90002378552B1BD8264B9847224B834698477E
:106FA0000623B0FBF3F1BBFBF3FB23784FEA8B0B1B
:106FB00089005B19ABF10F0B01390095CDF80490F6
:106FC0005FFA8BF0C9B20222DBB21A4DA8472378D0
:106FD000542B17D8B8470546B0470622B5FBF2F543
:106FE0000523B0FBF2F25D435343591E237801227F
:106FF0000F3D02330092013A0192E8B2C9B2023267
:10700000DBB2C04750460C4B9847002005B0BDE8A6
:10701000F08F00BFBC0500200906002013060020E9
:10702000E95B000863610108215D0008B55E0108A5
:107030005F610108855A0108B56D0008AD5B010864
:1070400030B51D4C85B0A0470123A0F123020021DB
:107050002220D2B20093194D09330191029103917C
:10706000A847A047164B044616489847433C84421D
:10707000154C0FDC154B134898472378114AC3F180
:107080000A0303EBD3735910FF2300930193C9B292
:107090000F4C0EE00F4B0B4898472378094AC3F179
:1070A0000A0303EBD37359100B4CFF230093019396
:1070B000C9B2A04705B030BD5F610108FD590108A4
:1070C000195E010888090020380100204D5D000884
:1070D0006D5E0108215D0008B55E010870B5254EA2
:1070E0004EF66023716D88B0B1FBF3F101240222EA
:1070F0000023214D05A809B20094A8471F4905A8FF
:107100001F4B984705A81F4B9847726D4FF47A7331
:10711000B2FBF3F23C23B2FBF3F103FB112305AA0C
:1071200019B21018002302220094A847002001463B
:10713000222200940190029003900A23124CA0474F
:1071400005A8124B9847124BC0F12200197800EBAA
:10715000D070C1F10A0101EBD171FF234010491039
:1071600000930193C9B205AA0A4CC0B2A04708B067
:1071700070BD00BF643C0020655200087E8E01088F
:10718000D1010008B1040008FD5901083D5E010865
:10719000380100206D5E01082DE9F04F2B4C89B0BD
:1071A00007468B46A0472A4E0546B0474FF0010AD6
:1071B0006A1F431F00250A21D2B2DBB20195029556
:1071C00003950520DFF89480CDF800A0C047A047C4
:1071D0000446B047621F431FFF240A21D2B2DBB22C
:1071E00000950520019402940394C047DFF8708055
:1071F0003846C0478146B04720FA0AF106393A4678
:107200002346009401944846C9B2DFF85890C84715
:107210000FFA8BF12A462B46CDF800A005A80D4D9C
:10722000A84705A8C0470546B04720FA0AF106312D
:107230002346009401942846C9B205AAC847384697
:10724000054B984709B0BDE8F08F00BF5F610108AA
:107250006361010865520008B56D0008AD5B010867
:10726000215D0008B55E01080129F8B506461446FF
:1072700010D11568224B284698471DA3D3E9002357
:10728000204FB84720B128464FF07E511E4B11E0E9
:107290001E4B13E0022917D11568194B2846984751
:1072A00015A3D3E900231A4FB84730B1194B28462C
:1072B0004FF07E519847206001E0174B2360204635
:1072C0000421164B984707E0032905D110460131E8
:1072D000124B98470120F8BD2068114B9847114B7D
:1072E0000146304698470020F8BD00BFAFF300804C
:1072F00085EB51B8FE87C34085EB51B8FE87C3C00C
:107300004D130008D9180008651A0008F63F1CC67E
:1073100015190008611A0008F63F1C46E95B0008D1
:107320000120000899710008F8B54B1EDBB2012B53
:10733000154604462A4B2B4A0BD81878884208D1A8
:107340002948067877B2312F01DC02360670062014
:1073500009E0127850B2002803DD2248013A027099
:1073600002E0214A00201070012919700CD11E4B37
:107370002A781B7859B2C1F1FF018A4201DA013340
:107380000BE08BB1FF230FE0022911D1164B2A78B5
:107390001B7859B28A4203DDDB43D2182A7004E01D
:1073A0000BB9FF3300E000232B702846012106E0D3
:1073B000042907D12B7828465B422B7003390B4BED
:1073C000984707E0032905D128460239074B98471B
:1073D0000120F8BD20462978054B98470020F8BDCC
:1073E000E30500200406002014060020E95B0008E5
:1073F00099710008F8B54B1EDBB2012B1546044607
:107400002D4B2E4A0BD81878884208D12C48067884
:1074100077B2312F01DC02360670062009E01278BF
:1074200050B2002803DD2548013A027002E0244AE8
:1074300000201070012919700FD1214B2A781B7878
:1074400050B259B2C1F17F01884201DA01330FE035
:107450000BB9813313E07F2311E0022913D1184BBC
:107460002A781B7851B258B27E38884203DCDB435D
:10747000D2182A7004E00BB97F3300E081232B700F
:107480002846012106E0042907D12B7828465B42D3
:107490002B7003390B4B984707E0032905D1284689
:1074A0000239084B98470120F8BD204695F9001095
:1074B000054B98470020F8BDCC050020E2050020D0
:1074C00010060020E95B000899710008F0B5184B20
:1074D00085B093F84A300546072B02D9154B9847DB
:1074E00024E0154FB8470123821F00241621D2B291
:1074F000009305204233114E019402940394B04747
:10750000B847821F1621D2B200940520FF344323CE
:10751000019402940394B047094B2846984700947D
:107520000194234623212A46064CA04705B0F0BD0E
:10753000643C0020B56D00085F610108AD5B010887
:10754000215D0008B55E01082DE9F04F002291B0E1
:107550000125DFF87C8107901346584C009508A858
:1075600009B2A04708F5125494F84A30544F072B3B
:10757000DFF86091DFF860A1DFF860B137D9514ED4
:10758000B04794F84A3005900693B8470746B0478D
:10759000069B059ADB43D218013F431E0020D1B25F
:1075A000DBB2FAB20095019002900390C84708A898
:1075B000D0470546B047444B94F84A201B7894F8CE
:1075C0004A10CB1A03EBD373C2EB63014118FF23BC
:1075D0002846C9B208AA00930193D847079B4FEAEF
:1075E000431CE04408F12C00384B984763E0B8474F
:1075F0000026A0F11602162045230146D2B20095BE
:10760000019602960396C847B847FF24A0F11602D8
:1076100016200146D2B245230194029403940096A9
:10762000C847079B4FEA431C08EB0C0909F12C09DA
:107630004846CDF818C0D047192123464A46009441
:107640000194D84708A8D0472F21234608AA0094C0
:107650000194D847DDF818C01B20E04408F1380435
:10766000E2792B4600960146DFF87480C047A37983
:10767000642B06D1B8472A380096C0B21B2142229B
:1076800017E094F80690B9F1000F07D1B8472A38EF
:10769000CDF80090C0B21B2143220AE0A3795BB26F
:1076A00013F1640F07D1B8472A380096C0B21B21E6
:1076B00044222B46C04711B0BDE8F08F6552000848
:1076C0005F6101086361010838010020B56D0008A1
:1076D000E4170020AD5B0108215D0008B55E0108DC
:1076E000955701082DE9F043254F85B08946054699
:1076F000B847244E0446B04700210091AB310191B8
:10770000A4F10A022231FF24A0F10C030A20D2B214
:10771000DBB20291DFF8788001460394C047B84796
:107720000746B0470121009142310191223902916F
:10773000A7F10C021239A0F10C030C200391D2B274
:107740000146DBB2C047104F2846B847DFF84480F7
:1077500014212A46234600940194C0474846B8475E
:107760000746B04741082346009401943846C9B201
:107770004A46C0472846054B984705B0BDE8F08308
:107780005F61010863610108215D0008B56D0008B3
:10779000AD5B0108B55E01082DE9F04F93B00446DA
:1077A0009DF87000A04F10920D930E908A4680466F
:1077B000B8479E4E6FF0090996F84A304FF0160C04
:1077C000C3EB090981445FFA89F9B9FBFCFC0CF1B0
:1077D000FF3C5FFA8CFC964DCDF81CC0954B2046C3
:1077E0009847A8470446B84796F84A30621E0121D8
:1077F0000024C31AD2B22046DBB2009101940931B1
:1078000002940394DFF834B2D847B84796F84A3068
:10781000DDF834C06FF00A02D21AB9FBFCF902EBB2
:10782000000BC9EB0B0B08FB0BFB0CF1FF3E9BFBAA
:10783000FEFBCDF834E009F106017F4BCDF8309026
:107840008B449847A847DFF800925FFA8BFB99F8C2
:107850000010A34508BF4FF0010BC1F10101411811
:1078600089B20991A8470A90B84796F84A200A9B1E
:10787000821A02EBD2725210023A013B92B209997B
:10788000DFF8C8C19BB2009201940A2202940394CB
:10789000049405944120E047A84799F80030C3F1CB
:1078A0000103C3189BB20F93B84796F84A200A9079
:1078B0000B92A8470990B8470A9B0B9A96F84AC0C2
:1078C0009A1A6FF001030999CCEB030302EBD27211
:1078D0005210C31801F1FF3E023A9BB292B2DFF898
:1078E0006CC10F99009301941FFA8EF302940394D4
:1078F000049405944220E047A84799F80010C1F18C
:1079000001014118C9B20991A8470A90B8470A9BDA
:1079100096F84A2003F1FF3E6FF0010309999B1A84
:10792000C31801205FFA8EF2DBB2DFF810C10090BD
:107930000194084602940A210394E047A84799F865
:107940000010C1F101014118C9B20991A8470A907C
:10795000B8470A9B96F84A2003F1FF3E6FF00103F7
:1079600009999B1AC3180094FF345FFA8EF2DFF86E
:10797000CCC0DBB2084601940A2102940394E0478C
:10798000A84799F80090C9F103098144B84796F8CF
:107990004A600746A847DDF830E06FF009039B1BFB
:1079A000CEEB0303DB1908FB03F10D9A0BF1010386
:1079B00091FBF2F10C31C21E5FFA89F901200090AF
:1079C000019402940394DBB24846C9B2D2B21B4C74
:1079D000A0479AF80030DDF81CC0434584BFDDF8AD
:1079E00038B08AF800B0E04508D99AF8003063440E
:1079F0009845C4BFCCEB08088AF800809AF800309C
:107A000007980133109900EB030C0D4B81F800C06F
:107A10001B780C4AC3F1160303EBD3735B100133DD
:107A2000137013B0BDE8F08F63610108643C00205F
:107A30005F610108B56D0008B95C0008AD5B010825
:107A4000380100200001002088010020E95C0008C6
:107A50002DE9F04F8BB09B469DF85030444F099272
:107A6000089388461C460546B847424E6FF0090900
:107A700096F84A30DFF80CA1C3EB090981441623BC
:107A8000284699FBF3F93C4B9847B84796F84A309B
:107A90000025C31A4FF0010C0A2131222846DBB21F
:107AA000CDF800C0CDF814C0019502950395D047DC
:107AB000B84796F84A300A21C31A30222C20DBB28C
:107AC0000095FF35019502950395D047B84796F884
:107AD0004A3006900793B847079B96F84A606FF0C4
:107AE0000D01069AC91A6FF00E039B1B89181B180B
:107AF0006143634391FBFBF193FBFBF30C310F33C9
:107B0000DDF814C02D202F22DBB2C9B2CDF800C0A1
:107B1000019502950395D04798F8003009F1FF3997
:107B2000A34288BF089B5FFA89F988BF88F80030B4
:107B30004C4508D998F800304B449C42C4BFC9EB6F
:107B4000040488F8004098F800300C4A0133994446
:107B5000099B83F800900A4B1B78C3F1160303EBD3
:107B6000D3735B10013313700BB0BDE8F08F00BF0F
:107B700063610108643C0020B56D0008000100202D
:107B800038010020AD5B01082DE9F04F87B09DF86A
:107B900040509DF844A09DF848B0059004911E46C1
:107BA00017460AEB03090BEB05083E4CDAB9012333
:107BB0005FFA89F95FFA88F80093019202920392C2
:107BC0004346304629464A46A047049B012B66D1CE
:107BD000FE330193029303930097304629464A46A9
:107BE0004346A0475BE0002701235FFA89F95FFA6B
:107BF00088F8009301974346029703973046294639
:107C00004A46A047049B012B09D1FE3301930293FE
:107C100003930097304629464A464346A047BAF1A7
:107C20003C0F2FD906EB5A0AFF245FFA8AFAEB1CA5
:107C30001D4F504629465246DBB2009401940294EF
:107C4000B847A8F1030143465046C9B252460094D2
:107C50000194029405EB5B08B8475FFA88F8F21CC0
:107C600030464146D2B24346009401940294B8474C
:107C7000A9F10300009401940294C0B241464A461F
:107C80004346B847BBF1280F09D9FF23B01CA91CF4
:107C900000930193C0B2C9B2059A044CA04707B043
:107CA000BDE8F08FFD590108015D01086D5E010816
:107CB0002DE9F04F814693B09DF878500D9199F9D8
:107CC000001008936943C823680891FBF3F19DF8FD
:107CD0007CA04118C9B205914FEA5A01079199F960
:107CE0000110079C01FB0AF191FBF3F39DF87080F2
:107CF0009DF87460E318DBB2114609900693924830
:107D000001224346914C00960195CDF808A0A0476A
:107D10000998089900EB080301FB05F040F6FE7C8A
:107D200090FBFCF01818FF27C0B20AEB06030246CE
:107D3000CDF810C00097019702973146DBB2DFF80B
:107D400018B2D847824C642108224B460898A047B5
:107D50000AFB00F0079ADDF810C0931990FBFCF1C4
:107D60005918C9B205EB08020097019702974046DF
:107D7000D2B20B46D847FF3F03E0CDF818C0CDF88C
:107D800014B009EB070219F907B092F901C00BFB17
:107D900005FB0CFB0AFCC823099C07989BFBF3FB23
:107DA0009CFBF3FCA34484443C2D5FFA8BFB5FFAFD
:107DB0008CFC19D90CEB06030BEB0802D2B2DBB238
:107DC0000024501E591E00940132FF3401330194E7
:107DD00002940394CDF810C0C0B2C9B2D2B2DBB2E3
:107DE0005C4CA047DDF810C00599069AFF240CEB07
:107DF000060301EB080091190BEB080200940194B3
:107E00000294CDF810C0C0B2C9B2D2B2DBB2524CAB
:107E10000437A047202FDDF810C0AED10D98002107
:107E200009EB800005900691C346B1460D9A069B6A
:107E30009A427FD1059CC82394F9002094F901C08F
:107E40006A430CFB0AFC099892FBF3F2079982182B
:107E5000D2B29CFBF3FC8C4402EB0B035FFA8CFC6C
:107E6000DBB20C920CEB0908DA1E03335FFA88F8D8
:107E7000DBB20A9308F10303FF24D2B2DBB200267F
:107E8000A8F10301089210460B9300960194029406
:107E90000394C9B20A9A2F4FCDF810C0B847642D89
:107EA00048D9059A012392F900102C4F32460093CD
:107EB0000FA83346B8472A492A4B0FA898472A4BA0
:107EC0000FA89847059A012392F901100FAA009371
:107ED000101833463246B8470C9B0998234E83420C
:107EE000DDF810C015D30799214B8C4509D30FA895
:107EF0009847089AA8F10B01101A00940194C0B297
:107F000014E00FA89847089B0094181A0194C0B277
:107F100005E00798844504D20A98009401940B99CF
:107F200005E00A98A8F10B0100940194C9B20FAAC8
:107F30002346B04706994B1CDBB2082B06937FF40F
:107F400075AF13B0BDE8F08F678F0108897B00081B
:107F50006D4C0008FD590108015D010865520008DB
:107F6000088F0108D1010008B1040008B55E0108BE
:107F7000195E01082DE9F0430446994610F8043BC8
:107F800085B03F2B0E4617469DF83080134B144D9D
:107F900013D898470246204610F8143B11495B015C
:107FA0005B18B3F804E0FF2100960197CDF8089024
:107FB000CDF80C800FFA8EF30BE09847009602463E
:107FC0000197CDF80890CDF80C8004F11400FF2142
:107FD0000023A84705B0BDE8F08300BF594D000855
:107FE000B17C00081C180020F7B50C4606461F4659
:107FF0000846114B11469847104D11492046A84795
:108000002046104B9847002201230093394613461F
:1080100020180D4FB8470D492046A84720460C4B65
:1080200098471623153090FBF3F04343D8B2B04283
:1080300038BF3046FEBD00BFF5030008D10100087F
:108040000A8F0108B104000865520008798F010801
:108050003D5E01082DE9F04F8FB003909DF8600060
:1080600004939DF864B000238A46914605901F460C
:108070007E49342202FB031202F5A45230321279F7
:10808000039E8846B24201D10137FFB20133402B33
:10809000EED1002F00F0E5800026029635460A2436
:1080A000BB46342303FB068303F5A45393F8342023
:1080B0000398824240F09C8093F8402038333F2A56
:1080C0001DD81A7A6949182000FB02125B7A02F562
:1080D0000262204606A90C325BB2654CA04705EB54
:1080E00009010446C0EB0A00FF23DFF888C1C0B2D3
:1080F000C9B206AA00930193E0470835EDB23423D4
:1081000003FB068303F5A45393F8422038333F2A38
:108110001DD89A7A5549182000FB0212DB7A02F525
:108120000262204606A90C325BB2514CA04705EB17
:1081300009010446C0EB0A00FF23DFF838C1C0B2D2
:10814000C9B206AA00930193E0470835EDB2342383
:1081500003FB068303F5A6531A793F2A1DD81A7923
:108160004249182000FB02125B7902F502622046A8
:1081700006A90C325BB23E4CA04705EB0901044650
:10818000C0EB0A00FF23DFF8ECC0C0B2C9B206AAF8
:1081900000930193E0470835EDB2342303FB0683D7
:1081A00003F5A6539A793F2A1AD89A792F491820AD
:1081B00000FB0212DB7902F50262204606A90C32AE
:1081C0005BB22B4CA04705EB0901FF230446C0EB33
:1081D0000A00284D00930193C0B2C9B206AAA8476D
:1081E0000299162393FBFBF3CB18DBB202931D46D7
:1081F0000136402E7FF455AF02345F465FFA84FBB0
:10820000002425463422624308EB020303F5A453FD
:1082100030331B79039EB3421BD11448059E80184E
:10822000049AB6FBF7F3CBEB0A01891A023B09F17A
:108230000102AA18DBB200F5A45000933430049B6D
:10824000C9B2D2B20C4EB047162393FBF7F3ED1828
:10825000EDB20134402CD5D10BF1170B5FFA8BF046
:1082600000E038460FB0BDE8F08F00BFE4170020F3
:10827000E97F00086D5E0108757F00082DE9F04F69
:1082800093B007939DF8743005929DF87020089381
:10829000002304460491099299469E48342101FB2B
:1082A000030101F5A45292F840503832A5428046AD
:1082B0000AD0927AA24207D001F5A6521179A142C2
:1082C00002D09279A24203D109F101095FFA89F93A
:1082D0000133402BE1D1B9F1000F00F016810027E6
:1082E000DDF820B03E46BA460A25342303FB078357
:1082F00003F5A45292F834103F2900F2958092F8C9
:1083000040103832A1420BD0927AA24208D003F535
:10831000A6531A79A24203D09B79A34240F08480ED
:10832000342303FB078303F5A45393F84020383329
:10833000A24216D15B7A28460AA9774A5BB2774DEA
:10834000A847049A059B0546F118101AFF23DFF889
:10835000D0C100930193C0B2C9B20AAAE04708365F
:10836000F6B2342303FB078303F5A45393F84220AA
:108370003833A24216D1DB7A28460AA9664A5BB294
:10838000664DA847049A059B0546F118101AFF236D
:10839000DFF88CC100930193C0B2C9B20AAAE047CA
:1083A0000836F6B2342303FB078303F5A6531A7984
:1083B000A24216D15B7928460AA9574A5BB2574DAB
:1083C000A847049A059B0546F118101AFF23DFF809
:1083D00050C100930193C0B2C9B20AAAE04708365F
:1083E000F6B2342303FB078303F5A6539A79A2421E
:1083F00013D1DB7928460AA9474A5BB2474DA84703
:10840000049A059B0546F118101AFF23444E009369
:108410000193C0B2C9B20AAAB047162393FBF9F37D
:108420009A445FFA8AFA56460137402F7FF45DAFCF
:108430000235EDB206950025AA46342303FB0583D9
:1084400003F5A45292F834103F2956D892F8401000
:108450003832A1420AD0927AA24207D003F5A6533D
:108460001A79A24202D09B79A34246D1049A069B74
:108470004FF0340BC3EB020C059A0BFB05FB079B7B
:10848000571C099A5FFA8CFCC3EB0C01B2FBF9F3A1
:1084900008EB0B005744023BFFB2DBB200F5A450DF
:1084A0003A46CDF80CC000933430C9B2079B1D4E3C
:1084B000C344B0470BF5A45393F834100AA84901FC
:1084C00041442C31184B9847184B0AA89847DDF8BF
:1084D0000CC015300CF1FF3CC0B2FF23C0EB0C0008
:1084E000009301930E4EC0B239460AAAB047162334
:1084F00093FBF9F39A445FFA8AFA0135402D9CD137
:10850000069B03F11700C0B200E0484613B0BDE877
:10851000F08F00BFE4170020EA840108E97F00081B
:108520006D5E0108757F0008F50300083D5E0108D7
:108530002DE9F04F8DB007469DF858009B460390FB
:10854000624B894616469DF85CA09847604B614A8D
:108550001978342303FB072303F5A45393F834401D
:1085600090463F2C00F2AE8093F84020411A01EB78
:10857000D171CBEB610438333F2AE4B219D81A7AAF
:10858000182101FB02825B7A02F50262204604A9EF
:108590000C325BB2504CA047FF230446C0EB0900ED
:1085A0004E4D00930193C0B2314604AAA847082556
:1085B00000E00025342303FB078303F5A45393F85D
:1085C000422038333F2A1CD89A7A4249182000FBAF
:1085D0000212DB7A02F50262204604A90C325BB279
:1085E0003D4CA047A9190446C0EB0900FF23DFF862
:1085F000ECC0C0B2C9B204AA00930193E0470835A9
:10860000EDB2342303FB078303F5A6531A793F2AFF
:108610001CD81A792F49182000FB02125B7902F549
:108620000262204604A90C325BB22B4CA047A91968
:108630000446C0EB0900FF23DFF8A0C0C0B2C9B2F6
:1086400004AA00930193E0470835EDB2342303FBFD
:10865000078303F5A6539A793F2A1AD89A791D49B8
:10866000182000FB0212DB7902F50262204604A901
:108670000C325BB2184CA047A9190446C0EB0900A4
:10868000FF23DFF858C0C0B2C9B204AA0093019317
:10869000E047342303FB078703980634E4B2C4EBB6
:1086A0000909831EDBB2CBEB0901721C07F5A4504C
:1086B00000933430C9B2D2B25B46094D1734A84793
:1086C000E0B200E000200DB0BDE8F08F5F6101086E
:1086D00088010020E4170020E97F00086D5E010892
:1086E000757F00082DE9F04F95B09DF878C09DF892
:1086F0007C509DF880900D900C920993CDF800C0AD
:108700000122634CCDF818C00195CDF8089061485E
:10871000A047DDF818C04FEA5903099C6A080B937B
:10872000634402EB04080027DBB20A925FFA88F880
:10873000079308973C46CDF84CC02E4678E0DFF80A
:1087400084B12046D84705463046D847DFF878A19F
:108750004FF07C51D047504B01462846984705467C
:1087600009FB04F04D4B90FBF6F09847CDE90E0164
:1087700029462846D0472946D047494B014605930C
:10878000284698478446474A0B98CDF818C090472A
:10879000DDF818C001466046D047059B01462846D3
:1087A0009847414DA847CDE910010D98D847A847F3
:1087B00000223E4B3E4DA8473E4D02460B46DDE9AA
:1087C0001001A8473C4D02460B46DDE90E01A847C3
:1087D0003A4B9847DDF81CC0089D5FFA80FA07EB1A
:1087E0000C0105EB080004EB0802FF250AEB0C0363
:1087F000009501950295C0B2C9B2D2B2DBB2DFF8E2
:10880000C0C0E047089A079BC2EB0800D91BC4EB25
:108810000802CAEB0303009501950295DBB2C0B2D2
:10882000C9B2D2B2264DA847631C08945746DCB2A1
:10883000DDF828C0644582D30C9A354602FB06F069
:10884000C826DDF84CC090FBF6F08044FF245FFAA8
:1088500088F009EB0C0361460246009401940294EF
:10886000DBB2174FB847DDF830C0079A0CFB09F1AF
:10887000099B91FBF6F15118C9B2EA181846009409
:1088800001940294D2B20B46B84715B0BDE8F08F00
:10889000897B00080C8F0108DD1D000829130008E2
:1088A000611A0008CD1B00084D1300080000594054
:1088B00049160008F51300089110000879190008FE
:1088C000015D0108C51B0008751C00082DE9F04F6B
:1088D0008BB09DF854509DF858809DF85C709DF8C1
:1088E00060B008910992194601222B46CDF800800C
:1088F0000197CDF808B0354C9DF950A0A047089AD3
:108900004FEA5B0C02FB0CF105EB5703DBB20CEBFF
:10891000080606936FF06303F6B291FBF3F171184A
:10892000FF24DFF8AC902846069A3346C9B2CDF84A
:1089300014C0009401940294C847DDF814C0099A49
:108940007B19DBB2079302FB0CF34FF0640C93FB33
:10895000FCF3F31806983146079ADBB2CDF814C041
:10896000009401940294C8470AFB07F0C82390FBC7
:10897000F3F0069B41461818C0B20BEB0803024601
:10898000DBB2009401940294C847BAF1000FCBBF48
:10899000099A089B02FB0AFA03FB0AFADDF814C0E5
:1089A000C8239AFBFCFC4FFA8CFC0BFB0CFC9CFBD9
:1089B000F3FC66443733F1B20093019302932846E7
:1089C000079A0B46C8470BB0BDE8F08F897B0008BB
:1089D000015D01082DE9F04F9946454B8BB00646E5
:1089E00005930846BDF950A09DF854509DF8588055
:1089F0009DF85C709DF860B014469847059B089000
:108A0000204698473B4C09904946304601222B4668
:108A1000CDF800800197CDF808B0A047089A4FEA3A
:108A20005B0C0CFB02F105EB5703DBB20CEB080609
:108A300006936FF06303F6B291FBF3F1FF24711814
:108A4000DFF8B4902846069A3346CDF814C0009457
:108A500001940294C9B2C847DDF814C0099A7B1981
:108A6000DBB207930CFB02F34FF0640C93FBFCF3B7
:108A7000F318CDF814C006983146079A0094019473
:108A80000294DBB2C8470AFB07F040F6FE7390FB86
:108A9000F3F0069B41461818C0B20BEB08030246E0
:108AA000DBB2009401940294C847BAF1000FCBBF27
:108AB000099A089B0AFB02FA0AFB03FADDF814C0C4
:108AC00040F6FE739AFBFCFC0FFA8CFC0BFB0CFCD3
:108AD0009CFBF3FC6644FF23F1B2009301930293E5
:108AE0002846079A0B46C8470BB0BDE8F08F00BF79
:108AF0000D4D0008897B0008015D01082DE9F04F4C
:108B00008DB0BDF958C006469DF86800CDF814C078
:108B10000990534F08469DF85C809DF860A09DF831
:108B2000649014461D46B8470A902046B8470999F4
:108B30000B90CDF80490029130462946012243461D
:108B4000CDF800A0474CA0470A9B4FEA590B0BFBFE
:108B500003F20BEB08076FF06303FFB2099892FB77
:108B6000F3F20A99BA184008D2B2079200FB01F258
:108B700000EB0A06F6B292FBF3F3F318FF24DBB224
:108B8000394D06900893079819463A4633460094A3
:108B900001940294A84708994046079A0B4600940E
:108BA00001940294A8470B9A06980BFB02F34FF02E
:108BB000640B93FBFBF3FB18DBB2079300FB02F3A0
:108BC00093FBFBF3F318DBB2069338463146079A62
:108BD000009401940294A847069909EB0803DBB2BC
:108BE000089307981A4600940B4601940294A847EC
:108BF000DDF814C040F6FE730CFB09F9099999FBE6
:108C0000F3F94F44F8B201EB0A030246DBB25146D6
:108C1000009401940294A847DDF814C00998BCF1AF
:108C2000000FCBBF0B9A0A9B0CFB02FC0CFB03FC56
:108C30009CFBFBFB0FFA8BFB00FB0BFB40F6FE7370
:108C40009BFBF3FB5E44FF23F1B20093019302937D
:108C50004046089A0B46A8470DB0BDE8F08F00BF0C
:108C60000D4D0008897B0008015D01082DE9F04FDA
:108C70008DB0064609929DF858009DF85C200A9335
:108C80000023884608900B921D46FF2E09D1484AC2
:108C90000C2101FB032202F5945230321279424535
:108CA0000FD0B8F1FF0F0ED1DAB296420BD1404A85
:108CB0000C2101FB062202F59452303212793F2A30
:108CC00001D80135EDB20133102BDED1002D6BD070
:108CD0000024A1462F46FF2E09D1354B0C2202FB62
:108CE000043303F5945330331B7943450FD0B8F167
:108CF000FF0F54D1E3B29E4251D12D4B0C2202FB07
:108D0000063303F5945330331B793F2B47D84FF08C
:108D10000C0B0BFB04FBDFF898A00BF594530AEB4C
:108D200003023C32234D069310460792A847079A48
:108D3000014607911046A847069B0546534403F198
:108D400038001D4B9847D3440BF5945230321279BA
:108D50000346520192449AF83E20DDF824E0089838
:108D600052B20092C0EB0E020A98D2B20192421C9B
:108D70004A44D2B20292DDF82CE0089A0F480392DE
:108D8000BEFBF7F2023AD2B2049207992A460C4D82
:108D9000A847162393FBF7F399445FFA89F9013446
:108DA000102C98D1172000E028460DB0BDE8F08FB8
:108DB000E41700200D4D0008594D0008118F0108DF
:108DC000CD8800082DE9F04F89B006469DF84C008B
:108DD00006939DF848A000238846059207901D46FB
:108DE000FF2E09D1424A0C2101FB032202F58E52CB
:108DF0003032127942450FD0B8F1FF0F0ED1DAB2FE
:108E000096420BD13A4A0C2101FB062202F58E5202
:108E1000303212793F2A01D80135EDB20133102BDF
:108E2000DED1002D60D00024A1462F46FF2E09D1AF
:108E30002F4B0C2202FB043303F58E5330331B7986
:108E400043450FD0B8F1FF0F49D1E3B29E4246D15E
:108E5000274B0C2202FB063303F58E5330331B796C
:108E60003F2B3CD84FF00C0B0BFB04FB204D0BF5BC
:108E70008E53E8181F4A04933C309047049B844665
:108E8000EB1803F13800CDF810C01B4B9847AB44EA
:108E90000BF58E5330331B7901465B01ED1895F8C5
:108EA0003E20059DDDF810C0CAEB0503069DDBB230
:108EB000681C4844079DC0B20090A81E90FBF7F0C4
:108EC000C0B20290CDF804A05FFA8CF052B20B4D04
:108ED000A847162393FBF7F399445FFA89F9013405
:108EE000102CA3D1172000E0284609B0BDE8F08F70
:108EF000E41700200D4D0008594D0008E5860008D4
:108F00002DE9F04F8DB0064609929DF858009DF866
:108F10005C200A930023884608900B921D46FF2E82
:108F200009D1494A142101FB032202F59A52303239
:108F3000527942450FD0B8F1FF0F0ED1DAB2964206
:108F40000BD1414A142101FB062202F59A5230321C
:108F500052793F2A01D80135EDB20133102BDED111
:108F6000002D6CD00024A1462F46FF2E09D1364B90
:108F7000142202FB043303F59A5330335B794345E3
:108F80000FD0B8F1FF0F55D1E3B29E4252D12E4B14
:108F9000142202FB063303F59A5330335B793F2BDF
:108FA00048D84FF0140B0BFB04FBDFF89CA00BF52B
:108FB0009A5303F138025244244D0693101D079230
:108FC000A847079A0146079102F10800A847069BA7
:108FD0000546534403F138001D4B9847D3440BF525
:108FE0009A52303252790346520192449AF83E2006
:108FF000DDF824E0089852B20092C0EB0E020A9805
:10900000D2B20192421C4A44D2B20292DDF82CE064
:10901000089A10480392BEFBF7F2023AD2B20492C9
:1090200007992A460C4DA847162393FBF7F399445A
:109030005FFA89F90134102C97D1172000E02846F7
:109040000DB0BDE8F08F00BFE41700200D4D000803
:10905000594D00081A8F0108CD8800082DE9F04FFE
:109060008DB00A939DF85C309DF858A00B930023B7
:109070000646884609921D46FF2E08D103F5067262
:109080004049033201EB0212127942450ED0B8F189
:10909000FF0F0DD1DAB296420AD106F506723949B0
:1090A000033201EB021212793F2A01D80135EDB2E9
:1090B0000133102BE0D1002D60D00024A1462F46B3
:1090C000FF2E08D104F506732E4A033302EB031377
:1090D0001B7943450ED0B8F1FF0F4AD1E3B29E424F
:1090E00047D106F50673274A033302EB03131B79B6
:1090F0003F2B3ED82201234D02F50652383204F5AB
:10910000067B52190BF1030B02F1080105EB0B1B57
:1091100004321D4B089107920BF108009847034653
:109120009BF804004FF0180E0EFB005000F5026093
:1091300070448088099D00B20090CAEB05000A9D2A
:10914000C0B20190681C48440B9DC0B20290B5FBB0
:10915000F7F00238C0B20490CDF80CA00B48089983
:10916000079A0B4DA847162393FBF7F399445FFA30
:1091700089F90134102CA3D1172000E028460DB046
:10918000BDE8F08FE4170020594D0008218F010839
:10919000D58900082DE9F04F8DB00A939DF85C3019
:1091A0009DF858A00B9300230646884609921D4659
:1091B000FF2E08D103F50A724049033201EB021277
:1091C000127942450ED0B8F1FF0F0DD1DAB29642B6
:1091D0000AD106F50A723949033201EB02121279FB
:1091E0003F2A01D80135EDB20133102BE0D1002D1B
:1091F00060D00024A1462F46FF2E08D104F50A7343
:109200002E4A033302EB03131B7943450ED0B8F10A
:10921000FF0F4AD1E3B29E4247D106F50A73274AAF
:10922000033302EB03131B793F2B3ED82201234D5E
:1092300002F50A52383204F50A7B52190BF1030B7E
:1092400002F1080105EB0B1B04321D4B089107923C
:109250000BF10800984703469BF804004FF0180EE6
:109260000EFB005000F5026070448088099D00B23A
:109270000090CAEB05000A9DC0B20190681C4844EA
:109280000B9DC0B20290B5FBF7F00238C0B204905B
:10929000CDF80CA00B480899079A0B4DA847162348
:1092A00093FBF7F399445FFA89F90134102CA3D1A9
:1092B000172000E028460DB0BDE8F08FE41700202D
:1092C000594D0008258F0108FD8A00082DE9F04F4F
:1092D0008FB081469DF86400904600220791069069
:1092E0001346AC48342101FB020101F5A45191F869
:1092F00038404C4503D038310979494501D1013313
:109300009BB20132402AECD1403ADFF888C20C21EE
:1093100001FB02C101F58E5191F83800484503D098
:1093200038310979494501D101339BB20132102A04
:10933000EBD1103A97480C2101FB020101F5945141
:1093400091F83800484503D038310979494501D1B1
:1093500001339BB20132102AECD1103ADFF834C24B
:10936000142101FB02C101F59A5191F838004845DA
:1093700007D091F83C003831484502D0097A494578
:1093800001D101339BB20132102AE7D1103A02F524
:1093900006718048033100EB0111097A49450ED06E
:1093A00002F58071013100EB011101F58C5191F84A
:1093B0002C002831484502D0097A494501D10133B2
:1093C0009BB20132102AE2D1103A02F50A71DFF89D
:1093D000C4C103310CEB0111097A49450ED002F5E5
:1093E000887101310CEB011101F58C5191F82C00C1
:1093F0002831484502D0097A494501D101339BB251
:109400000132102AE1D1002B00F02685042B28BF61
:109410000423049304980A2393FBF0F3023BDBB28A
:109420004FF0000B079DCA4605931C465E46C14699
:10943000584A342707FB0B2707F5A45797F838300D
:109440003037534533D15449544B08A8984739799C
:10945000504B490159182C31514B08A89847514F8E
:1094600008A8B847A5F10A03181A04EB0901FF235D
:1094700000930193C9B208AADFF83C81C0B2C0478B
:10948000DDF810C0142393FBFCF308A8E418B847D8
:10949000B042E4B203D908A8424B98470646142CC0
:1094A00005D90F3DAD1B059C05F0FF0500263420B6
:1094B00000FB0BF0374A02EB000C0CF5A45C9CF8A7
:1094C0003C30534548D10DF13808002708F8187D85
:1094D0000CF13C00CDF80CC0334B984701233A46C1
:1094E0000146009340463B46304FB8472C4F304929
:1094F0004046B847DDF80CC040469CF83410DFF811
:1095000094C0490161442C31B847264F4046B847C2
:10951000A5F10A03181A04EB0901FF230093019334
:10952000C9B24246DFF890C0C0B2E04704981423A5
:1095300093FBF0F308A8E418B847B042E4B203D9AB
:1095400008A8184B98470646142C05D90F3DAD1BAB
:10955000059C05F0FF0500260BF1010BBBF1400F48
:109560007FF466AFABF1400B0A4A0C2707FB0B27D1
:1095700007F58E5797F838303037534549D10D49A4
:10958000064B08A898473979024B490159182C31E4
:1095900014E000BFE41700202E8F0108F503000837
:1095A000D10100083D5E01080D4D0008655200081C
:1095B0002D8F0108358F01086D5E0108AA4B08A8A0
:1095C0009847AA4F08A8B847A5F10A03181A04EB50
:1095D0000901FF2300930193C9B208AADFF8B08202
:1095E000C0B2C047DDF810C0142393FBFCF308A8F9
:1095F000E418B847B042E4B203D908A89B4B984797
:109600000646142C05D90F3DAD1B059C05F0FF0542
:1096100000260C2000FB0BF0954A02EB000C0CF529
:109620008E5C9CF83C30534548D10DF1380800273A
:1096300008F8187D0CF13C00CDF80CC08D4B984714
:1096400001233A460146009340463B468A4FB847BD
:10965000854F8A494046B847DDF80CC040469CF823
:109660003410DFF80CC2490161442C31B8477F4FF8
:109670004046B847A5F10A03181A04EB0901FF2375
:1096800000930193C9B24246DFF804C2C0B2E0477A
:109690000498142393FBF0F308A8E418B847B042E9
:1096A000E4B203D908A8714B98470646142C05D993
:1096B0000F3DAD1B059C05F0FF0500260BF1010BCE
:1096C000BBF1100F7FF450AFABF1100B684A0C27C1
:1096D00007FB0B2707F5945797F838303037534579
:1096E00033D16749674B08A898473979604B4901DE
:1096F00059182C315C4B08A898475C4F08A8B8470C
:10970000A5F10A03181A04EB0901FF230093019342
:10971000C9B208AADFF87881C0B2C047DDF810C02E
:10972000142393FBFCF308A8E418B847B042E4B252
:1097300003D908A84D4B98470646142C05D90F3D70
:10974000AD1B059C05F0FF0500260C2000FB0BF06F
:10975000474A02EB000C0CF5945C9CF83C305345F6
:1097600048D10DF13808002708F8187D0CF13C00AD
:10977000CDF80CC03F4B984701233A460146009371
:1097800040463B463C4FB847374F3F494046B847B5
:10979000DDF80CC040469CF83410DFF8D4C0490115
:1097A00061442C31B847314F4046B847A5F10A0310
:1097B000181A04EB0901FF2300930193C9B2424632
:1097C000DFF8CCC0C0B2E0470498142393FBF0F359
:1097D00008A8E418B847B042E4B203D908A8234B5C
:1097E00098470646142C05D90F3DAD1B059C05F086
:1097F000FF0500260BF1010BBBF1100F7FF466AFE4
:10980000ABF1100B1A4B142707FB0B3707F59A57D0
:1098100097F838203037524549D11C49194B08A8D0
:1098200098477979124A490151182C310E4B08A8F2
:1098300098470E4F08A8B847A5F10A03181A04EB79
:109840000901FF2300930193C9B208AADFF8408001
:10985000C0B2C047DDF810C0142393FBFCF308A886
:10986000E418B847B04215E0D10100083D5E010898
:10987000E41700200D4D000865520008348F0108E0
:109880003C8F0108F50300083B8F0108428F010857
:109890006D5E0108E4B203D908A8A74B98470646B5
:1098A000142C04D90F3DAD1B059C05F0FF051420B9
:1098B00000FB0BF0A14A02EB000C0CF59A5C9CF843
:1098C0003C30534548D10DF13808002708F8187D81
:1098D0000CF13C00CDF80CC0994B984701233A4657
:1098E0000146009340463B46964FB847964F9749EE
:1098F0004046B847DDF80CC040469CF83510DFF80C
:109900003CC2490161442C31B8478B4F4046B847AF
:10991000A5F10A03181A04EB0901FF230093019330
:10992000C9B24246DFF834C2C0B2E04704981423FB
:1099300093FBF0F308A8E418B847B042E4B203D9A7
:1099400008A87D4B98470646142C05D90F3DAD1B42
:10995000059C05F0FF050026142000FB0BF0774A5C
:1099600002EB000C0CF59A5C9CF84030534549D151
:109970000DF138080027101808F8187D704BCDF845
:109980000CC000F59C50984701233A4601460093CD
:1099900040463B466B4FB8476B4F6C494046B84713
:1099A000DDF80CC040469CF83510DFF890C1490145
:1099B00061442C31B847604F4046B847A5F10A03CF
:1099C000181A04EB0901FF2300930193C9B2424620
:1099D000DFF888C1C0B2E0470498142393FBF0F38A
:1099E00008A8E418B847B042E4B203D908A8524B1B
:1099F00098470646142C05D90F3DAD1B059C05F074
:109A0000FF0500260BF1010BBBF1100F7FF4FAAE3E
:109A1000ABF1100B0BF50677484A033702EB07173B
:109A20003B7A534532D14A494A4B08A8984739797D
:109A3000424B490159182C31434B08A898473E4FD7
:109A400008A8B847A5F10A03181A04EB0901FF2377
:109A500000930193C9B208AADFF80081C0B2C047E1
:109A6000DDF810C0142393FBFCF308A8E418B847F2
:109A7000B042E4B203D908A82F4B98470646142CED
:109A800004D90F3DAD1B059C05F0FF050BF580705B
:109A90000130DFF8A8C000010CEB000303F58C5384
:109AA00028331B79534563D160440DF138080027F2
:109AB00000F58C5008F8187D2C30CDF80CC0204BE8
:109AC000984701233A460146009340463B461D4FC6
:109AD000B8471D4F20494046B847DDF80CC00BF58C
:109AE000067303330CEB03131B7940465B019C4464
:109AF0000CF12C01B847104F4046B847A5F10A03B6
:109B0000181A04EB0901FF2300930193C9B24246DE
:109B1000DFF848C0C0B2E0470498142393FBF0F389
:109B200008A8E418B847B042E4B219D908A8024B13
:109B30009847064614E000BF3D5E0108E417002088
:109B40000D4D000865520008D1010008418F010841
:109B5000488F0108F5030008478F01086D5E010872
:109B6000142C05D90F3DAD1B059C05F0FF05002603
:109B70000BF580700130DFF8CCC200010CEB000364
:109B800003F58C5328331B7A53454DD160440DF1B6
:109B90003808002700F58C5008F8187D3030CDF8D3
:109BA0000CC0A34B984701233A4601460093404618
:109BB0003B46A04FB847A04FA0494046B847DDF804
:109BC0000CC00BF5067303330CEB03131B794046F3
:109BD0005B019C440CF12C01B847994F4046B847B3
:109BE000A5F10A03181A04EB0901FF23009301935E
:109BF000C9B24246DFF85CC2C0B2E0470498142301
:109C000093FBF0F308A8E418B847B042E4B203D9D4
:109C100008A88B4B98470646142C05D90F3DAD1B61
:109C2000059C05F0FF0500260BF1010BBBF1100FA1
:109C30007FF4F0AEC846ABF1100B0BF50A77814A02
:109C4000033702EB07173B7A534532D17E497F4BEE
:109C500008A8984739797B4B490159182C31764B24
:109C600008A89847764F08A8B847A5F10A03181A1C
:109C700004EB0901FF2300930193C9B208AADFF89E
:109C8000D481C0B2C047DDF810C0142393FBFCF3AD
:109C900008A8E418B847B042E4B203D908A8684B52
:109CA00098470646142C04D90F3DAD1B059C05F0C2
:109CB000FF050BF588700130DFF888C100010CEB5F
:109CC000000303F58C5328331B7953454DD1604471
:109CD0000DF13808002700F58C5008F8187D2C305D
:109CE000CDF80CC0524B984701233A4601460093E9
:109CF00040463B464F4FB8474F4F55494046B847FF
:109D0000DDF80CC00BF50A7303330CEB03131B795E
:109D100040465B019C440CF12C01B847484F40463B
:109D2000B847A5F10A03181A04EB0901FF230093B1
:109D30000193C9B24246DFF81CC1C0B2E0470498A3
:109D4000142393FBF0F308A8E418B847B042E4B238
:109D500003D908A83A4B98470646142C05D90F3D5D
:109D6000AD1B059C05F0FF0500260BF58870013042
:109D7000DFF8D0C000010CEB000303F58C5328334F
:109D80001B7A53454DD160440DF13808002700F58A
:109D90008C5008F8187D3030CDF80CC0244B984713
:109DA00001233A460146009340463B46214FB847BF
:109DB000214F27494046B847DDF80CC00BF50A7320
:109DC00003330CEB03131B7940465B019C440CF1FD
:109DD0002C01B8471A4F4046B847A5F10A03181A94
:109DE00004EB0901FF2300930193C9B24246DFF857
:109DF00064C0C0B2E0470498142393FBF0F308A8B2
:109E0000E418B847B042E4B203D908A80C4B98470D
:109E10000646142C05D90F3DAD1B059C05F0FF052A
:109E200000260BF1010BBBF1100F7FF406AF14E01D
:109E30000D4D000865520008D1010008478F010848
:109E40003D5E0108E41700204E8F0108F50300086D
:109E5000538F01086D5E0108079D079A551BE8B2F4
:109E60000FB0BDE8F08F00BF012908B5104605D13D
:109E700013785AB2632A0ADC013307E002290BD1B6
:109E800013785AB212F1630F01DB013B0370012119
:109E9000074B9847002008BD0339C9B2012904D8EF
:109EA0000121034B9847012008BD002008BD00BFD9
:109EB000E95B00082DE9F043464B05461E7889B062
:109EC000FF2E084690461C4663D1434E032132467E
:109ED000424CA0473378424C009328462146414DDE
:109EE0000DF11F020323A847B14624780A254BE051
:109EF000022C45D899F8001028460B1B594241EB1B
:109F00000301394B9847012C334E0AD0022C1DD047
:109F100031782846D1F1010138BF0021334B9847F1
:109F20002EE03349334B03A89847334B03A8984797
:109F3000002203AB98F900101818009413462F4F15
:109F4000B8473278284603A9012A14E02C49294B46
:109F500003A89847284B03A89847012300220093A1
:109F600003AB98F901101818244F1346B8473278FC
:109F7000284603A9022A14BF00220122214B984738
:109F800016350134EDB2E4B29DF81F30A342AFD8CC
:109F90001CE0012E09D002D3022E17D108E01A4A84
:109FA00001201070FF221A7011E0184B586802E06F
:109FB000164B01329868FF23154DA847012805D19B
:109FC000114B1870FF232370013800E0002009B006
:109FD000BDE8F083E900002017060020256C00088A
:109FE00003060020517A0008DD6A0008116C0008A1
:109FF00084950108F5030008B104000865520008C3
:10A000005A8F0108A16900084600002004010020C1
:10A01000699E00082DE9F04F814B8DB093F80080C8
:10A020008246B8F1FF0F0E4614461D4665D17D4F9E
:10A0300008463A4611217C4EB047DFF818823B783B
:10A0400041460093794E81460DF12F02504611236F
:10A05000B04798F800604FF00A0831E03978404680
:10A060008B1B594241EB0301714B98473A783EB93B
:10A07000D2F10101404638BF00216E4B984719E0EC
:10A08000082E09D8C6EB020CDCF10002404631462E
:10A0900042EB0C02684B0CE0684BC6EB020EA6F1DB
:10A0A000090153F82110DEF10002654B404642EBF6
:10A0B0000E02984708F1160801365FFA88F8F6B2E2
:10A0C0009DF82F30B342C9D85E4B3E7898475E4B1F
:10A0D00007469847013E3223333F0B38F6B20093D0
:10A0E000FFB2283BC0B2019303903146029720464D
:10A0F00001220A3B554EB04760E1B8F1000F05D18F
:10A10000534A01201070FF221A707AE1B8F1090F4A
:10A110000ED100231A46072192FBF1F16439C832AF
:10A12000E018E1540433B2F5C86F4170F3D148E14F
:10A13000B8F10A0F0ED100236422E118E25404336F
:10A14000202B4A70F8D17C33237063709C3B2371C1
:10A15000637136E1B8F10B0F1BD100226423A11803
:10A16000A3540432202A4B70F8D17C3222706270E2
:10A17000627133322272CF3ACE2162723120627321
:10A180003232227421712073637423756375313AFE
:10A1900018E1B8F10C0F0BD10023E21892F901106D
:10A1A000043301EBD1714910202B5170F5D108E136
:10A1B000B8F10D0F08D10023E21851780433494259
:10A1C000202B5170F8D1FCE0B8F10E0F12D1002312
:10A1D000E21851780139517049B211F1640F01DA76
:10A1E0009C2102E0642901DD642151700433202B9D
:10A1F000EED1E6E0B8F10F0F2ED10023E21851782E
:10A200000131517049B211F1640F01DA9C2102E071
:10A21000642901DD642151700433202BEED1D0E09C
:10A22000BD000020E7050020256C0008517A0008D9
:10A23000DD6A0008116C00087D69000898000020A4
:10A24000A16900085F61010863610108B17C000831
:10A2500046000020FC050020B8F1100F6A4FDFF81F
:10A26000C091DFF8C0B16ED1DFF8A881FF23674E3F
:10A2700067484246B04798F80030099046460BB907
:10A28000013333703378402B02D9624B40221A706D
:10A2900095F800C096F800A00CF1FF3C5FFA8CFC2A
:10A2A000DFF884813423CDF814C00AF1FF3A03FBB0
:10A2B0000A8AB8470690C8470790B8470890B84739
:10A2C0000746C847069A079BD208D2B200920522D9
:10A2D000B3FBF2F303EB4303DBB20899019383086A
:10A2E0000139013BDDF814C00AF5A65AA1EB970726
:10A2F000DBB20AF1080A0393043A0023FFB2504686
:10A3000061460297D847099B012B5FD10022134673
:10A3100030780D21013801FB003000F5A66008EB14
:10A320008000007AA0543078013801FB003101F53B
:10A33000A66108EB8101487A0133A1180432082B89
:10A340004870E5D13DE0B8470746C84732230B388F
:10A350000093333F283BC0B208F1FF310122019343
:10A36000FFB20A3B0390C9B220460297D8472B7828
:10A370005046013B04EB83023146DBB2264FB8471F
:10A38000012E81460DD1234604F11C011A7893F960
:10A39000046050B28642B8BF1A7104338B42F5D1C3
:10A3A0000CE0022E0AD10023E2181279E05651B2D5
:10A3B0008842C8BFE25404331C2BF5D1B9F1010F18
:10A3C00004D10122154B1A70FF232B700023E25693
:10A3D00012F1640F01DA9C2202E0642A01DD64229A
:10A3E000E254E21892F9011011F1640F01DA9C2194
:10A3F00002E0642901DD642151700433202BE6D191
:10A4000000200DB0BDE8F08F5F61010829730008DE
:10A410005D8F0108CD050020B59E00084600002094
:10A4200063610108B17C0008E41700202DE9FF47B3
:10A430004B4E824635781446FF2D69D1DFF83481C2
:10A440000846424643213346464FB847DFF84C9111
:10A4500098F800300DF10F020093434F432350460C
:10A460004946B847414B47461A78FF2A04D01B7823
:10A470000127237035706FE099F800400A2541E00C
:10A48000397828460B1B594241EB0301384B394EB2
:10A4900098473CB932782846D2F10102364938BF94
:10A4A00000220FE0012C04D1327828463349012ADA
:10A4B00005E0022C08D1327831492846022A14BF1F
:10A4C000002201222F4B18E0422C17D83278284660
:10A4D000C4EB020CDCF1000242EB0C022A49294BCE
:10A4E00098473278294B6101C4EB020EC918DEF19E
:10A4F0000002274B284642EB0E02984716350134DE
:10A50000EDB2E4B29DF80F30A342B9D8002723E0A2
:10A51000204A214B2DB9FF2101272170177031707E
:10A5200017E0012D09D1FE2121701570FF22327034
:10A530002046294698472F460EE0022D4FF001078E
:10A5400002D1FD21217001E0033D25701770FF222B
:10A550003270204639469847384604B0BDE8F08747
:10A56000FF010020256C00089977000816020020E2
:10A57000596B0008D80500206D8F01087C8F0108F9
:10A580008C8F010801670008988F0108B017002020
:10A590002567000846000020E95B0008020600204D
:10A5A000F0B5334B064610461A7885B0FF2A4CD1D9
:10A5B000304C0846224641212F4DA84723782F4D85
:10A5C0000093304629462E4E0DF10F024123B0472D
:10A5D0002D780A2633E0217830464B1B594241EB57
:10A5E0000301284B234F984745B93A783046D2F1BA
:10A5F0000102254938BF0022244B1BE0402D1AD808
:10A600003A783046C5EB020CDCF1000242EB0C025A
:10A610001F491E4B98471F4B6A1E182101FB023130
:10A620003A780431C5EB020EDEF100021A4B3046D7
:10A6300042EB0E02984716360135F6B2EDB29DF8A0
:10A640000F30AB42C7D800200FE014490124144D4D
:10A650001AB9FF3202700C7003E0013A02700C70FC
:10A66000FF221A702146A847204605B0F0BD00BF62
:10A67000BF000020FE050020256C00080006002019
:10A6800099770008596B00089E8F01080167000840
:10A69000A38F01080C200020256700084600002039
:10A6A000E95B00082DE9F04F137889B0FD2B0746D0
:10A6B00014460BD003F1020A5FFA8AFABAF1010FCD
:10A6C00094BF4FF0020A4FF0040A01E04FF0030A72
:10A6D0008B4D95F80180B8F1FF0F40F0DC80084603
:10A6E0002A4651466B1C874EB0472B7886490DF1A0
:10A6F0001F0238460093854E5346854FB047B847F2
:10A70000DFF86CB20646D8478146B8470122A6F169
:10A710001601009200264A46DFF858920346019639
:10A72000029603963046C9B2DFF8E8C1E04799F8CF
:10A730004A30002B3AD0B84799F84A300490059334
:10A74000D8478346B847059B049ADB43D2180BF1E0
:10A75000FF3B431E0121304600910196D1B2029683
:10A760005FFA8BF20396DBB26A4EB0476A4E2B78E3
:10A7700056F82300694B98478346B847684B99F8C9
:10A780004A201B7899F84A10CDF80080CB1A03EBC9
:10A79000D373C2EB63012B784118CDF8048056F8CF
:10A7A00023205846C9B243465E4EB047564B0A2650
:10A7B0001F786BE029783046CB1B594241EB0301EF
:10A7C000594B984757455DD223785849FD2B584B34
:10A7D0000DD1022F0BD14A4A304612780969A2F1F5
:10A7E000020CDCF1000242EB0C02984734E02A78BC
:10A7F0003046C7EB020EDEF1000242EB0E0251F8CA
:10A8000027109847022F27D03D4B032F1A7829D0C5
:10A81000012F484B2FD194F800E0BEF1FF0F02D179
:10A82000304645490AE0BEF1FE0F02D130464349A9
:10A8300004E0BEF1FD0F03D141493046012A1DE07D
:10A84000BEF13F0F05D83F494FEA4E1E30467144D6
:10A85000F4E730463C49F1E72A78304694F9011094
:10A86000022A03E094F902103046032A14BF0022A2
:10A870000122364B05E036493046BA4214BF002269
:10A880000122984716360137F6B2FFB29DF81F3005
:10A89000BB428FD87DE0B8F1030F7AD8DFE808F02B
:10A8A000020D246C2B4B01261E70FF236B7020467B
:10A8B0000421294B984730466CE01C4B274E5868C2
:10A8C0002246FF23B047264F06463B78FF2B5AD03F
:10A8D000244B98473878244B9847002801DD64239F
:10A8E00000E09C2363704EE0FD2B104B04F101024D
:10A8F0000CBF186998681D4EFF23B04742E000BFA7
:10A900008B010020256C00080606002099770008BE
:10A9100063610108FD59010824010020215D000840
:10A9200038010020B55E0108596B000804000020C2
:10A9300001670008256700086D8F01087C8F0108FA
:10A940008C8F010810180020AA8F01083D690008AB
:10A950004193010846000020E95B00082DA400088F
:10A9600016020020FD6C0108D96E0108F57300087D
:10A970005F610108643C0020084BA21CD868084CA9
:10A98000FF23A0470646012E03D1064B1E70FF236E
:10A990006B70002009B0BDE8F08F00BF04000020FC
:10A9A000F5730008460000202DE9F04F137891B0B0
:10A9B000FD2B0746154601D10233137095F800A010
:10A9C000974C0AF1020A94F805805FFA8AFABAF104
:10A9D000010F94BF4FF0020A4FF0050AB8F1FF0FC4
:10A9E00040F0F0800846221D5146631D8D4EB04751
:10A9F00023798D490DF13F02384600938B4E534623
:10AA00008B4FB047B847DFF89CB20646D84781461F
:10AA1000B8470122A6F11601009200264A46DFF847
:10AA2000889203460196029603963046C9B2DFF833
:10AA300004C2E04799F84A30002B3AD0B84799F859
:10AA40004A3004900593D8478346B847059B049A3B
:10AA5000DB43D2180BF1FF3B431E0121304600912E
:10AA60000196D1B202965FFA8BF20396DBB2714E79
:10AA7000B047714E237956F82300704B98478346B0
:10AA8000B8476F4B99F84A201B7899F84A10CDF8CF
:10AA90000080CB1A03EBD373C2EB63012379411817
:10AAA000CDF8048056F823205846C9B24346654E77
:10AAB000B0475D4B0A261F787EE021793046C7EB10
:10AAC000010CDCF1000141EB0C015F4B984757454D
:10AAD0006ED2534B30461A795C4BC7EB020EDEF157
:10AAE000000253F8271042EB0E02594B98477B1E89
:10AAF000032B52D8DFE803F002353B452978DFF815
:10AB00008481FF2903D122793046524922E0FE296F
:10AB100003D12279304650491CE0A1F14003DBB259
:10AB2000BD2B14D94D4B4901C91807A84C4B984768
:10AB30004C4B284698474C4B10B107A84B4901E0B5
:10AB40004B4907A898472279304607A902E02279A5
:10AB500048493046A2F101035A4242EB0302C04782
:10AB600026E02279304695F90110022A04E0227984
:10AB700095F902103046032A14BF002201223E4BF1
:10AB800015E022793046A2F1040CDCF1000295F9BF
:10AB9000031042EB0C02394B09E022793849C7EB2C
:10ABA000020EDEF10002374B304642EB0E029847B0
:10ABB00016360137F6B2FFB29DF83F30BB423FF682
:10ABC0007CAF80E0B8F1040F7DD8DFE808F0030E19
:10ABD00020236F002C4B01261E70FF236371284633
:10ABE00004212A4B984730466EE0184B284E58688F
:10ABF0002A46FF23B047274B06461B78FF2B5CD025
:10AC0000254B984764236B70503BAB7055E023484D
:10AC10006A1C02E00D4BAA1CD868FF23204D4AE0B5
:10AC20008B010020256C0008CE05002099770008D4
:10AC300063610108FD59010884000020215D0008BE
:10AC400038010020B55E0108596B0008EC000020B7
:10AC500001670008FE8E0108F58E0108101800201B
:10AC6000F5030008594D0008D1010008E88E0108DD
:10AC7000EE8E0108AA8F01083D6900086D67000883
:10AC8000419301082567000846000020E95B0008A1
:10AC90002DA4000816020020FD6C0108F40000201D
:10ACA000F57300085F610108643C0020084BEA1C52
:10ACB000084D1869FF23A8470646012E03D1064B0D
:10ACC0001E70FF236371002011B0BDE8F08F00BF3C
:10ACD000EC000020995D00084600002010B5094BEB
:10ACE00004469847C0B208E0235C01382F2BC0B25D
:10ACF00003D120182F3B437001E00028F4D12046F7
:10AD000010BD00BFB10400082DE9F04F054683488F
:10AD10009DB0037E2F2B03D018308149814B98477B
:10AD20008148824CA047DFF80882064648B97C4932
:10AD30007C4B7D4898477C48A0470646002800F099
:10AD4000D18098F800107A4CFF2955D1794F2346CD
:10AD5000284631463A46784CA047784D3B782946FC
:10AD60000093774C82460DF16F0276483346A04738
:10AD7000BB462C780A253AE09BF800102846C4EB25
:10AD8000010CDCF1000141EB0C016F4BDFF8A491E9
:10AD900098474CB999F800102846D1F1010138BF05
:10ADA00000216A4B98471EE0B4421CD2611E642306
:10ADB000C9B202AA5C48664FB84799F8002041B270
:10ADC000C4EB020EDEF1000242EB0E022846614B9C
:10ADD000984799F800202846131B5A4242EB030279
:10ADE00002A95D4B984716350134EDB2A4B29DF827
:10ADF0006F30A342C0D884E000297CD0013964239D
:10AE0000564D4948C9B202AAA847012805460DD1A6
:10AE10004349534E4448B047434802A9B047514BB9
:10AE20001D70444B1D70FF23237073E058B94E4BC7
:10AE30003D4898474B4A012313703E4A28461370F9
:10AE4000FE33237067E0022853D102A84749484CDB
:10AE5000A04720B902A84749A04700283FD0464C48
:10AE600000204649A0472F4D45494648A847464E31
:10AE7000444A42F2884302A94448B047002044496A
:10AE8000A04700204349A04700204349A047002095
:10AE90003C49A04700204149A0473A483D49404B22
:10AEA00098470646A0B902A93E48A84730463E4901
:10AEB000A04730463349A04730463C49A04730467A
:10AEC0003B49A04730463549A0473A4B984702E0F6
:10AED00039483A4B98472F492A48A84702E0364854
:10AEE000364B98471F4B01201870FF2388F800301D
:10AEF00011E004280ED11B4B01201870FF23237092
:10AF000009E0BAF1010F05D1164B83F800A0FF2329
:10AF100088F8003000201DB0BDE8F08FE43D00202F
:10AF2000B18F0108F5030008FC3D002061270008EF
:10AF3000E80000200B060020256C0008F105002029
:10AF400099770008B38F0108596B0008E96B000876
:10AF5000512900089D67000801670008DD270008E7
:10AF6000D101000846000020DDAC00080B8C010870
:10AF700075080008118C010891700108B88F01084C
:10AF8000C88F0108E41700208D280008EA84010812
:10AF9000CE8F0108B88B0108DC8F0108E884010816
:10AFA00019020008FC3C0020E38F0108E18F010832
:10AFB000FC170020915B0008EC8F01087D730108ED
:10AFC0002DE9F04F05468B489DB0037E2F2B03D013
:10AFD00018308949894B984789488A4CA0470130E5
:10AFE000C6B2DFF8288276B98349844B84489847F3
:10AFF0008348A047064630B9834B01241C70FF23C9
:10B0000088F800304FE198F80010804CFF2955D1A6
:10B010007F4F2346284631463A467E4CA0473B7830
:10B020007D4C009321467D4D82460DF16F027C4898
:10B030003346A847BB4624780A253AE09BF800101F
:10B040002846C4EB010CDCF1000141EB0C01754B0F
:10B05000DFF8BC9198474CB999F800102846D1F117
:10B06000010138BF0021704B98471EE0B4421CD24A
:10B07000611E6423C9B202AA61486C4FB84799F8AF
:10B08000002041B2C4EB020EDEF1000242EB0E02E0
:10B090002846674B984799F800202846131B5A42C8
:10B0A00042EB030202A9634B984716350134EDB217
:10B0B000E4B29DF86F30A342C0D8E7E019B9524B13
:10B0C00001251D7093E0013964235B4E4C48C9B2E1
:10B0D00002AAB047012806460DD14749574D4848B6
:10B0E000A847474802A9A847474B1E70484B1E7007
:10B0F000FF232370D6E058B9514B41489847424A44
:10B1000001231370424A1370FE3323703446CAE0A1
:10B11000022835D14B4B1A78012A01D900221A7026
:10B12000484EFF23484C494829463246A04701284B
:10B130004FF0000440F0B7803578012D40F0B38027
:10B140002F483470A0F5185202A9183A42F28843E9
:10B150003F4EB04738B120463E493F4B98473F48A5
:10B160003F4B984707E002A9244B3E4898473E4B87
:10B170009847254B1D70FF2388F800302C4692E03D
:10B18000042840F08F80394902A81C4EB047384946
:10B190002A4B02A8984702A83649374B98470028FF
:10B1A0007ED0002035492C4DA8471548284FA0F5E2
:10B1B000185202A9183A42F28843B847124F804603
:10B1C00070B100202E49A84700200FFA88F12D4BBE
:10B1D000984700202C49A8472048214B984704E075
:10B1E000204802A9B047204B984701253D70FF2316
:10B1F0002370C3E7E43D0020B18F0108F503000888
:10B20000FC3D002061270008460000208901002045
:10B21000C1050020256C0008C305002099770008AF
:10B22000FC8F0108596B0008E96B000851290008E0
:10B230009D67000801670008DD270008D1010008AC
:10B24000DDAC0008DC05002029730008019001082E
:10B250002D2A00081C900108917001083790010800
:10B260007D730108FC3C0020915B0008FC17002066
:10B27000B58401080B8C010875080008439001088B
:10B2800059900108157101082C900108BAF1010FBD
:10B2900008D1074B83F800A0FF2388F8003001E0B5
:10B2A000044600E0002420461DB0BDE8F08F00BF3A
:10B2B000460000202DE9F04F05466C489DB0037E06
:10B2C0002F2B03D018306A496A4B98476A486B4C59
:10B2D000A047DFF8AC81064648B96549654B66482A
:10B2E00098476548A0470646002800F0AA8098F8CD
:10B2F0000010634CFF295ED1624F23462846314639
:10B300003A46614CA0473B78604C00932146604D23
:10B3100083460DF16F025F483346A847BA4624784A
:10B320000A2543E09AF800102846C4EB010CDCF132
:10B33000000141EB0C01584BDFF8489198474CB99C
:10B3400099F800102846D1F1010138BF0021534B74
:10B35000984727E0B44225D2611E64234648C9B20B
:10B3600002AA4F4FB847042804D199F80020284674
:10B370004C4905E002280BD099F800204A4928469C
:10B38000C4EB020EDEF1000242EB0E02474B98477F
:10B390009AF800202846131B5A4242EB030202A9E6
:10B3A000434B984716350134EDB2E4B29DF86F3047
:10B3B000A342B7D84CE029B93E4B01201870FF23B7
:10B3C00023704FE001396423354E2B48C9B202AADD
:10B3D000B047012806460DD12549374D2648A847D4
:10B3E000254802A9A847334B1E70264B1E70FF2329
:10B3F000237036E058B9314B1F4898472D4A012336
:10B400001370204A30461370FE3323702AE002285E
:10B4100027D12B4B1A78012A01D900221A70284C07
:10B420002946FF2327482246274DA847012818D13F
:10B430002378012B05D1013B23700F4802A9234B30
:10B4400098471C4B01201870FF2388F8003009E052
:10B45000BBF1010F05D1174B83F800B0FF2388F82B
:10B46000003000201DB0BDE8F08F00BFE43D00209B
:10B47000B18F0108F5030008FC3D0020612700089A
:10B48000BC000020FD050020256C000801060020FE
:10B4900099770008FC8F0108596B0008E96B0008D8
:10B4A000DD2700086D900108419301082567000819
:10B4B0000167000846000020D1010008DDAC00084B
:10B4C000150600207190010829730008052B00085B
:10B4D0002DE9F04F874D8FB0874C8146A0472B78E0
:10B4E000FF2B40F082814FF00A08A0F10C0696FB7A
:10B4F000F8F6F6B28148824B98474FEA460A814FE8
:10B50000402191FBFAF13A4601312B4648467E4DE7
:10B51000DFF80492A847C8470C3800EBD070401001
:10B5200080B20690A0473B78A0F10B055B0095FB2D
:10B53000F6F55E43C8470746A0477A1E431E012121
:10B54000002000910190414602900390D2B2DBB2FC
:10B550006E4FB84706990698C9B2F6B2400801F195
:10B5600008035FFA80F9DBB206F1010B564409F1DA
:10B570000408EAB299440A35013609905FFA88F85E
:10B580000A9107935FFA89F90B92EDB20D960C249C
:10B5900020E1059E5E4A7301D31838339B796FF022
:10B5A00063015BB28B42B8BF0B46069F642BA8BFFA
:10B5B000642303FB07F0C921DDF824C090FBF1F1FF
:10B5C000614489B2002B0C914FF0010301F1040298
:10B5D0000DDD0093FE330193643B0293963B03938E
:10B5E00040462146D2B22B46484EB0470BE000936E
:10B5F000FF230193FA3B02930393D0B221464246C4
:10B600002B46424FB84704F1020AFF269B275FFAF8
:10B610008AFA4046214642465346DFF800C100966A
:10B6200001970297E047AB1EDBB2194608934046EC
:10B6300042462B46DFF8E4C0009601970297E047A8
:10B640000C99DFF8D8C0081DC0B202465146089BCD
:10B65000009601970297E04705982D4942018A1804
:10B660002C32104604922B4B9847A8EB50005146C1
:10B67000049A3346DFF8A8C000960196C0B2E047AE
:10B680000A980023021D009304202146D2B22B46C3
:10B69000DFF878C0019602960396E0471C484FEA0F
:10B6A0004B13C31838339B796FF063025BB293423C
:10B6B000B8BF1346069A642BA8BF642303FB02F1AC
:10B6C000DDF824C0C92291FBF2F26244079892B2DD
:10B6D000002B05924FF00103024423DD0093043355
:10B6E00001960393029748462146D2B22B46074E55
:10B6F000B04722E08A0100206361010889900108B7
:10B70000B56D0008C7050020256C0008AD5B010879
:10B71000E41700203D5E01085F610108015D01083A
:10B720006D5E01080093052302930393D0B2019646
:10B7300021464A462B46324FB847FF269B272146D3
:10B7400000960197029748464A465346DFF8B4C030
:10B75000E0472B46DFF8ACC00096019702974846B9
:10B7600008994A46E0470799059A089B8818C0B28D
:10B7700002460096019702975146224FB847DFF8DC
:10B7800094C04FEA4B1767442C3738461E49884708
:10B79000A9EB50003A4633460096019651461B4F9E
:10B7A000C0B2B847DDF828C000234FEA4C02083287
:10B7B000009301960296039621462B46079802F0C5
:10B7C000FE020F4EB0470B9F0BF1020BE419ED196F
:10B7D000E4B2EDB2DDF834C0E3450CD00BF1FF303C
:10B7E0003F2805907FF7D5AE05E0094B0120187082
:10B7F000FF232B7000E000200FB0BDE8F08F00BFEA
:10B80000AD5B0108015D01083D5E01086D5E010848
:10B8100046000020E41700202DE9F04F8E4D91B036
:10B820008E4C8146A0472B78FF2B40F092814FF041
:10B830000A08A0F10C0696FBF8F6F6B28848894B88
:10B8400098474FEA460A884F402191FBFAF13A4661
:10B8500001312B464846854DDFF81C92A847C84762
:10B860000C3800EBD070401080B20890A0473B78B5
:10B87000A0F10B055B0095FBF6F55E43C847074654
:10B88000A0477A1E431E01210020009101904146ED
:10B8900002900390D2B2DBB2754FB847089908986E
:10B8A000C9B2F6B2400801F108035FFA80F9DBB2D1
:10B8B00006F1010B564409F10408EAB299440A352D
:10B8C00001360B905FFA88F80C9109935FFA89F9B9
:10B8D0000D92EDB20F960C2430E1664A079E1823B4
:10B8E00003FB062303F5026318339B8814211BB264
:10B8F00093FBF1F378398B42B8BF0B46089F642B5A
:10B90000A8BF642303FB07F0C921DDF82CC090FB1E
:10B91000F1F1614489B2002B0E914FF0010301F166
:10B9200004020DDD0093FE330193643B0293963BCA
:10B93000039340462146D2B22B464D4EB0470BE012
:10B940000093FF230193FA3B02930393D0B2214665
:10B9500042462B46464FB84704F1020AFF269B2772
:10B960005FFA8AFA4046214642465346DFF80CC148
:10B97000009601970297E047AB1EDBB219460A9387
:10B98000404642462B46DFF8F4C0009601970297E6
:10B99000E0470E990A9B081DC0B202465146DFF8E7
:10B9A000DCC0009601970297E0470798314B1821B9
:10B9B00001FB003202F502620C3210460692DFF8FB
:10B9C000C0C0E047A8EB50005146069A3346DFF866
:10B9D000B4C000960196C0B2E0470C980023021D47
:10B9E000009304202146D2B22B46DFF884C0019692
:10B9F00002960396E0471F49182000FB0B1C0CF52C
:10BA000002631B189B8814221BB293FBF2F3783A53
:10BA10009342B8BF1346089A642BA8BF642303FB64
:10BA200002F1DDF82CC0C92291FBF2F262440998C0
:10BA300092B2002B07924FF00103024424DD0093E1
:10BA4000043301960393029748462146D2B22B460F
:10BA5000074EB04723E000BF4500002063610108A6
:10BA600098900108B56D0008DF050020256C0008DE
:10BA7000AD5B0108E41700205F610108015D01086A
:10BA80003D5E01086D5E0108009305230293039358
:10BA9000D0B2019621464A462B46334FB847FF267F
:10BAA0009B27214600960197029748464A465346EF
:10BAB000DFF8B8C0E0472B46DFF8B0C0009601972A
:10BAC000029748460A994A46E0470999079A0A9B0D
:10BAD0008818C0B202460096019702975146234F3C
:10BAE000B847DFF898C0182707FB0BC707F50267B0
:10BAF0000C3738461E498847A9EB50003A46334672
:10BB00000096019651461B4FC0B2B847DDF830C0D1
:10BB100000234FEA4C0208320093019602960396E6
:10BB200021462B46099802F0FE020F4EB0470D9FAA
:10BB30000BF1020BE419ED19E4B2EDB2DDF83CC0F3
:10BB4000E3450CD00BF1FF303F2807907FF7C5AEDF
:10BB500005E0094B01201870FF232B7000E0002046
:10BB600011B0BDE8F08F00BFAD5B0108015D0108B9
:10BB70003D5E01086D5E010846000020E4170020CC
:10BB80002DE9F04FA84C93B0A4F51250A74B94F8B0
:10BB900008A094F809B0A67A9847A54B98470123C6
:10BBA0008DF84130DB188DF8423001338DF8433089
:10BBB00001338DF8443001338DF8453001330027CF
:10BBC0008DF84630013384F808A08DF8407084F871
:10BBD00009B08DF84730A672964C780120182C30A9
:10BBE0009549964D0137A847402FF5D1403F182081
:10BBF00000FB074000F502600C308F490137A84771
:10BC0000402FF4D10020342101FB0041FF2301F536
:10BC1000A45181F8343001F1300238310B724FF009
:10BC2000FE0E9B3B4B72013082F808E0FD220A7148
:10BC30004B71643B40287F4F8B71E4D187F84A30C9
:10BC400087F8493087F8482087F86A3087F86930E4
:10BC500087F8682087F88A3087F8893087F8882045
:10BC600087F8AA3087F8A93087F8A82007F5105779
:10BC70002F3A87F8552087F8572087F8592087F8FA
:10BC80005B2087F85430013387F85630013387F84A
:10BC90005830013387F85A30694B102E00F25C8718
:10BCA000DFE816F011001100110011001100110061
:10BCB0000903090309035A075A07DC05DC055A077B
:10BCC0009D0664069D060022711E84F828201046F9
:10BCD0000132042908D8DFE801F007030303060056
:10BCE00084F8280002E0022284F82820554853F8FE
:10BCF0002610A847BAF1020F18D0BAF1030F1ED0D0
:10BD0000BAF1000F4FF003080CBF4FF0020C4FF0D8
:10BD1000010CCDF82080CDF818C00CBF4FF0010801
:10BD20004FF0020818BF4FF0000A0EE00020032178
:10BD300008904FF00108CDF818A0079107E0002205
:10BD4000012308924FF002080693CDF81CA0079F2C
:10BD50003D49780120182C30A847DDF818A03B4950
:10BD60004FEA4A1020182C30A8474FEA48102018F4
:10BD700037492C30A847DDF820C036494FEA4C102F
:10BD800020182C30A84734493448A8479DF8420071
:10BD900033494001201800F5B670A84731493248B0
:10BDA000A84732493248A84732493348A84733495F
:10BDB0003348A84733483449A84700220123BBF140
:10BDC000030F73D8DFE80BF0020E20628DF84130CC
:10BDD00002238DF8423001338DF843308DF8402036
:10BDE00001331CE08DF8403002238DF84130023BD6
:10BDF0008DF8423003338DF8433001338DF84430F1
:10BE000003338DF8453051E08DF8413003238DF830
:10BE10004230013B8DF843308DF8402002338DF8DD
:10BE200044300133EDE700BF643C0020F94A0008CC
:10BE30006D4E0008E4170020AA8F0108F5030008E2
:10BE40003C010020FC170020A8900108AD900108DB
:10BE50004B8B0108B2900108B8900108901800209F
:10BE6000C09001080C8F0108101A0020118F0108E2
:10BE7000701A0020C9900108501A0020CC900108C7
:10BE8000D0190020F0190020D39001088DF844301B
:10BE900002238DF8413001338DF8453001338DF8A0
:10BEA000433001338DF840208DF842309DF840102A
:10BEB0004FF0180909FB01FA04EB0A0000F50260D3
:10BEC00009910C307949A8479DF8412078490B9297
:10BED00009FB02F2A01800F5026003920C30A8479B
:10BEE0009DF842B0734909FB0B4000F502600C302D
:10BEF000A8479DF84330704909FB034000F50260F4
:10BF00000D930C30A8479DF844C06C4909FB0CF315
:10BF1000E01800F502600493CDF828C00C30A84763
:10BF20009DF84500664909FB00FC0C9004EB0C00F1
:10BF300000F50260CDF814C00C30A8479DF84610FB
:10BF4000604F09FB014000F502600E910C305E4924
:10BF5000A8479DF847005D490F9009FB004000F598
:10BF600002600C30A84707F50E60A2440C30584917
:10BF7000A8470AF502650020FD214D44A8726872A9
:10BF80002972049BE31803F502634B4498725872BC
:10BF90001972039AA21802F502624A449072507212
:10BFA0001172DDF814C0644404F502644C44A072BC
:10BFB00060722172079A07F5A45484F83420099B13
:10BFC00007F5A6521370642353700A9D4FF09C0C22
:10BFD00009F1E609957082F803C084F8389084F876
:10BFE0003C1084F83EC084F83D30DDF818A0012EE6
:10BFF00082F828A00B9C82F8344082F835300C9DE2
:10C0000082F8365082F8373082F82C9082F830105F
:10C0100082F832C082F83130DDF820A007F5A8524E
:10C0200082F81CA00D9C08F1020A82F8284007F54E
:10C03000A95482F8293084F8009082F8241007F57A
:10C04000AC5482F826C082F8253007F5AE5241D8AC
:10C050004FEA4A1A574401250426BD7102F8706C54
:10C06000DDF838A002F864AC02F8633C02F86C9C7E
:10C0700002F8681C02F866CC02F8673C84F8048079
:10C0800084F810B0637484F80890217384F83860E1
:10C09000DDF824C082F804C053710A9D9571D371F4
:10C0A00084F83C90117090705370C3E0D9900108EF
:10C0B000E09001084B8B0108B2900108E79001085D
:10C0C000EE900108E4170020B8900108CC90010818
:10C0D000D39001084FEA4A1A07EB0A054FF0010A0C
:10C0E00085F806A00D95C74D4FF00E0A85F8108013
:10C0F00085F81CB06B7785F81490297685F81AC0FE
:10C100006B7684F804A00F9D25740825637484F869
:10C110000890217384F80EC0637384F83880157119
:10C120000735537184F83C50117082F802C0537087
:10C130000D9DFF242C720BF10A0507F50654A84645
:10C1400007F5075584F834B084F8389084F83C102B
:10C1500084F83E0084F83D3085F800804B2584F853
:10C1600042304FF0EC0884F8415007F50A5484F847
:10C1700034B084F838A084F8398084F83AC084F860
:10C180003C1084F83E0084F83DC007F50B5C8CF849
:10C1900000104FF0140C84F84200042E84F8413053
:10C1A00084F844B084F848A084F849C00CF1A60C87
:10C1B00084F84A8084F84C1084F84E0084F84DC00E
:10C1C00084F8501084F8520084F8513032D112248F
:10C1D00082F83040079E82F82C60DDF82C80B5266E
:10C1E00082F8388082F83950DDF830A082F83AA021
:10C1F00082F83B6082F8341082F8360082F83530DD
:10C2000007F5B05282F82440DDF818C007F5B157A1
:10C2100087F800C0099C82F82C4082F82D500A9EB5
:10C2200082F82E6082F82F5082F8281082F82A00B7
:10C2300082F82930744A079FFD2100242D20102503
:10C2400082F8347082F8385082F83C1082F83E4010
:10C2500082F83D00DDF81880134603F8408F1D7109
:10C2600019729C725872DDF820A083F80CA01D741E
:10C2700019759C7558751334053082F8F47082F87E
:10C28000F84082F8FC1082F8FE00193082F8FD00B8
:10C2900002F5807382F8008182F8044182F8081167
:10C2A00014229A72587283F80CA01C7419759A752E
:10C2B000587500F08ABC042284F82820534853F8AB
:10C2C0002610A847BAF1020F16D0BAF1030F1BD0FF
:10C2D000BAF1000F4FF0030CCDF818C00CBF4FF0AF
:10C2E00001084FF002080CBF4FF002094FF001099E
:10C2F00018BF4FF0000A0DE00020D14606904FF025
:10C3000001084FF0030A05E0002106914FF00208F2
:10C310004FF001094FEA4A1020182C303C49A84739
:10C320004FEA491020182C303A49A8474FEA4810E4
:10C3300020182C303849A847069A3849500120184F
:10C340002C30A84736493748A84737493748A847C7
:10C3500037493848A84738493848A84738493948FC
:10C36000A84739493948A8470AF102035B01E31895
:10C37000187A3749400120182C30A84709F10203E8
:10C380005B01E318187A3349400120182C30A84784
:10C3900008F102035B01E318187A2F4940012018C5
:10C3A0002C30A847069F2D49BB1C5B01E318187A67
:10C3B0000027400120182C30A84784F8E070284955
:10C3C00084F8DE702748A84784F80071264984F86D
:10C3D000FE702648A84784F82071254984F81E710C
:10C3E0002448A84784F84071234884F83E712349C3
:10C3F000A8470523BBF1030F67D8DFE80BF05841CE
:10C400004B5800BF242D0020A4290020FC17002039
:10C41000F5900108FA900108FF900108B290010818
:10C420000C8F0108101A0020118F0108F01900204C
:10C43000C9900108501A0020CC900108D0190020A2
:10C4400005910108701A00200A9101089018002037
:10C45000159101081F9101082991010834910108E3
:10C4600040910108B01800204F910108D018002019
:10C470005E910108F0180020101900206991010850
:10C4800001228DF8413002238DF842308DF8402092
:10C490009B1808E08DF8403001238DF84130DB18FF
:10C4A0008DF8423001338DF84330033B0BE001231C
:10C4B0008DF84130DB188DF8423001338DF8433070
:10C4C0008DF8407001338DF844309DF840304FF0C6
:10C4D000180B0BFB034C0CF5026C0CF10C0C6046BA
:10C4E0000493CDF814C0D149A8479DF84120D04FFE
:10C4F0000BFB02F0211801F502610C310392099047
:10C5000007910846CB49A8479DF842100BFB01F064
:10C510000A90201800F5026008910C30C649A8471F
:10C520009DF84300C5490BFB00F00B90201800F567
:10C5300002600C30A8479DF844100BFB01FB04EB94
:10C540000B0000F502600C30BD49A84707F50A60F2
:10C550000430BC49A847062E07F5A65407F5A45693
:10C5600007F5A855039A049BDDF814C05ED108F1C5
:10C5700002004001012138188171DDF828C007EB65
:10C580000C0080F83E18DDF824C007EB0C0080F8A2
:10C590003E18DDF82CC007EB0C005F4480F83E1815
:10C5A00087F83E18563186F834A0237061705231F6
:10C5B000A2704FF0FE0CE170FD274539002086F88F
:10C5C00038C086F83C7086F83E0086F83D10CE26CE
:10C5D00084F8289084F8343084F8356084F8362064
:10C5E00084F83760089E84F8386084F8391084F83D
:10C5F0002CC084F8307084F8320084F8311085F84B
:10C600001C8085F8283085F8291085F82A2085F8BF
:10C610002B1085F82C6085F82D1084F860C085F803
:10C62000247085F8260085F8251038E060460392CE
:10C630000493854F8549B84785490798B84786F8D8
:10C6400034A0049BFE272370FD2064230021637027
:10C6500086F8387086F83C0086F83E1086F83D3043
:10C6600084F82890DDF820C084F834C084F8353090
:10C6700084F82C7084F8300084F8321084F831305B
:10C6800085F81C80039A85F82820724A85F829309D
:10C69000177085F8240085F8261085F825306E4A35
:10C6A000642182F810809DF843C0FE26082382F89A
:10C6B0001CC0517716751376DA339376C43B5376E4
:10C6C00082F844809DF84470FD20002582F8507067
:10C6D00082F8511082F8486082F84C0082F84E507F
:10C6E00082F84D10DDF81880042402F5546382F8B6
:10C6F000788082F884C082F885104FF0130C82F89D
:10C700007C6082F8800082F8825082F8811082F882
:10C71000AC40013482F8B84082F8B91082F8B060B9
:10C7200082F8B40082F8B65082F8B51083F83470FD
:10C7300083F838C0ACF10C0C83F83CC00CF1210C30
:10C7400083F83EC00CF1B00C83F83DC04FF00E08EA
:10C750004FF0140C82F8800D83F8425083F841109A
:10C7600083F8447083F8488083F849C00CF1D80CF2
:10C7700083F84AC083F84C40013483F84E5083F864
:10C780004D1083F85040963483F8525083F851404E
:10C7900083F8547083F8588083F859C083F85A405E
:10C7A00083F85C0083F85E5083F85D1083F86000C6
:10C7B00083F8625083F861409DF8401002F54463AD
:10C7C00083F83410322183F8386083F83C0083F812
:10C7D0003E1083F83D1082F8800C83F8421083F8F5
:10C7E00041109DF8412083F8442083F8486083F885
:10C7F0004C0083F84E1083F84D1083F8500083F8F6
:10C80000521083F851109DF8422083F8542083F889
:10C81000586083F85C0083F85E1083F85D1083F83D
:10C82000600083F8621083F86110CEE1779101080F
:10C83000E41700207E910108FA900108B2900108E7
:10C840004B8B01080A910108F5030008F5900108D7
:10C85000FF900108042D0020242D00200D2253F804
:10C86000261084F82820A848A847A849A848A8471F
:10C87000A849A948A847A949A948A847A949AA4831
:10C88000A847AA49AA48A8479DF84090182606FB41
:10C89000094000F50260A7490C30A8479DF8418087
:10C8A000A54906FB084000F502600C30A8479DF83A
:10C8B0004270A24906FB074000F502600C30A84711
:10C8C0009DF843A09E4906FB0A4404F502600C3023
:10C8D000A8479C49012381F834300B4603F8408F68
:10C8E0006422FD249C20FE25183E5A709F70DA7049
:10C8F00083F804A05A7181F8385081F83C4081F8DF
:10C900003E6081F83D2083F8286083F8349083F8F6
:10C91000352083F82C5083F8304083F8320083F8B8
:10C92000312081F89C60032381F8A88081F8A92038
:10C9300081F8AA70122781F8AB0081F8A07081F805
:10C94000A44081F8A60081F8A52081F8D0309DF898
:10C95000443081F8DC3081F8DD2081F8D45081F852
:10C96000D84081F8DA0081F8D9202EE1132284F82A
:10C970002820D96B6448A847002101200A463E2997
:10C9800026DC342606FB0246642506F5A45300F196
:10C99000010C06F5A65683F8342083F8401083F87E
:10C9A000415083F8420083F8435086F804C000F1F8
:10C9B000020C757186F806C0F571FE2683F83860A2
:10C9C000013E83F83C60FD3E83F83E6083F83D50B5
:10C9D000013204300431402AC0B2D0D1F5E0132234
:10C9E00084F82820484853F82610A84700274FEA23
:10C9F000471804EB080A0AF12C0A53495046A84785
:10CA00005046DFF84CA1D04740444FF0010C0022C3
:10CA1000791C2018CDF800C02C301346CDF814C076
:10CA200009B2DFF830B1D847A044002288F840208E
:10CA3000102E5FFA87F9DDF814C004D1043288F8AB
:10CA4000412088F842C0B9F10F0F21D80C2303FB15
:10CA50000743FF2003F58E5282F83490FD2182F8BF
:10CA60003800FF3882F83C1082F83E002D3082F802
:10CA70003D0003F594533222D13083F8349083F88B
:10CA8000380083F83C1083F83E20921883F83D204C
:10CA90000137402FABD10023342202FB034202F5C1
:10CAA000A45282F83430642182F84030FE260133EB
:10CAB00082F84110FD2082F83860FE3E402B82F85B
:10CAC0003C0082F83E6082F83D10E5D14FF0180836
:10CAD00008FB06F804EB080707F502670C371B494B
:10CAE0003846A8473846D047404420180123002242
:10CAF000013600F5026000930C3031B21346D8477E
:10CB0000402EE3D161E000BFFC17002085910108B1
:10CB1000101800208D91010830180020969101080E
:10CB2000501800209A91010870180020A491010863
:10CB3000501A0020AD910108B3910108BA91010883
:10CB4000C1910108642C0020C8910108D19101080D
:10CB5000B104000865520008052253F8261084F835
:10CB600028201C48A8471C491C48A8471C491D48A8
:10CB7000A8471D491D48A8471D481E49A8470D2E16
:10CB800005D11023FB73093B7B73073BBB73002369
:10CB9000342202FB0342FE2002F5A452FD2582F856
:10CBA000343082F8380082F83C50613D82F83E50C3
:10CBB000383D82F83D5082F84030013302F13001B7
:10CBC000102B82F841500872E2D1012013B0BDE869
:10CBD000F08F00BFFC17002085910108101800207D
:10CBE0008D910108301800209691010850180020FE
:10CBF00070180020D89101082DE9F0473D4C88B00D
:10CC000063780546FF2B264666D12246631C0846FC
:10CC1000394C1121A0473378384C0DF11F022146C1
:10CC20002846DFF810810093354D1123A847C047EF
:10CC3000344B354F93F84A908246B8470546C04773
:10CC4000C9EB0A09034601220020009201902A46FE
:10CC500002902E4D03905FFA89F1A847B8462478D8
:10CC60000A2533E0317828460A1B514241EB020184
:10CC7000274B9847102C25D81E4B28461A78254B51
:10CC8000254F53F82410131B5A4242EB0302234B47
:10CC90009847234BFF2219572846224B9847C047F5
:10CCA000214B05F115021B780092DB430022C318CB
:10CCB00001920292039204920592204602212A4692
:10CCC0009BB2B84716350134EDB2E4B29DF81F307F
:10CCD000A342C7D8002009E013701046134B01216E
:10CCE0009847134B01201870FF23637008B0BDE80C
:10CCF000F08700BFD4000020256C0008E505002067
:10CD000099770008643C00205F610108FD59010823
:10CD1000596B00083C010020E95C0008016700082D
:10CD2000A88D01089D67000888010020E95B0008C4
:10CD300046000020636101082DE9F0473B4C88B0B4
:10CD400063780546FF2B264662D12246631C0846BF
:10CD5000374C0421A0473378364C0DF11F02214691
:10CD60002846DFF800810093334D0423A847C047CD
:10CD7000324B334F93F84A908246B8470546C04736
:10CD8000C9EB0A09034601220020009201902A46BD
:10CD900002902C4D03905FFA89F1A847B846247899
:10CDA0000A252FE031782846C4EB010EDEF10001A0
:10CDB00041EB0E01244B9847032C1FD81B4B2846F0
:10CDC0001A78224B171B7A4242EB070253F82410C1
:10CDD0001F4B9847C0471F4B05F115021B78009267
:10CDE000DB430022C318019202920392049205923F
:10CDF000204602212A469BB2174FB8471635013408
:10CE0000EDB2E4B29DF81F30A342CBD8002009E078
:10CE100013701046114B01219847114B01201870D7
:10CE2000FF23637008B0BDE8F08700BF0002002058
:10CE3000256C0008C205002099770008643C00209A
:10CE40005F610108FD590108596B0008D8000020F6
:10CE50000167000888010020E95C0008E95B000820
:10CE600046000020636101082DE9F0473B4C88B083
:10CE700063780546FF2B264662D12246631C08468E
:10CE8000374C0421A0473378364C0DF11F02214660
:10CE90002846DFF800810093334D0423A847C0479C
:10CEA000324B334F93F84A908246B8470546C04705
:10CEB000C9EB0A09034601220020009201902A468C
:10CEC00002902C4D03905FFA89F1A847B846247868
:10CED0000A252FE0317828460B1B594241EB03010C
:10CEE000254B9847032C21D81C4B28461A78234BF6
:10CEF000C4EB020CDCF1000242EB0C0253F82410EC
:10CF00001F4B9847C0471F4B05F115021B78009235
:10CF1000DB430022C318019202920392049205920D
:10CF2000204602212A469BB2174FB84716350134D6
:10CF3000EDB2E4B29DF81F30A342CBD8002009E047
:10CF400013701046114B01219847114B01201870A6
:10CF5000FF23637008B0BDE8F08700BFBA0000206F
:10CF6000256C0008C505002099770008643C002066
:10CF70005F610108FD590108596B00081800002085
:10CF80000167000888010020E95C0008E95B0008EF
:10CF900046000020636101082DE9F0473B4C88B052
:10CFA00063780546FF2B264662D12246631C08465D
:10CFB000374C0521A0473378364C0DF11F0221462E
:10CFC0002846DFF800810093334D0523A847C0476A
:10CFD000324B334F93F84A908246B8470546C047D4
:10CFE000C9EB0A09034601220020009201902A465B
:10CFF00002902C4D03905FFA89F1A847B846247837
:10D000000A252FE031782846C4EB010EDEF100013D
:10D0100041EB0E01244B9847042C1FD81B4B28468C
:10D020001A78224B171B7A4242EB070253F824105E
:10D030001F4B9847C0471F4B05F115021B78009204
:10D04000DB430022C31801920292039204920592DC
:10D05000204602212A469BB2174FB84716350134A5
:10D06000EDB2E4B29DF81F30A342CBD8002009E016
:10D0700013701046114B01219847114B0120187075
:10D08000FF23637008B0BDE8F08700BF8001002077
:10D09000256C0008CA05002099770008643C002030
:10D0A0005F610108FD590108596B0008C0000020AC
:10D0B0000167000888010020E95C0008E95B0008BE
:10D0C00046000020636101082DE9F04F8A4C8BB0C7
:10D0D00094F859800646B8F1FF0F914640F0D7808A
:10D0E000084604F15802052104F15903834DA8476D
:10D0F00094F8583082490DF1270230460093814D53
:10D100000523814FA847B847804EDFF820A296F844
:10D110004A500790D0478346B84707990122491BD8
:10D1200000250346009201955A460295039528462C
:10D13000C9B2DFF82CB2D84796F84A30002B3BD062
:10D14000B84796F84A2006900792D0478246B847DB
:10D15000079A069BD24399180AF1FF3A431E01220F
:10D16000C9B22846009201955FFA8AF202950395AA
:10D17000DBB2D847664D94F8583055F82300654B1C
:10D1800098478246B847644B96F84A201B7896F831
:10D190004A10CDF80080CB1A03EBD373C2EB6301C6
:10D1A00094F858304118CDF8048055F823205046A3
:10D1B000C9B24346594DA847514B0A251E7861E034
:10D1C00094F8581028468B1B594241EB0301544BED
:10D1D0009847042E52D8484B284693F85820514B74
:10D1E000C6EB020CDCF1000242EB0C0253F82610F5
:10D1F0004D4B98474D4B98474D4B05F115021B7809
:10D200000092DB430022C31801920292039204921F
:10D2100005929BB2304602212A46464FB847731EFC
:10D22000032B2BD8DFE803F0020C162099F800102E
:10D2300094F85820404B284653F82110012A18E052
:10D2400099F8011094F858203C4B284653F82110C7
:10D25000022A0EE099F8021094F85820384B28461C
:10D2600053F82110032A04E094F858203549284641
:10D27000042A14BF00220122334B98471635013689
:10D28000EDB2F6B29DF82730B34299D82FE0B8F14D
:10D29000040F2CD8DFE808F01D0309131A00214BF6
:10D2A0004A465868294DFF2305E01E4B284D9868D3
:10D2B00009F10102FF23A847012811D017E0194BFB
:10D2C00009F10202D868234DFF23F4E70846224BF8
:10D2D0009847224B01201870FF2384F8593007E04B
:10D2E0001E4B1870FF2384F85930013800E00020ED
:10D2F0000BB0BDE8F08F00BF8B010020256C00084B
:10D30000C90500209977000863610108643C00208A
:10D3100010010020215D000838010020B55E0108E1
:10D32000596B00082C000020016700085F610108AC
:10D3300088010020E95C0008D800002018000020C7
:10D340003C010020419301082567000839CD000801
:10D3500069CE0008F9CB000881BB00084600002018
:10D36000FD5901082DE9FF41C1EB030E9DF828C0CE
:10D370001FFA8EFE0CFB0EFCDCB26FF063039CFB0D
:10D38000F3FCCEB2E6446533C7B2D5B206EB0E016C
:10D3900000937F3301930293039338462A46234632
:10D3A000C9B2DFF82080C04700230093FF33019308
:10D3B00002930393384631462A462346C047BDE8C8
:10D3C000FF8100BFAD5B01082DE9F04F954B89B09F
:10D3D0000E469847944B044698470121A21F831F8D
:10D3E000FF2403200091013902910391D2B201463A
:10D3F000DBB28E4D0194A8470520009401940146AC
:10D400008B4A23468B4DA847012E05D18A4B1A78AB
:10D41000022A08D8013205E0022E04D1864B1A7880
:10D420000AB1013A1A70854A13789046CBB91A4668
:10D4300002F592618248013100EBC1010020C880F1
:10D440004FF6100088804FF4FE6008817D4900206F
:10D45000C8527D490132C8520233042AE8D101235F
:10D4600054E0012B55D1FF24784F7948B847234623
:10D470001B21774A00940194A8477648B847234671
:10D480003121744A00940194A8477348B847009426
:10D49000019423464721704AA847DFF8D4A1FF3CF6
:10D4A000B94620466D4B98470134E4B2042C2AF863
:10D4B000020FF6D1604B634F1B78002237F913102F
:10D4C0000123009305A81346654CA04705A8C8474B
:10D4D000FF235D210093019305AAA847032E40F086
:10D4E0009D806049002303F59262554C38880132D3
:10D4F00004EBC2020133D0800022042B27F8022B58
:10D5000021F8022FEFD198F80030013388F800306D
:10D5100084E0022B40F08280FF244C4F4C48B847F7
:10D5200023461B214A4A00940194A8474E48B84715
:10D53000234631214C4A00940194A8474648B847F5
:10D5400023464721444A00940194A8474748B847D6
:10D550000094019423465D21444AA847394F3A4C30
:10D560004FF00009BA46A34648463C4B984737F966
:10D57000023B09F10109984234F9023BB8BF27F890
:10D58000020C5FFA89F99842C8BF24F8020CB9F17D
:10D59000040FE9D1284F00223B78A9F10309FF24A9
:10D5A0003AF9131005A81346DFF8B4A0CDF800909F
:10D5B000D04773210A2005AA234600940194A84766
:10D5C0003B7800223BF9131005A81346CDF80090D4
:10D5D000D047642073210094019405AA2346A847EC
:10D5E000032E1BD122481F49002303F59262144CDD
:10D5F000013204EBC202D48830F8025F01332C1BE5
:10D600009480D48831F8025F042BC4EB05041481A4
:10D61000EBD1043B88F80030012000E0002009B085
:10D62000BDE8F08F5F61010863610108AD5B01082F
:10D63000449B0108B55E0108CF0500201A060020B2
:10D64000E4170020F4050020E8050020215D000813
:10D65000E1910108E8910108EF910108D96E0108F4
:10D6600065520008E6050020F6910108FB910108CB
:10D67000F20500202DE9F04F00238BB080464FF0DB
:10D6800001099A4A590151183831097A934619B952
:10D6900009F101095FFA89F90133402BF1D1B9F1A0
:10D6A000010F00F06A81924B5C781E46FF2C40F01F
:10D6B000F7801A46494601338E4D4046A8473378D5
:10D6C0008D4D00938D484B468D490DF12702A8479B
:10D6D0008C4D95F84A30002B34D0DFF87082C0476B
:10D6E00095F84A30884A0793824690470746C047D4
:10D6F000079B7A1EDB439A440121431E0020D2B2CD
:10D70000009101905FFA8AF102900390DBB27F4FA3
:10D71000B8477F4B7F4898470746C0477E4B95F8F0
:10D720004A201B7895F84A100094CB1A03EBD37368
:10D73000C2EB63014118019423463846C9B2754AC9
:10D74000764CA0476E4B0A251C78A3E0317828461A
:10D750000A1B514241EB0201714B98474C4580F046
:10D760009580F4B9624B28461A786E49D2F10102CD
:10D7700038BF00226C4B9847634B98476B4B05F1C1
:10D7800015021B780221DB43C31800920194029416
:10D7900003940494059420462A469BB2644FB847EC
:10D7A00036E04FF00008C2464FEA48130BEB030285
:10D7B00092F8407037BB621E52451FD14B4A284633
:10D7C000D318327803F12C01131B5A4242EB0302A7
:10D7D000554B98474C4B9847544B05F115021B7815
:10D7E0000221DB43C3180092019702970397049725
:10D7F000059720462A469BB24D4FB8470AF1010AC9
:10D800005FFA8AFA08F10108B8F1400FCCD14CB99F
:10D8100032782846D2F10102464938BF0022464BF1
:10D82000984733E04FF00008C2464FEA48135B4484
:10D8300038331A7A2ABB611E51451ED1597A012903
:10D840000FD19F7933787FB2C4EB030C6331DCF1E5
:10D85000000397FBF1F1284643EB0C03374FB84721
:10D860000BE032789979C4EB020EDEF10002284613
:10D8700049B242EB0E02324B98470AF1010A5FFAB5
:10D880008AFA08F10108B8F1400FCED116350134FB
:10D89000EDB2E4B29DF82730A3423FF657AF6EE0F9
:10D8A0002CB9284A01201070FF225A7068E0002429
:10D8B0002546204662010BEB02033833197A002912
:10D8C00050D17778013FAF424AD1587A01283FD1F1
:10D8D0009A7912B964329A7100E0997160015844E2
:10D8E0003E300121184B9847012039E0E417002011
:10D8F00083010020256C0008997700080292010836
:10D9000019060020643C00205F610108FD590108F0
:10D91000215D0008CF91010838010020B55E0108A3
:10D92000596B0008808E01080167000888010020FB
:10D93000E95C00084193010825670008E9670008D1
:10D940003D69000846000020E95B000863610108AA
:10D950000D4B0E489A1841463E32FF230C4FB847F4
:10D960000135EDB20134402CA4D1012807D1094B77
:10D970001870FF237370013802E0484600E0002071
:10D980000BB0BDE8F08F00BFE4170020928F0108B4
:10D99000F5730008460000202DE9F04F424E0024A8
:10D9A000737889B0FF2B07468DF81F406AD108466F
:10D9B00032460621731C3D4DA8473D4D337829461C
:10D9C0000DF11F02384600933A4F0623DFF81C91F1
:10D9D000B847C847384B394F93F84AA08346B847F1
:10D9E0008046C847CAEB0B0A012203460092204634
:10D9F00042460194029403945FFA8AF1304CA047A6
:10DA0000304B9847B8462C780A2535E031782846BF
:10DA1000C4EB010EDEF1000141EB0E012A4B9847E9
:10DA2000052C25D8204B28461A78284B171B7A42FC
:10DA300042EB070253F82410254B9847254BFF2251
:10DA400019572846244B9847C047244B05F1150227
:10DA50001B780092DB430022C318019202920392CA
:10DA600004920592204602212A469BB21C4FB847D9
:10DA700016350134EDB2E4B29DF81F30A342C5D88B
:10DA8000002007E04BB1013B137010460121154BFC
:10DA9000984702E009B0BDE8F08F134B01201870E1
:10DAA000FF237370F6E700BFB8000020256C000864
:10DAB0000706002099770008643C00205F61010898
:10DAC000FD590108B95C0008596B00086C00002082
:10DAD0000167000868A201089D670008880100200E
:10DAE000E95C0008E95B000846000020636101086A
:10DAF0002DE9F04F724D8BB06C782E46FF2C40F024
:10DB0000C3802A466B1C40216E4DA84733786E4D6A
:10DB100000936E4840236E490DF12702A8476D4DD2
:10DB200095F84A30002B33D0DFF8E881C0476A4BC4
:10DB3000814695F84AA098470746C0476FEA0A0A07
:10DB40007A1E431E01210020D144D2B200910190DF
:10DB50005FFA89F102900390DBB2604FB847604BE7
:10DB6000604898470746C0475F4B95F84A201B78A6
:10DB700095F84A100094CB1A03EBD373C2EB630100
:10DB80004118019423463846C9B2564A574CA0471B
:10DB90004F4B0A251C7872E031782846C4EB010C03
:10DBA000DCF1000141EB0C01514B98473F2C444FF5
:10DBB00061D8DFF824914F4BDFF85CA1DFF85CB14E
:10DBC000DFF85C810CBB3A784B49D2F1010238BFD7
:10DBD000002228469847C8479AF8003005F11502F8
:10DBE000DB43C3180221009220462A469BB20194CF
:10DBF0000294039404940594D84732782846D2F1CD
:10DC000001023E4938BF002234E0DFF800C13A7813
:10DC100061016144C4EB020E0C31DEF1000242EB03
:10DC20000E02CDF81CC028469847C8479AF8003025
:10DC300005F11502DB43C318009200220221019274
:10DC400002920392049205929BB22A462046D8473C
:10DC5000631CDDF81CC05B0163443A789B79C4EB1C
:10DC6000020C012B0CBF26492649DCF10002284694
:10DC700042EB0C02C04716350134EDB2E4B29DF818
:10DC80002730A34288D816E01F4E24B90120FF2375
:10DC900030706B7010E001341C4864010019837906
:10DCA0000121C3F1010300F8063F194B98470123F6
:10DCB0003370FE336B7000200BB0BDE8F08F00BFF7
:10DCC00040000020256C0008997700081192010897
:10DCD00005060020643C00205F610108FD59010831
:10DCE000215D0008CF91010838010020B55E0108D0
:10DCF000596B000801670008808E010841930108F4
:10DD000092940108948E010846000020E417002038
:10DD1000E95B00086361010888010020E95C0008F4
:10DD2000256700082DE9F04F7B4D8BB06C782E46AF
:10DD3000FF2C40F0CF802A466B1C4021774DA8472E
:10DD40003378774D00937748402377490DF12702C8
:10DD5000A847764D95F84A30002B33D0DFF80C8277
:10DD6000C047734B814695F84AA098470746C0477D
:10DD70006FEA0A0A7A1E431E01210020D144D2B262
:10DD8000009101905FFA89F102900390DBB2694F34
:10DD9000B847694B694898470746C047684B95F8AC
:10DDA0004A201B7895F84A100094CB1A03EBD373E2
:10DDB000C2EB63014118019423463846C9B25F4A59
:10DDC000604CA047584B0A251C787DE031782846E6
:10DDD000C4EB010CDCF1000141EB0C015A4B9847FC
:10DDE0003F2C4D4F6CD8DFF84891584BDFF880A19D
:10DDF000DFF880B1DFF880810CBB3A785449D2F16A
:10DE0000010238BF002228469847C8479AF80030D8
:10DE100005F11502DB43C3180221009220462A4671
:10DE20009BB201940294039404940594D8473278E9
:10DE30002846D2F10102474938BF00223FE0621E66
:10DE40004FF0180C0CFB02FCCDF81CC0079ADFF851
:10DE500014C128460CEB02013A7801F50261C4EBCB
:10DE6000020E0C31DEF1000242EB0E02CDF818C0BA
:10DE70009847C8479AF8003005F11502DB43C318EC
:10DE800000920022022101920292039204920592D2
:10DE90009BB22A462046D847079BDDF818C03A783F
:10DEA0009C440CF5026318339B792846012BC4EB84
:10DEB00002030CBF284929495A4242EB0302C047DA
:10DEC00016350134EDB2E4B29DF82730A3423FF697
:10DED0007DAF1CE0224E24B90120FF2330706B700F
:10DEE00016E01823013C5C431E480121031993F8F6
:10DEF0003E280019C2F1010200F5026083F83E28B5
:10DF00001E30194B984701233370FE336B7000208D
:10DF10000BB0BDE8F08F00BF28000020256C000882
:10DF20009977000820920108D4050020643C002065
:10DF30005F610108FD590108215D0008CF910108CA
:10DF400038010020B55E0108596B00080167000820
:10DF5000808E01084193010892940108948E010873
:10DF600046000020E4170020E95B00086361010817
:10DF700088010020E95C0008256700082DE9F04FC2
:10DF8000824C89B0657B8046FF2D164640F0CB80E1
:10DF9000084604F10C02072104F10D037C4FB84739
:10DFA000237B4046DFF8588200937A4907230DF11E
:10DFB0001F02794FB84798F84A30002B38D0DFF865
:10DFC0004492C847754B824698F84AB0984707462E
:10DFD000C8476FEA0B0BDA447A1E431E012100206A
:10DFE000D2B2009101905FFA8AF102900390DBB205
:10DFF0006B4FB847237B6B4F57F823006A4B98470A
:10E000008246C847694B98F84A201B7898F84A100E
:10E010000095CB1A03EBD373C2EB6301237B41184A
:10E02000019557F8232050462B46C9B2604DA847AA
:10E03000584B0A2593F8008070E0217B2846C8EBF6
:10E04000010CDCF1000141EB0C015A4B9847B8F18F
:10E05000060F4E4F5CD83A7B574BC8EB020EDEF1F1
:10E06000000253F8281042EB0E022846534B984703
:10E07000B8F1000F09D197F864203D21D2F10102D7
:10E08000284638BF00224E4B9847444B98474D4B8B
:10E0900005F115021B780092DB430022C3180192A0
:10E0A00002920392049205929BB2404602212A46B4
:10E0B000454FB84708F1FF33042B29D8DFE803F0B8
:10E0C000030D13191F00227B2846A2F101035A42B7
:10E0D00042EB030231463D4B19E0227B2846B6F95C
:10E0E0001010022A0FE0227B2846B6F91210032AEC
:10E0F00009E0227B2846B6F91410042A03E0227BAB
:10E10000B17D2846052A324B14BF002201229847D0
:10E11000163508F10108EDB25FFA88F89DF81F3056
:10E1200043458AD82EE0062D2CD8DFE805F0040AF6
:10E130000E1114191E00274B01201870FF23637362
:10E1400021E02548FF23254D13E02548103204E047
:10E150002448123201E024481432FF23234D08E002
:10E1600023481632FF23234D03E02348234D183262
:10E17000FF23A847012805D1164B1870FF236373AE
:10E18000013800E0002009B0BDE8F08F8B010020CD
:10E19000256C0008D3050020997700085F6101080D
:10E1A000FD590108DC8D0108215D000838010020BF
:10E1B000B55E0108596B000800A30108016700085B
:10E1C0009D67000888010020E95C000825670008B9
:10E1D0006D67000846000020D29D0108C562000856
:10E1E000928F01084B91010838950108456200089B
:10E1F000F78F0108995D0008099401086972000809
:10E20000643C0020636101082DE9F0479246444ACE
:10E2100088B0D37B0546FF2B164666D108460E32E2
:10E22000212106F10F033F4CA047B37B3E4C0093E6
:10E23000214681460DF11F02284621233B4DA84768
:10E2400024780A254CE0B17B2846C4EB010CDCF1B4
:10E25000000141EB0C01364B9847364B9847364B43
:10E2600005F115021B780092DB430022C3180192CE
:10E270000292039204920592204602212A469BB202
:10E280002E4FDFF89C80B8474CB998F80E102846FE
:10E29000D1F1010138BF0021294B98471CE0202C07
:10E2A0001AD8631E1C2707FB03A798F80E202846E0
:10E2B000C4EB020EDEF1000242EB0E023946214BA6
:10E2C000984798F80E202846131B5A4242EB030247
:10E2D000B7F910101C4B984716350134EDB2E4B273
:10E2E0009DF81F30A342AED80EE02BB9174B01208A
:10E2F0001870FF23D37310E0013B1C2202FB03A222
:10E30000134CDBB2A0478146B9F1010F04D10F4B8A
:10E3100083F80090FF23F373002008B0BDE8F08776
:10E320008B010020256C00080E060020997700085C
:10E33000596B00085F61010888010020E95C000852
:10E34000E96B0008016700086D67000846000020BF
:10E350007DDF00082DE9F04F8F4C89B0657E804647
:10E36000FF2D164640F0E280084604F1180207210E
:10E3700004F11903894FB847237E4046DFF8A08295
:10E380000093874907230DF11F02864FB84798F87D
:10E390004A30002B38D0DFF88C92C847824B824637
:10E3A00098F84AB098470746C8476FEA0B0BDA441B
:10E3B0007A1E431E01210020D2B2009101905FFA23
:10E3C0008AF102900390DBB2784FB847237E784FF2
:10E3D00057F82300774B98478246C847764B98F802
:10E3E0004A201B7898F84A100095CB1A03EBD37398
:10E3F000C2EB6301237E4118019557F82320504654
:10E400002B46C9B26D4DA847654B0A2593F800808D
:10E4100086E0217E2846C8EB0102514241EB020111
:10E42000674B9847B8F1060F5B4F73D83A7E654B40
:10E43000284653F82810C8EB02035A4242EB030265
:10E44000614B9847B8F1000F09D197F864203D213E
:10E45000D2F10102284638BF00225C4B9847524B4C
:10E4600098475B4B05F115021B780092DB430022B5
:10E47000C318019202920392049205929BB2404605
:10E4800002212A46534FB84708F1FF33052B41D8E4
:10E49000DFE803F003081C253036227E2846317859
:10E4A000012A17E077784C4B3F2F03D9227E28466C
:10E4B0004A4904E04A497F01227E28467918A2F1A0
:10E4C000020CDCF1000242EB0C0222E0227EB17869
:10E4D0002846032A14BF00220122424B19E0227E63
:10E4E000311DA2F1040EDEF10002284642EB0E02BD
:10E4F0003D4B0EE0227E284606F10801052A04E085
:10E50000227E284606F10C01062A384B14BF002251
:10E5100001229847163508F10108EDB25FFA88F834
:10E520009DF81F3043453FF674AF30E0062D2ED8DE
:10E53000DFE805F0040A0E13181D20002C4B012003
:10E540001870FF23637623E02A48FF232A4D15E045
:10E550002A480132FF232A4D10E02A480232FF23C5
:10E56000294D0BE029480432FF23294D06E02948B4
:10E57000083201E028480C32284DFF23A847012823
:10E5800005D11B4B1870FF236376013800E0002093
:10E5900009B0BDE8F08F00BF8B010020256C00089A
:10E5A000D0050020997700085F610108FD59010836
:10E5B000BCA30108215D000838010020B55E0108F8
:10E5C000596B0008308D0108016700089D6700083D
:10E5D00088010020E95C000825670008AA8F01086F
:10E5E000101800206D670008616A0008C5690008FE
:10E5F00046000020F78F0108995D0008A6930108E6
:10E600002DA40008499201082973000859920108B5
:10E61000A9A9000862920108C78E0108A5A60008F2
:10E62000643C0020636101082DE9F04F8DB0089231
:10E630006F4A9A46D37E0446FF2B164640F0AD80C3
:10E6400008461A32112106F11B036A4DA8476A4D8C
:10E65000B37E0790009320462946684C0DF12F02A7
:10E660001123A0472C780A2591E0B17E644B0A1B48
:10E67000514241EB02012846DFF890B19847D84754
:10E68000DFF8B0914FF0000899F80030CDF8048021
:10E69000DB43C31805F1150082B209900092CDF852
:10E6A0000880CDF80C80CDF81080CDF8148020467D
:10E6B00002212A469BB2534FB84754B94C4B2846C7
:10E6C000997EC8EB0103594241EB03014E4B984739
:10E6D00059E0102C57D80899631E4FF0140B0BFB10
:10E6E000031B9BF80130534514D1484A904799F8D1
:10E6F00000306FF00302D21A099FFF2382180193A2
:10E7000002930393CDF80080FBB202202946D2B2D7
:10E710003F4FB8479BF801703E4B3F2F15D9B27E53
:10E720002846C4EB020CDCF1000242EB0C023A4931
:10E730009847B27E2846C4EB020EDEF1000237494C
:10E7400042EB0E02364B98471DE0B27E35497F0101
:10E750007918171B7A4242EB0702284698472B4943
:10E76000884799F800306FF00302D21A82181620F9
:10E77000611E6B1C009003380190D2B2C8B2DBB2AC
:10E78000FF21294FB84716350134EDB2E4B29DF8A8
:10E790002F30A3423FF669AF1EE02BB9234B012077
:10E7A0001870FF23D3761FE0BAF1FF0F09D0089F3E
:10E7B0001422013B02FB03735A78FF2A08BF83F837
:10E7C00001A0F37E2046089C013B142202FB034279
:10E7D000DBB2174CA0470790079F012F03D1134BC3
:10E7E0001F70FF23F37600200DB0BDE8F08F00BF4F
:10E7F0008B010020256C0008BA05002099770008DD
:10E80000596B0008E95C0008E96B00085F610108CA
:10E81000FD59010801670008AA8F010865920108E7
:10E820002567000810180020018F0008460000200E
:10E8300055E30008880100202DE9F04F834C89B092
:10E84000657F0746FF2D904640F0D380084604F1CF
:10E850001C02052104F11D037D4EB047237F38467D
:10E860007C4F00937C4905230DF11F027B4EB0477E
:10E8700097F84A30002B38D0DFF85092C847784BD1
:10E88000824697F84AB098470646C8476FEA0B0B8E
:10E89000DA44721E431E01210020D2B20091019081
:10E8A0005FFA8AF102900390DBB26E4EB047237F8D
:10E8B0006D4E56F823006D4B98478246C8476C4B07
:10E8C00097F84A201B7897F84A100095CB1A03EB6B
:10E8D000D373C2EB6301237F4118019556F82320BF
:10E8E00050462B46C9B2634DA8475B4B0A251E789C
:10E8F0007AE0217F28468B1B594241EB03015E4B96
:10E900009847042E514F6BD83A7F5C4BC6EB020CF4
:10E91000DCF1000253F8261042EB0C022846584B5B
:10E9200098474EB997F864203D21D2F1010228465C
:10E9300038BF0022534B9847494B9847524B05F13B
:10E9400015021B780092DB430022C3180192029249
:10E950000392049205929BB2304602212A464B4F05
:10E96000B847731E032B3BD8DFE803F00217222EB3
:10E9700098F80070464B3F2F03D9227F284645491F
:10E9800004E045497F01227F28467918A2F1010E53
:10E99000DEF1000242EB0E0221E0227F2846A2F1C6
:10E9A00002035A4242EB030298F801103B4B16E077
:10E9B000227F2846A2F1030CDCF1000208F10401D9
:10E9C00042EB0C02364B0AE0227F364BA2F1040EDA
:10E9D000DEF10002284608F1080142EB0E029847DA
:10E9E00016350136EDB2F6B29DF81F30B34280D82D
:10E9F00027E0042D25D8DFE805F003090D121700E4
:10EA0000294B01201870FF2363771BE02748FF2361
:10EA1000274D0DE027480132FF23274D08E0274806
:10EA20000432FF23264D03E02648274D0832FF23FA
:10EA3000A847012805D11C4B1870FF2363770138C4
:10EA400000E0002009B0BDE8F08F00BF8B0100207E
:10EA5000256C0008643C0020BE0500209977000862
:10EA60005F610108FD5901081C8D0108215D000846
:10EA700038010020B55E0108596B0008548E01086A
:10EA8000016700089D67000888010020E95C000814
:10EA900025670008AA8F0108101800206D6700087C
:10EAA000616A0008C569000846000020A6930108B5
:10EAB0002DA40008F78F0108995D000859920108FC
:10EAC000A9A900086C920108A5A6000863610108C5
:10EAD0002DE9F04F91466F4A8DB00893D37F0446DD
:10EAE000FF2B164640F0AD8008461E32112106F17C
:10EAF0001F03694DA847694DB37F079000932046D7
:10EB00002946674C0DF12F021123A0472C780A25C6
:10EB100091E0B17F634B0A1B514241EB0201284651
:10EB2000DFF88CB19847D847DFF8ACA105F11501A3
:10EB30009AF800304FF00008DB438AB2C3180991FD
:10EB40000092CDF80480CDF80880CDF80C80CDF887
:10EB50001080CDF81480204602212A469BB2524FE5
:10EB6000B84754B94B4B2846997FC8EB010359422B
:10EB700041EB03014D4B984759E0102C57D8631EC9
:10EB80004FF00C0B0BFB03FB089A19F80B30934268
:10EB900014D1474B98479AF800306FF00302D21A0D
:10EBA000099FFF238218019302930393CDF80080FD
:10EBB000FBB202202946D2B23E4FB84719F80B707B
:10EBC0003D4B3F2F15D9B27F2846C4EB020CDCF138
:10EBD000000242EB0C0239499847B27F2846C4EB49
:10EBE000020EDEF10002364942EB0E02354B984729
:10EBF0001DE0B27F34497F017918171B7A4242EB3E
:10EC00000702284698472A4988479AF800306FF04B
:10EC10000302D21A82181620611E6B1C0090033862
:10EC20000190D2B2C8B2DBB2FF21284FB8471635E7
:10EC30000134EDB2E4B29DF82F30A3423FF669AF44
:10EC40001DE02BB9224B01201870FF23D3771EE063
:10EC5000089AFF2A09D00C22013B534319F80320DC
:10EC6000FF2A04BF089F09F80370F37F0C22013BC1
:10EC7000204602FB0392174CDBB2A047079007998E
:10EC8000012903D1124B1970FF23F37700200DB037
:10EC9000BDE8F08F8B010020256C0008DE05002008
:10ECA00099770008596B0008E95C0008E96B0008D7
:10ECB0005F610108FD59010801670008AA8F01087A
:10ECC000759201082567000810180020C58D0008FE
:10ECD0004600002039E80008880100202DE9F04FA7
:10ECE000804C89B094F821500746FF2D904640F0A3
:10ECF000D080084604F12002042104F121037A4E59
:10ED0000B04794F820303846784F00937849042370
:10ED10000DF11F02774EB04797F84A30002B3AD0DA
:10ED2000DFF83492C847744B824697F84AB0984748
:10ED30000646C8476FEA0B0BDA44721E431E0121D8
:10ED40000020D2B2009101905FFA8AF10290039004
:10ED5000DBB26A4EB04794F82030694E56F8230073
:10ED6000684B98478246C847674B97F84A201B78FC
:10ED700097F84A100095CB1A03EBD373C2EB6301EB
:10ED800094F820304118019556F8232050462B4620
:10ED9000C9B25E4DA847564B0A261D7874E094F818
:10EDA000201030464B1B594241EB0301584B98470A
:10EDB000032D4C4F64D897F82020564BC5EB020C1E
:10EDC000DCF1000253F8251042EB0C023046524BA6
:10EDD00098474DB997F864203D21D2F101023046A1
:10EDE00038BF00224D4B9847434B98474C4B06F198
:10EDF00015021B780092DB430022C3180192029295
:10EE00000392049205920221284632469BB2454F56
:10EE1000B847022D1AD0032D25D0012D30D198F8F6
:10EE20000070414B3F2F04D994F8202030463F49D1
:10EE300005E03F497F0194F8202030467918A2F17F
:10EE4000010EDEF1000242EB0E0218E094F82020E1
:10EE50003046A2F1020CDCF1000208F1040142EBA1
:10EE60000C02344B0BE094F82020334BA2F1030E3C
:10EE7000DEF10002304608F1080142EB0E0298472D
:10EE800016360135F6B2EDB29DF81F30AB4286D88A
:10EE900023E0032D21D8DFE805F002090D12274BEE
:10EEA00001201870FF2384F8213017E02448FF2345
:10EEB000244D08E024480432FF23244D03E0244875
:10EEC000244D0832FF23A847012806D11B4B187098
:10EED000FF2384F82130013800E0002009B0BDE8AC
:10EEE000F08F00BF8B010020256C0008643C0020DF
:10EEF000F3050020997700085F610108FD590108BA
:10EF00007C8D0108215D000838010020B55E0108F4
:10EF1000596B0008FCA10108016700089D67000803
:10EF200088010020E95C000825670008AA8F010815
:10EF300010180020616A0008C5690008460000201A
:10EF4000A69301082DA4000859920108A9A9000858
:10EF50007A920108A5A60008636101082DE9F04F27
:10EF60009146744A8DB0089392F823300446FF2BE3
:10EF7000164640F0B38008462232112106F12303E1
:10EF80006D4DA8476D4D96F82230079000932046AE
:10EF900029466B4C0DF12F021123A0472C780A252E
:10EFA00096E096F82210674B0A1B514241EB020192
:10EFB0002846DFF89CB19847D847DFF8BCA105F197
:10EFC00015019AF800304FF00008DB438AB2C318ED
:10EFD00009910092CDF80480CDF80880CDF80C801E
:10EFE000CDF81080CDF81480204602212A469BB22D
:10EFF000554FB8475CB94F4B284693F82210C8EBE1
:10F000000103594241EB0301504B98475CE0102C3F
:10F010005AD8631E4FF00C0B0BFB03FB089A19F830
:10F020000B30934214D14A4B98479AF800306FF056
:10F030000302D21A099FFF238218019302930393BC
:10F04000CDF80080FBB202202946D2B2414FB8472A
:10F0500019F80B70404B3F2F17D996F822202846FD
:10F06000C4EB020CDCF1000242EB0C023B49984776
:10F0700096F822202846C4EB020EDEF10002384941
:10F0800042EB0E02374B98471EE096F82220364995
:10F090007F017918171B7A4242EB070228469847EE
:10F0A0002B4988479AF800306FF00302D21A821871
:10F0B0001620611E6B1C009003380190D2B2C8B2BA
:10F0C000DBB2FF21294FB84716350134EDB2E4B267
:10F0D0009DF82F30A3423FF664AF1FE033B9244BB5
:10F0E00001201870FF2382F8233020E0089AFF2ABD
:10F0F00009D00C22013B534319F80320FF2A04BF17
:10F10000089F09F8037096F823300C22013B204633
:10F1100002FB0392174CDBB2A04707900799012925
:10F1200004D1134B1970FF2386F8233000200DB053
:10F13000BDE8F08F8B010020256C0008C805002079
:10F1400099770008596B0008E95C0008E96B000832
:10F150005F610108FD59010801670008AA8F0108D5
:10F160008092010825670008101800206D8C0008A7
:10F1700046000020DDEC0008880100202DE9F04F5A
:10F180009F4C89B094F825608046FF2E154640F0CC
:10F190007E81084604F124020D2104F12503994FD4
:10F1A000B84794F824304046DFF8AC820093964983
:10F1B0000D230DF11F02954FB84798F84A30002BE8
:10F1C0003AD0DFF89892C847914B824698F84AB0F7
:10F1D00098470746C8476FEA0B0BDA447A1E431E6E
:10F1E00001210020D2B2009101905FFA8AF10290D1
:10F1F0000390DBB2874FB84794F82430864F57F816
:10F200002300864B98478246C847854B98F84A208A
:10F210001B7898F84A100096CB1A03EBD373C2EB15
:10F22000630194F824304118019657F82320504682
:10F230003346C9B27B4EB047734B0A2693F8008021
:10F240001FE194F824103046C8EB0102514241EB13
:10F250000201754B9847B8F10C0F694F00F20B8112
:10F2600097F82420714B304653F82810C8EB02035E
:10F270005A4242EB03026E4B9847B8F1000F09D196
:10F2800097F864203D21D2F10102304638BF0022B8
:10F29000684B98475E4B9847674B06F115021B7801
:10F2A0000092DB430022C31801920292039204925F
:10F2B00005929BB2404602213246604FB84708F1A2
:10F2C000FF330A2B00F2D780DFE813F00B001C009D
:10F2D0002800350048004F00620069007C00830070
:10F2E000CA002F78564B3F2F04D994F8242030467B
:10F2F000544905E054497F0194F824203046791898
:10F30000012A78E094F82420291DA2F1020CDCF1F6
:10F310000002304642EB0C024C4BABE094F8242048
:10F320003046A2F1030EDEF1000205F1080142EBC6
:10F330000E02474B9EE02A7B414B3F2A04D994F8AA
:10F34000242030463F4907E04249182000FB0211C3
:10F3500094F8242030460431042A4CE094F8242008
:10F36000304695F90D10052A80E0AA7B344B3F2AE0
:10F3700004D994F824203046324907E03549182052
:10F3800000FB021194F8242030460431062A32E0B2
:10F3900094F82420304695F90F10072A66E02A7C5D
:10F3A000274B3F2A04D994F824203046254907E00A
:10F3B0002849182000FB021194F82420304604311B
:10F3C000082A18E094F82420304695F91110092AEB
:10F3D0004CE0AA7C1A4B3F2A04D994F824203046EA
:10F3E000184907E01B49182000FB021194F824205B
:10F3F000304604310A2A14BF002201223AE000BF3D
:10F400008B010020256C0008BD05002099770008BD
:10F410005F610108FD590108A8A20108215D0008EB
:10F4200038010020B55E0108596B00089C8C01086A
:10F43000016700089D67000888010020E95C00085A
:10F4400025670008AA8F010810180020616A0008CB
:10F45000C56900080C200020643C0020636101089D
:10F4600094F8242095F9131030460B2A2E4B14BF24
:10F47000002201229847163608F10108F6B25FFA19
:10F4800088F89DF81F3043453FF6DBAE47E00C2E71
:10F4900045D8DFE806F0070E10151A1D202326298F
:10F4A0002C313600214B01201870FF2384F82530C1
:10F4B00036E01F481DE01F480432FF231E4D24E0A4
:10F4C0001E480832FF231E4D1FE01E480C3210E07C
:10F4D0001D480D3212E01D480E320AE01C480F3262
:10F4E0000CE01C48103204E01B48113206E01B48B7
:10F4F0001232FF231A4D08E01A481332FF231A4D27
:10F5000003E01A481A4D1432FF23A847012806D1F8
:10F51000064B1870FF2384F82530013800E00020E6
:10F5200009B0BDE8F08F00BF6D67000846000020FD
:10F530008992010859920108A9A90008949201082A
:10F54000A5A600089C920108A9920108B89201089A
:10F55000C5920108D4920108E1920108F0920108D5
:10F5600029730008FD920108F57300080C93010847
:10F5700015A000082DE9F04F9E4C9F4B99B00D4609
:10F5800098472378072B0BD19C4B34211A789C4B3E
:10F590009C4801FB02322946083200239A4D0CE0B8
:10F5A000082B13D1954B34211A78984B984801FBBE
:10F5B00002322946974D04320023A847012841F022
:10F5C000D881FF232370013801F0D4B9012D924B6B
:10F5D00004D11A78013D01321A7006E0022D04D1DF
:10F5E0001A7812B1013A1A70023D1B78AB460A93A1
:10F5F0001C46C1E2342202FB059202F5A45101F13E
:10F60000300318793F2810D83831087A84420AD05C
:10F61000897A8C4207D002F5A65211798C4202D029
:10F620009279944201D11B790EE00135EDB23F2D64
:10F63000DFF8F89108D8794988470A9AAB1A162258
:10F64000534325338342D5DBDFF8E481C0470B9B6E
:10F650001822DBB20C930C9D16236B4302FB049221
:10F66000DBB20D930B33DBB24638FF27C0B2991DD6
:10F6700002F50262099300973B460197C9B20C322A
:10F68000674E0890B047DDF820C00998ACF1050A34
:10F6900000F10A0600255FFA8AFAF6B22B465046B8
:10F6A00031460322009501975E4FB847C047DDF809
:10F6B00024C040080CF10907FFB22C305246DFF895
:10F6C00068C139463B46009501950295C0B2E047B6
:10F6D000C04740082C305246009501950295C0B2B3
:10F6E00031463346504DA847C0474508EDB22C354A
:10F6F000DFF83481A246CDF838B04FE1342202FB66
:10F70000049202F5A45292F8341002F130033F291A
:10F7100000F2338192F8401038328A453AD11B7991
:10F72000527A0A2152B292FBF1F211B200291FFA69
:10F7300082FBE8B217DA6E215943C9B200916FF02B
:10F7400019015943C9B201916FF06E014B43C2F1E7
:10F75000000B1FFA8BFBDBB200EB0B020293394666
:10F76000D2B23B4612E06E215943C9B200916FF00C
:10F7700019015943C9B201916FF06E014B4300EB7F
:10F780000B02DBB202933146D2B23346C047013599
:10F790005D44ADB2342303FB049303F5A45393F803
:10F7A000421003F138028A455BD130331B79D27A9B
:10F7B0000A2152B292FBF1F211B200291FFA82FB28
:10F7C000E8B237DA6E215943C9B200916FF01901DE
:10F7D0005943C9B201916FF06E014B43C2F1000B66
:10F7E0001FFA8BFBDBB200EB0B0202933946D2B25D
:10F7F0003B4632E082010020B95C0008870100200E
:10F80000A42C00200C93010815A00008942C0020C3
:10F81000678F01087DF10008C605002063610108BB
:10F820006D5E0108315F0108015D0108E4170020E9
:10F830005F6101086E215943C9B200916FF019014F
:10F840005943C9B201916FF06E014B4300EB0B02BB
:10F85000DBB202933146D2B23346C04701355D4434
:10F86000ADB2342303FB049303F5A65211798A4504
:10F870003DD103F5A45330331B7952790A2152B29A
:10F8800092FBF1F211B200291FFA82FBE8B217DAFB
:10F890006E215943C9B200916FF019015943C9B2A1
:10F8A00001916FF06E014B43C2F1000B1FFA8BFB0D
:10F8B000DBB200EB0B0202933946D2B23B4612E0B8
:10F8C0006E215943C9B200916FF019015943C9B271
:10F8D00001916FF06E014B4300EB0B02DBB2029320
:10F8E0003146D2B23346C04701355D44ADB2342310
:10F8F00003FB049303F5A65291798A453DD103F5A4
:10F90000A45330331B79D2790A2152B292FBF1F21F
:10F9100011B200291FFA82FBE8B217DA6E215943AF
:10F92000C9B200916FF019015943C9B201916FF04A
:10F930006E014B43C2F1000B1FFA8BFBDBB200EBF5
:10F940000B0202933946D2B23B4612E06E21594374
:10F95000C9B200916FF019015943C9B201916FF01A
:10F960006E014B4300EB0B02DBB202933146D2B285
:10F970003346C04701355D44ADB20134E4B23F2C9B
:10F980000AD8DFF874C2E0470A991622631A534373
:10F9900025338342FFF6B2AE0135ADB2089A531F4C
:10F9A0009D4201DA0A9CEAE7874BDDF838B09847B8
:10F9B0004008FF2500232C30052200933146C0B2B9
:10F9C000824F0195B847DFF800C2E0477E490746FD
:10F9D00088477F08420829372F3231463346F8B22C
:10F9E000D2B2009501950295C047774A9047764B71
:10F9F00006469847099F420876082C36F91D2C3296
:10FA000007F10D03C9B2009501950295F0B2D2B28B
:10FA1000DBB2C047BAF10F0F544607F10E0109D807
:10FA2000009501950898C9B2694A2B46DFF8A8C12C
:10FA3000E0471FE0BAF11F0F08D8009501952B464B
:10FA40000898C9B2634A644DA84713E0BAF12F0F72
:10FA500008D8009501950898C9B2604A2B465E4EB9
:10FA6000B04707E0009501950898C9B25C4A2B465B
:10FA7000594FB847544FB8475A480378013BDBB257
:10FA8000032B77D8B8470B9906468DB2B8474FF08D
:10FA90001608710808FB05F6013508FB05F5083561
:10FAA000ADB20A36831F0095C9B200254FF6FE722B
:10FAB0002C3106EA02029BB24B4E0195029503954A
:10FAC000049505952046B047B8470646B8470C9FB1
:10FAD0000D9A7B1C08FB03F876082C3602F10A010C
:10FAE00008F10803821FFF20019002900390009507
:10FAF000F0B201F0FE01D2B203F0FE033B4EB0477C
:10FB0000BBF1630F36D93A4BABF1640B83F800B00D
:10FB1000344B1B78012B09D1364B34221B7802FB66
:10FB2000039909F5A45383F840B022E0022B09D1D0
:10FB3000304B34221B7802FB039909F5A45383F858
:10FB400042B016E0032B09D12A4B34221B7802FB6A
:10FB5000039909F5A65383F804B00AE0042B08D1F1
:10FB6000244B34221B7802FB039909F5A65383F832
:10FB700006B0AB460134E4B23F2C0FD8DDF828C004
:10FB80001D4DCCEB040CCDF82CC0A8470B991623C7
:10FB90004B432533834201DA0A9D48E50A9A6FF008
:10FBA00019035343DBB208936FF06E035D46534372
:10FBB0004FF06E0B0BFB02FBDBB25FFA8BFB099382
:10FBC0009146A846CCE000BF5F610108315F0108A3
:10FBD00012930108199301086D5E01082093010832
:10FBE0002893010882010020E95C0008FD59010802
:10FBF000BE00002087010020636101081A33DFB2D4
:10FC0000DFF88CA20C934FEA49123B1FFF25DBB2B1
:10FC1000524419462C320B930A202B46934C944E97
:10FC200000950195A047B047089B4208099C4C3AB3
:10FC30003C20019302943946D2B23B468D4CCDF81C
:10FC400000B0A047DFF84CC2002403223C20394614
:10FC50002346CDF81CC000940195E047B04740080A
:10FC60004C38C0B203222346DDF81CC00094019535
:10FC70003946E047DFF810C260460378062B5BD8B0
:10FC80009CF900304FF006429A4055D50C99CDF8BA
:10FC90001CC08AB2131F1A3292B200924FF6FE7243
:10FCA0000A2103EA020201946E230294039404944D
:10FCB00005944846704EB04707F11A0300940A2095
:10FCC0006E220195029503950B9903F0FE036B4C90
:10FCD000A047B8F1630FDDF81CC02DD9684BA8F11F
:10FCE000640883F800809CF800304BB9654B3422DF
:10FCF0001B7802FB03AA0AF5A45383F8348016E0AC
:10FD0000052B09D15F4B34221B7802FB03AA0AF5AD
:10FD1000A45383F838800AE0062B08D1594B3422CB
:10FD20001B7802FB03AA0AF5A45383F83C80564AC9
:10FD3000FF2313704FF000084D4B9847089C099D16
:10FD4000A4F11A03DBB20893A5F16F0309F10109CD
:10FD50000BF16E0BDBB25FFA89F95FFA8BFB09934B
:10FD6000B9F13F0F0BD8494B0A9E9847C6EB0904DF
:10FD70001623634303F125028242FFF63FAF454657
:10FD80000C95DDF82880BAE2414A342303FB0823AE
:10FD900003F5A45393F834A09346BAF13F0F37D834
:10FDA000334CA0478146A0476E2303FB0AF3DBB226
:10FDB00000936FF0190303FB0AF3DDF828C0DBB2F0
:10FDC000CCEB0A0101936FF06E034D4303FB0AF382
:10FDD00042081A364FEA5909F6B205F11A01DBB2A8
:10FDE000A9F14C092C3A01F0FE01D2B202935FFA5C
:10FDF00089F033461F4DA847A0474008FF222C3802
:10FE0000002301920093C0B23146FC3A214CA04736
:10FE10004FF0160909FB07F7FFB207F10F095FFA68
:10FE200089F9CDF8249007F1130908975FFA89F949
:10FE30000125032D4FF0340310D0042D2CD003FBEB
:10FE400008B3022D03F5A45315BF93F8404093F86F
:10FE5000424093F841C093F843C024E003FB08B349
:10FE600003F5A6531C7993F805C01CE06D5E0108EC
:10FE70005F610108015D0108E95C0008FD590108A6
:10FE8000BE0000208701002082010020636101087C
:10FE9000E4170020315F010803FB08B303F5A65304
:10FEA0009C7993F807C0342303FB08B303F5A453EC
:10FEB00030331B794FFA8CFC3F2B88BF4FF0000A80
:10FEC0003F2C7AD8CDF81CC0644FB8470646B847D7
:10FED0006E2101FB0AF1C9B200916FF0190101FB1B
:10FEE0000AF142080A98C9B2241A162301916FF048
:10FEF0006E01634301FB0AF1760821362C3215337B
:10FF0000C9B2F0B2D2B2DBB20291554C4946A04719
:10FF1000B847400800241C30052249462346009477
:10FF20000194C0B24F4EB047B847A9F10503DBB208
:10FF30000B930646B84773084208163B01211C3252
:10FF400009F10506D8B2D2B2F3B20091019402943D
:10FF500003940B99444EB0474449454B10A8984729
:10FF6000444A10A8904710AE01232246009330184F
:10FF7000234629B2404EB0474049414E10A8B047F1
:10FF80003C4910A88847DDF81CC0012210AB0FFACD
:10FF90008CF10092181822462346374CA047394965
:10FFA00010A8B047B8474008FF23133800930193C7
:10FFB000C0B20B9910AA344CA0470135ADB209F17B
:10FFC0000409052D5FFA89F97FF433AF234FB84751
:10FFD000342606FB08F60BEB0604410804F5A4548E
:10FFE0005E44343414232C3906F5A456009320467D
:10FFF0000233264C3036C9B2099AA047357A3C46BE
:020000040801F1
:10000000FD2D02D110A8224918E0FF2D12D121495F
:10001000174B10A89847204B10A89847B84740089E
:100020002838099900950195C0B210AA2B46164DA3
:10003000A847A1E0FE2D33D1184910A80C4B9847D2
:10004000154B10A89847B8474008FF23283800935D
:100050000193C0B2099910AAE9E700BF5F610108E6
:10006000015D0108315F0108FD5901083093010865
:10007000F5030008B1040008655200087E8E0108EF
:10008000D1010008E68E01086D5E0108757F000849
:1000900034930108389301083D5E01083C93010840
:1000A0003F2D69D89D499E4B10A898479D4F10A899
:1000B000B847B17A00224FF001090DF1400C134608
:1000C000CDF80090604449B2DFF874A2D047DFF861
:1000D00074C29549CDF81CC010A8E04710A8B847D5
:1000E000717A10AA101800221346CDF8009049B278
:1000F000D047DDF81CC08D4910A8E0478C4B10A8F4
:100100009847A047099B400803F104095FFA89F961
:10011000FF272838A9F10401C9B210AA3B46854E31
:1001200000970197C0B2B047A0470A9E1621AB1BAB
:1001300059436E236B43DBB200936FF019036B439B
:10014000DBB201936FF06E035D434208EDB21A31EA
:100150002C3A01F0FE01D2B24B4602953C20764D7E
:10016000A847A04740082C38002300930197C0B24D
:1001700049460322714DA847342606FB08BB0BF500
:10018000A45638363579FD2D1FD16449644B10A82B
:100190009847644B10A8984771790022012310AF4B
:1001A000009349B213463818654DA8475F49654B1F
:1001B00010A898475E4B10A89847A047DDF820C0CC
:1001C000400828380CF11B0126E0FF2D15D15E49AF
:1001D000534B10A89847564B10A89847A047089A29
:1001E000400802F11B01283800950195C0B2C9B240
:1001F00010AA2B464F4CA0477DE0FE2D13D153494A
:10020000474B10A898474A4B10A89847A047089B0F
:100210004008283803F11B01FF2300930193C0B26B
:10022000C9B210AAE6E73F2D65D83C493C4B10A85F
:1002300098473C4F10A8B847B1790DF1400C002207
:100240004FF0010960441346CDF8009049B2DFF841
:10025000F0A0D047DFF8ECB0334910A8D84710A879
:10026000B847717910AA101800221346CDF80090F3
:1002700049B2D0472D4910A8D8472D4B10A8984710
:10028000A047089B400803F11F095FFA89F9FF277F
:100290002838A9F10401C9B210AA3B46254E00979F
:1002A0000197C0B2B047A0470A9E1621AB1B594325
:1002B0006E236B43DBB200936FF019036B43DBB229
:1002C00001936FF06E035D434208EDB21A312C3A90
:1002D00001F0FE01D2B24B4602953C20164DA847D4
:1002E000A04740082C38002300930197C0B249462C
:1002F0000322124CA04708F101085FFA88F8B8F110
:100300003F0F25D90A9F16227B4253434FF0000C22
:100310009BB20C9D0E93CDF820C029E0EA84010821
:10032000F5030008B10400083F930108E68E0108B8
:100330003D5E01086D5E0108015D0108315F010845
:1003400065520008D1010008E58E010843930108B9
:100350000A98064BC0EB08079847162505FB07F6D9
:1003600006F125038342FFF60FADCBE76361010879
:10037000DFF8ACA208999AF8003057468B421BD19F
:10038000A44CA0470646A047089A0A9C1621131BB6
:1003900059430F314208C9B2002076082C3E163A64
:1003A00001F116030090FF30019002900390D2B249
:1003B000F0B2DBB2984CA0479AF80090B9F1FF0F69
:1003C0003ED1DFF85082C0470446C0470E9E610808
:1003D0004308C9B206F12500DBB200242C3906F12E
:1003E0000F02163B80B289B292B29BB200908B4E44
:1003F000019402940394049405940898B047C0476C
:100400000646C047DDF838C042085FFA8CF376082C
:100410002C3E03F10F01163A2533F0B20094CDF8CB
:100420000490CDF80890CDF80C90C9B2D2B2DBB2EE
:10043000794EB047632D03D9794B643D1D70254635
:1004400078480678FF2E40F076829AF800300899B6
:100450008B4240F070826F4CA0478046A047089ABC
:10046000DDF828C04FF0160ACCEB02030AFB03FAB2
:100470000AF11A0A5FFA8AF942084FEA580801217C
:10048000A8F12108613209F17E03009101960296DC
:1004900003965FFA88F04946D2B203F0FE035E4E3F
:1004A000B047614814211FFA8AFA0F9009914FF062
:1004B000000B584EB0470446B04709F10D03DBB2BC
:1004C0000B93420863080124213B2F320094013C26
:1004D000D8B24946D2B20B9BDFF83CC101940294DA
:1004E0000394E047B04709F10203DBB219464FF02D
:1004F000FF080C930F9BCDF80080CDF8048053F8D3
:10050000042F40081F38DFF828C10F93C0B24346BC
:10051000E047B0470790B047079B0AF10D02590822
:10052000C9B2430892B22139DBB20D9200922F3347
:10053000019402940394049405945FFA8BF089B2B9
:100540005246DFF8D8C0E047BBF1050F7FD1B04776
:100550000790B047079B52465B08D9B243080D98F5
:10056000DBB233316133DFF8B4C000900194029400
:100570000394049405940998E047B0470790B04766
:10058000079B42085B083333012061324946D2B2EF
:10059000DFF884C000900194D8B202940B9B0394BE
:1005A000E047B047400835300C99204A4346DFF811
:1005B00080C0CDF80080CDF80480C0B2E047B047DD
:1005C0000790B047099B079903F10A0249084308BD
:1005D0000D98C9B2DBB265319333DFF840C00090AB
:1005E00001940294039404940594D0B25246E047D7
:1005F000B0470790B047079B42085B08653301206E
:100600006D3A4946D2B200900194D8B20294039454
:100610000B9B0FE05F610108FD590108E95C0008D0
:10062000870100208201002044000020FC9801087E
:100630006D5E01089F4CA047B04740086730CDF879
:100640000080CDF80480C0B20C999B4A74E0BBF1E5
:10065000060F37D1B0470790B0470799DDF824C09F
:10066000430849080D980CF11402C9B2DBB2DFF857
:1006700064C29731C53300900194029403940494AA
:100680000594D0B25246E047B0470790B047079B69
:1006900042085B08693B01203B3A4946D2B20090D0
:1006A0000194D8B2029403940B9B824CA047B047AC
:1006B00040086738CDF80080CDF80480C0B20C99AE
:1006C0007E4A39E0BBF1050F39D8B0470790B047F3
:1006D0000799DDF824C0430849080D98ACF10A02D7
:1006E000C9B2DBB2DFF8ECC1333161330090019461
:1006F0000294039404940594D0B25246E047B04764
:100700000790B047079B42085B08333301206132F2
:100710004946D2B200900194D8B2029403940B9B44
:10072000644CA047B047400835300C99644ACDF876
:100730000080CDF80480C0B24346624EB0478B2D96
:1007400021D97435EDB2052D0AD15F4A3B783421A9
:1007500001FB0323FD2203F5A45383F838200BE0AB
:10076000062D09D1584A3B78342101FB0323FD2291
:1007700003F5A45383F83C20544A5548FF233B70AB
:1007800013700370C0E0812D21D97E35EDB2052DA7
:100790000AD14D4A3B78342101FB0323FF2203F5A4
:1007A000A45383F838200BE0062D09D1464A3B7844
:1007B000342101FB0323FF2203F5A45383F83C20DB
:1007C000424A4349FF233B7013700B709CE0772D26
:1007D00021D9783DEDB2052D0AD13B4A3B78342131
:1007E00001FB0323FE2203F5A45383F838200BE01A
:1007F000062D09D1344A3B78342101FB0323FE2224
:1008000003F5A45383F83C20304AFF231370304A89
:100810003B70137078E06D2D71D96E3DEDB255B916
:10082000294A3B78342101FB0323FF2203F5A4531B
:1008300083F834205CE0012D0AD1234A3B7834212F
:1008400001FB0323FF2203F5A45383F840204FE06C
:10085000022D0AD11C4A3B78342101FB0323FF22DD
:1008600003F5A45383F8422042E0032D09D1164A30
:100870003B78342101FB0323FF2203F5A6531A71B1
:1008800036E0042D09D1104A3B78342101FB0323C3
:10089000FF2203F5A6539A712AE0052D1CD10A4ABE
:1008A0003B78342101FB0323FF2203F5A45383F893
:1008B00038201DE0FD590108499301084D930108B6
:1008C000519301086D5E0108E4170020BE0000206E
:1008D00082010020E95C0008062D09D1274A3B78F7
:1008E000342101FB0323FF2203F5A45383F83C20AA
:1008F000234A244CFF233B701370237004E0632DC4
:1009000003D9204E643D35700025DDF824C00BF17D
:10091000010B1FFA8BFB0CF1010309F10E090AF11F
:100920000E0ADBB2BBF1090F5FFA89F91FFA8AFAE6
:1009300009937FF4BEAD08980E99431CDBB208936F
:10094000089A01F116039BB2402A0E937FF410AD72
:10095000042D0ED13B780A4AFF2B04D1094C1370A9
:100960002370012006E00849064DFF230B70137029
:100970002B70002019B0BDE8F08F00BFE4170020F5
:10098000BE00002082010020870100202DE9F04FE9
:100990009046714A994692F827308BB0FF2B074654
:1009A000164640F0AE8008462632412106F1270364
:1009B0006A4CA0476A4D96F8263007900093294666
:1009C000684C38460DF127024123A0472C780A25B0
:1009D00091E096F82610644BC4EB010CDCF10001A9
:1009E00041EB0C012846DFF8A8A19847D0475F49A2
:1009F00005F115020B780092DB430022C318019227
:100A00000292039204920592594F204602212A46EF
:100A10009BB2B847DFF840B157464CB99BF8261057
:100A20002846D1F1010138BF0021524B98475EE0C2
:100A3000402C5CD8631E4FF0340A0AFB03FA18F806
:100A40000AE09BF82620BEF1FF0F4B4B02D128464F
:100A50004A4910E0BEF1FE0F02D1284648490AE09B
:100A6000BEF13F0F05D847494FEA4E1E2846714454
:100A700001E045492846C4EB020EDEF1000242EBDC
:100A80000E029847B8473949631E0A786FF0010192
:100A9000891A41181320009096F826006A1C071B3B
:100AA000784240EB07000190C9B2D8B2D2B2162307
:100AB000364FB847B9F1FF0F19D018F80A304B4537
:100AC00015D1334B9847294B6FF001021B78002159
:100AD000D21A821805F115030091FF31019102919C
:100AE000039102202946D2B2DBB22A4FB84716350D
:100AF0000134EDB2E4B29DF82730A3423FF669AF6E
:100B00001EE033B9244B01201870FF2382F82730F0
:100B10001FE0B9F1FF0F08D03422013B534318F80E
:100B20000320FF2A08BF08F8039096F827303422E4
:100B3000013B02FB03823846DBB2184CA04707900A
:100B4000079A012A04D1144B1A70FF2386F8273024
:100B500000200BB0BDE8F08F8B010020256C000851
:100B6000C005002099770008596B00088801002013
:100B7000E95C0008E96B0008016700086D8F010857
:100B80007C8F010810180020AA8F01083185000809
:100B90005F610108FD590108460000207DF1000851
:100BA0002DE9F04F934C8BB0667C8046FF2E1546A6
:100BB0009B4640F07181084604F110020E2104F1B9
:100BC00011038D4FB847237C4046DFF884820093A1
:100BD0008A490E230DF12702894FB84798F84A3009
:100BE000002B39D0DFF86C92C84798F84A30854A14
:100BF0000793824690470746C847079B7A1EDB4308
:100C00009A440121431E0020D2B2009101905FFA64
:100C10008AF102900390DBB27B4FB847237C7B4F75
:100C200057F823007A4B98478246C847794B98F883
:100C30004A201B7898F84A100096CB1A03EBD3731E
:100C4000C2EB6301237C4118019657F823205046DC
:100C50003346C9B2704EB047684B4FF00B0A93F859
:100C6000008010E1217C3046C8EB0103594241EB82
:100C700003016A4B9847B8F10D0F5E4F00F2FB80FD
:100C80003A7C674BC8EB0209D9F1000253F82810EF
:100C900042EB09023046634B9847B8F1000F09D187
:100CA00097F864203D21D2F10102304638BF00227E
:100CB0005D4B9847534B5D4F079398473A786FF0D9
:100CC0000309C2EB0909079B814498473B7806F169
:100CD0001502DB43C3180092002201920292039294
:100CE000049205929BB2404602213246504FB847CB
:100CF00008F1FF335FFA89F90C2B00F2BC80DFE8C2
:100D000003F007121D2930373D44505B656FAB007F
:100D1000227C3046A2F1010CDCF10002294642EBB4
:100D20000C02444B08E0227C95F912103046022A4E
:100D3000414B14BF0022012298479CE0227C3046A0
:100D4000A2F1030EDEF1000295F9131042EB0E0240
:100D5000354BF1E7237C0222304695F91410042B21
:100D600019E0237C0322304695F91510052B12E07B
:100D7000227C304695F91610062AD9E7237C0122F9
:100D8000304695F91A10072B05E0237C95F91B10C6
:100D900005223046082B14BF00230123274EB047FD
:100DA00069E0227C3046A2F10906724205F11C017D
:100DB00042EB0602224BBFE716230093033B01934D
:100DC000FF2059464A4653461E4E53E016230093D1
:100DD000033B0193FF2059464A4653461A4E49E0C9
:100DE00016230093033B0193FF2059464A4653467E
:100DF000164E3FE08B010020256C0008DA0500202C
:100E0000997700085F610108FD59010870A2010887
:100E1000215D000838010020B55E0108596B00080B
:100E200020A40108016700089D67000888010020D0
:100E3000E95C0008256700086D670008E96700089D
:100E4000C56900086D8C0008C58D0008018F000879
:100E5000643C00206361010813230093237C3A4E15
:100E6000A3F10D02534243EB020301935846494656
:100E700052461623B04708F101080AF1160A5FFA34
:100E800088F85FFA8AFA9DF827300AF1FF36434561
:100E9000F6B23FF6E7AE52E00D2E50D8DFE806F08E
:100EA000070D1114191C2126292E33383D42274BDA
:100EB00001201870FF23637442E02548FF23254D6D
:100EC00034E0254812320EE024481332FF23244D2B
:100ED0002CE0244814320EE023481532FF23234D22
:100EE00024E023481632FF23224D1FE022481A3205
:100EF00001E022481B32FF23214D17E021481C321C
:100F0000FF23214D12E02148214A5B46214D0DE08F
:100F10002148224A5B46224D08E02248224A5B468D
:100F2000224D03E02248234A234D5B46A84701286F
:100F300005D1064B1870FF236374013800E00020D0
:100F40000BB0BDE8F08F00BF5580000846000020C0
:100F5000D29D0108C5620008928F0108FA98010825
:100F6000E56D000857930108F78F010899D900082B
:100F700062930108F5730008929401086A930108CE
:100F8000995D000876930108A5A60008118F010855
:100F9000982A00205DEF00080C8F0108D829002056
:100FA000D1EA00081A8F0108582B002029E6000812
:100FB000678F0108982C00208D0901082DE9F04F5A
:100FC0008DB009928A4A0546D37CFF2B40F0F5800C
:100FD0001232531C0846874C4121A047844A864C54
:100FE000937C0790009328462146844D0DF12F02F3
:100FF0004123A84724780A25D9E07D4B2846997CCF
:101000007F4BC4EB010CDCF1000141EB0C01984774
:101010007C4A90477C4A4FF00009137805F115028D
:10102000DB43C3180092CDF80490CDF80890CDF8BA
:101030000C90CDF81090CDF81490204602212A464D
:101040009BB2724EB0475CB9694B2846997C704B95
:10105000C9EB010EDEF1000141EB0E019847A2E061
:10106000402C00F2A080099A04F1FF3A4FEA4A139B
:10107000D31808935E4B08999A7C2846161B724237
:1010800042EB0602634B98475E4A90475E4A4FF038
:1010900013081378564ACDF800806FF0030BC3EBAA
:1010A0000B0B937C8344191B6E1C4B4243EB0103D7
:1010B0005FFA8AFAF6B25FFA8BFB59460193324621
:1010C0001623554F5046B847C0EB0B0B5FFA8BFC0D
:1010D0004FF0160B6246FF20514633464F4FCDF876
:1010E00018C0CDF800B0CDF80480B847DDF818C0BE
:1010F0005146C0EB0C0C5FFA8CFC6246FF20334675
:10110000474FCDF818C0CDF800B0CDF80480B847EF
:10111000DDF818C05146C0EB0C0C5FFA8CFC62463F
:10112000FF2033463F4FCDF818C0CDF800B0CDF8C2
:101130000480B8472E4ACDF80080937CDDF818C0B3
:101140001A1B5342C0EB0C0C43EB02035FFA8CFCFE
:10115000614632460193344F5B46CDF818C0504685
:10116000B847DDF818C0274BC0EB0C0C5FFA8CF7C2
:101170009847254B1A786FF003039B1A1B189F4260
:1011800011D1089A163F92F91230FFB264210093F0
:1011900002960197CDF80CB0CDF8108023480A468E
:1011A0004B46234EB04716350134EDB2E4B29DF8FC
:1011B0002F30A3423FF621AF0EE02BB91D4B01208B
:1011C0001870FF23D37410E0099C013B5A01A21848
:1011D000DBB2194CA0470790079A012A04D1154B9E
:1011E000034C1A70FF23E37400200DB0BDE8F08FAC
:1011F0008B010020256C0008E0050020997700088D
:10120000596B00085F61010888010020E95C000853
:10121000E96B000801670008558000086D8C000824
:10122000C58D0008018F0008CD9200087D9301084C
:10123000CD88000846000020A10B01082DE9F04FE1
:10124000864C89B094F829500746FF2D904640F00F
:10125000D880084604F12802052104F12903804EB4
:10126000B04794F8283038467E4F00937E490523D6
:101270000DF11F027D4EB04797F84A30002B3AD04F
:10128000DFF85092C8477A4B824697F84AB09847A1
:101290000646C8476FEA0B0BDA44721E431E012153
:1012A0000020D2B2009101905FFA8AF1029003907F
:1012B000DBB2704EB04794F828306F4E56F82300DA
:1012C0006E4B98478246C8476D4B97F84A201B786B
:1012D00097F84A100095CB1A03EBD373C2EB630166
:1012E00094F828304118019556F8232050462B4693
:1012F000C9B2644DA8475C4B0A251E787BE094F880
:10130000281028468B1B594241EB03015E4B98473E
:10131000042E524F6BD897F828205C4BC6EB020C7A
:10132000DCF1000253F8261042EB0C022846584B21
:1013300098474EB997F864203D21D2F10102284622
:1013400038BF0022534B9847494B9847524B05F101
:1013500015021B780092DB430022C318019202920F
:101360000392049205929BB2304602212A464B4FCB
:10137000B847731E032B3AD8DFE803F0021B272E71
:1013800098F80020464B3F2A04D994F82820284694
:10139000444907E04449182000FB021194F8282032
:1013A00028460431A2F1010EDEF1000242EB0E02EA
:1013B0001CE094F828202846A2F102035A4242EB8E
:1013C000030208F10401394B10E094F82820284664
:1013D00008F10801032A05E094F82820284608F1BE
:1013E0000C01042A324B14BF002201229847163503
:1013F0000136EDB2F6B29DF81F30B3423FF67FAF33
:1014000027E0042D25D8DFE805F0030A0E131600A7
:10141000284B01201870FF2384F829301AE0264851
:10142000FF23264D0BE026480432FF23254D06E01E
:101430002548083201E025480C32254DFF23A847F6
:10144000012806D11B4B1870FF2384F8293001387E
:1014500000E0002009B0BDE8F08F00BF8B01002044
:10146000256C0008643C0020F005002099770008F6
:101470005F610108FD59010854A20108215D0008BF
:1014800038010020B55E0108596B0008408E010844
:10149000016700089D67000888010020E95C0008DA
:1014A00025670008AA8F01080C200020616A000847
:1014B000C569000846000020A6930108A1A5000800
:1014C00059920108A9A9000862920108C78E010873
:1014D000A5A60008636101082DE9F04F9146744A02
:1014E0008DB0089392F82B300446FF2B164640F03F
:1014F000B48008462A32112106F12B036D4DA8470E
:101500006D4D96F82A3007900093204629466B4C83
:101510000DF12F021123A0472C780A2597E096F8A9
:101520002A10674B0A1B514241EB02012846DFF8A3
:101530009CB19847D847DFF8BCA105F115019AF88E
:1015400000304FF00008DB438AB2C31809910092C3
:10155000CDF80480CDF80880CDF80C80CDF810804F
:10156000CDF81480204602212A469BB2554FB84739
:101570005CB94F4B284693F82A10C8EB0103594237
:1015800041EB0301504B98475DE0102C5BD804F110
:10159000FF3B4FEA0B1B19F80B30089A934214D10A
:1015A0004A4B98479AF800306FF00302D21A099F0D
:1015B000FF238218019302930393CDF80080FBB2BE
:1015C00002202946D2B2424FB84719F80B20414BAE
:1015D0003F2A17D996F82A202846C4EB020CDCF1E2
:1015E000000242EB0C023C49984796F82A20284614
:1015F000C4EB020EDEF10002384942EB0E02384B1A
:10160000984720E03749182000FB021196F82A205D
:101610000431171B7A4242EB0702284698472B49B0
:1016200088479AF800306FF00302D21A8218162009
:10163000611E6B1C009003380190D2B2C8B2DBB2BD
:10164000FF21294FB84716350134EDB2E4B29DF8B9
:101650002F30A3423FF663AF1DE033B9234B012087
:101660001870FF2382F82B301EE0089AFF2A08D05A
:10167000013B1B0119F80320FF2A04BF089F09F84A
:10168000037096F82B302046013B09EB0312184CEF
:10169000DBB2A04707900799012904D1134B1970B9
:1016A000FF2386F82B3000200DB0BDE8F08F00BF7F
:1016B0008B010020256C0008E605002099770008C2
:1016C000596B0008E95C0008E96B00085F610108DC
:1016D000FD59010801670008AA8F010883930108DA
:1016E000256700080C2000205D90000846000020BF
:1016F0003D120108880100202DE9F04F854C89B08A
:1017000094F82D500746FF2D904640F0D6800846AD
:1017100004F12C02052104F12D037F4EB04794F80B
:101720002C3038467D4F00937D4905230DF11F0273
:101730007C4EB04797F84A30002B3AD0DFF84C92F5
:10174000C847794B824697F84AB098470646C8473B
:101750006FEA0B0BDA44721E431E01210020D2B245
:10176000009101905FFA8AF102900390DBB26F4E14
:10177000B04794F82C306E4E56F823006D4B9847C6
:101780008246C8476C4B97F84A201B7897F84A1056
:101790000095CB1A03EBD373C2EB630194F82C30A2
:1017A0004118019556F8232050462B46C9B2634D87
:1017B000A8475B4B0A251E787AE094F82C1028463F
:1017C0008A1B514241EB02015D4B9847042E514F59
:1017D0006AD897F82C205B4B284653F82610931BA9
:1017E0005A4242EB0302584B98474EB997F864208F
:1017F0003D21D2F10102284638BF0022534B9847C1
:10180000494B9847524B05F115021B780092DB4378
:101810000022C318019202920392049205929BB295
:10182000304602212A464B4FB847731E032B3BD844
:10183000DFE803F0021B282F98F80020464B3F2AD0
:1018400004D994F82C202846444907E0444918203C
:1018500000FB021194F82C2028460431A2F1010C5F
:10186000DCF1000242EB0C021DE094F82C2028462B
:10187000A2F1020EDEF1000208F1040142EB0E02B9
:10188000384B10E094F82C20284608F10801032A70
:1018900005E094F82C20284608F10C01042A324B6C
:1018A00014BF00220122984716350136EDB2F6B278
:1018B0009DF81F30B34280D827E0042D25D8DFE8FB
:1018C00005F0030A0E131600284B01201870FF23A1
:1018D00084F82D301AE02648FF23264D0BE02648D9
:1018E0000432FF23254D06E02548083201E0254853
:1018F0000C32254DFF23A847012806D11B4B187039
:10190000FF2384F82D30013800E0002009B0BDE845
:10191000F08F00BF8B010020256C0008643C002084
:1019200016060020997700085F610108FD5901083B
:101930001CA30108215D000838010020B55E0108E4
:10194000596B000838A30108016700089D6700086B
:1019500088010020E95C000825670008AA8F0108BB
:101960000C200020616A0008C569000846000020BC
:10197000A6930108A1A5000859920108A9A9000889
:1019800062920108C78E0108A5A6000863610108DC
:101990002DE9F04F9146744A8DB0089392F82F309C
:1019A0000446FF2B164640F0B48008462E32112123
:1019B00006F12F036D4DA8476D4D96F82E30079018
:1019C0000093204629466B4C0DF12F021123A047AE
:1019D0002C780A2597E096F82E10674B0A1B514287
:1019E00041EB02012846DFF89CB19847D847DFF861
:1019F000BCA105F115019AF800304FF00008DB4357
:101A00008AB2C31809910092CDF80480CDF80880FD
:101A1000CDF80C80CDF81080CDF81480204602213E
:101A20002A469BB2554FB8475CB94F4B284693F8AE
:101A30002E10C8EB0103594241EB0301504B98476C
:101A40005DE0102C5BD804F1FF3B4FEA0B1B19F84B
:101A50000B30089A934214D14A4B98479AF80030B9
:101A60006FF00302D21A099FFF2382180193029399
:101A70000393CDF80080FBB202202946D2B2424F38
:101A8000B84719F80B20414B3F2A17D996F82E205A
:101A90002846C4EB020CDCF1000242EB0C023C498C
:101AA000984796F82E202846C4EB020EDEF100027D
:101AB000384942EB0E02384B984720E0374918204E
:101AC00000FB021196F82E200431171B7A4242EBDC
:101AD0000702284698472B4988479AF800306FF04C
:101AE0000302D21A82181620611E6B1C0090033864
:101AF0000190D2B2C8B2DBB2FF21294FB8471635E8
:101B00000134EDB2E4B29DF82F30A3423FF663AF4B
:101B10001DE033B9234B01201870FF2382F82F30CA
:101B20001EE0089AFF2A08D0013B1B0119F8032088
:101B3000FF2A04BF089F09F8037096F82F3020464B
:101B4000013B09EB0312184CDBB2A0470790079941
:101B5000012904D1134B1970FF2386F82F30002080
:101B60000DB0BDE8F08F00BF8B010020256C000890
:101B7000E405002099770008596B0008E95C00082B
:101B8000E96B00085F610108FD5901080167000861
:101B9000AA8F010887930108256700080C20002000
:101BA0009591000846000020F916010888010020E0
:101BB0002DE9F04F9C4C8BB094F831500746FF2D27
:101BC00090469B4640F00581084604F1300208210A
:101BD00004F13103954EB04794F830303846944FB5
:101BE0000093944908230DF12702934EB04797F8CC
:101BF0004A30002B3BD0DFF8C092C84797F84A30F4
